:100000000C946F220C94AF220C94AF220C94AF226C
:100010000C94AF220C94AF220C94AF220C94AF221C
:100020000C94AF220C94AF220C94AF220C94AF220C
:100030000C94AF220C94AF220C94AF220C94AF22FC
:100040000C94AF220C9427EC0C94AF220C94AF22AA
:100050000C94AF220C94F2EA0C94AF220D94224E31
:100060000C94AF220C948C5E0C94825E0C94AF22A4
:100070000C94AF220C94AF220C94AF220C94AF22BC
:100080000C94F2330C94AF220C94AF220C94AF2258
:100090000C94AF220C94AF220C94AF220C94AF229C
:1000A0000C94AF220C94AF220C94C4330C94AF2266
:1000B0000C94AF220C94AF220C94AF220C94AF227C
:1000C0000C94AF220C94AF220C94AF220C94AF226C
:1000D0000C94AF220C94AF220C94AF220C94AF225C
:1000E0000C94AF22084AD73B3BCE016E84BCBFFDC7
:1000F000C12F3D6C74319ABD56833DDA3D00C77FF8
:1001000011BED9E4BB4C3E916BAAAABE0000008090
:100110003F05A84CCDB2D44EB93836A9020C50B91F
:10012000918688083CA6AAAA2ABE000000803F004B
:100130000D94604D0D945C4D0D94E32A0D94915BEC
:100140000D94F3160D94974D0D94774D0D948D4DA0
:100150000D94934D0D94854D0D94E70E0D94894D9E
:100160000D94E22A0D94584D0D9480140D94BD57B2
:100170000D94CB5A0D94414D0D945F5A0D947F4DC3
:100180000D948B2B0D94674D0D94464D0D94DD5AB7
:100190000D949F570D94EC5A0D9438150D94CB1275
:1001A0000D94714D0D94644D0D946D4D0D947B4DDA
:1001B0000D94DE120D949D570D94B52A0D94BF1227
:1001C0004E414E494E495459494E46CDCCCC3D0A3C
:1001D000D7233C17B7D13877CC2B329595E6241F1F
:1001E000B14F0A000020410000C84200401C4620D8
:1001F000BCBE4CCA1B0E5AAEC59D7400407A10F3AB
:100200005A00A0724E18090010A5D4E80000E87644
:1002100048170000E40B54020000CA9A3B0000009B
:10022000E1F505000080969800000040420F0000B4
:1002300000A08601000000102700000000E8030075
:100240000000006400000000000A0000000000013F
:1002500000000000002C76D888DC674F0823DFC13F
:10026000DFAE59E1B1B796E5E3E453C63AE65199FA
:100270007696E8E6C28426EB898C9B62ED407C6F23
:10028000FCEFBC9C9F40F2BAA56FA5F490055A2ADA
:10029000F75C936B6CF9676DC11BFCE0E40D47FEE6
:1002A000F520E6B500D0ED902E03009435770500DB
:1002B00080841E080000204E0A000000C80C333362
:1002C00033330F986E12831141EF8D2114893BE671
:1002D0005516CFFEE6DB18D1844B381BF77C1D90FA
:1002E0001DA4BBE424203284725E228100C9F12463
:1002F000ECA1E53D27434F4D4D554E4943415449EF
:100300004F4E0044525952554E004552524F52538F
:1003100000494E464F004543484F004572726F7288
:100320002077726974696E6720746F20454550525A
:100330004F4D210A0053544F505045442E20005039
:1003400072696E7465722073746F70706564206476
:10035000756520746F206572726F72732E20466906
:100360007820746865206572726F7220616E6420F7
:10037000757365204D39393920746F207265737437
:100380006172742E202854656D7065726174757287
:10039000652069732072657365742E20536574201F
:1003A0006974206166746572207265737461727419
:1003B000696E67290A004E6F20436865636B737529
:1003C0006D2077697468206C696E65206E756D624A
:1003D00065722C204C617374204C696E653A200064
:1003E0004E6F20436865636B73756D207769746821
:1003F000206C696E65206E756D6265722C204C6193
:100400007374204C696E653A2000636865636B7392
:10041000756D206D69736D617463682C204C617318
:1004200074204C696E653A20004C696E65204E75EB
:100430006D626572206973206E6F74204C617374F5
:10044000204C696E65204E756D6265722B312C20D3
:100450004C617374204C696E653A20004D31313027
:100460000053657269616C20737461747573206DDB
:1004700069736D617463680A005344207265616436
:10048000206572726F720A004B494C4C2062757481
:10049000746F6E2F70696E0A002121204B494C4CFD
:1004A000206361757365642062792000746F6F202A
:1004B0006D75636820696E6163746976652074691F
:1004C0006D65202D2063757272656E7420636F6D8B
:1004D0006D616E643A20002121204B494C4C206311
:1004E00061757365642062792000706175736500C1
:1004F0004D363030002066696C616D656E745F72D8
:10050000756E6F7574200066696C616D656E745FE1
:1005100072756E6F757420540046696C616D656EFE
:100520007452756E6F75742054004D656469612056
:1005300052656D6F766564004D3130303053006226
:100540007573793A2070617573656420666F7220E7
:10055000696E7075740A00627573793A20706175FE
:1005600073656420666F7220757365720A00627528
:1005700073793A2070726F63657373696E670A00EE
:10058000506C656173652052657365740050524903
:100590004E5445522048414C5445440025533A207E
:1005A000255300706F7765726F6666004B494C4C3F
:1005B00045442E20005072696E7465722068616C2B
:1005C0007465642E206B696C6C28292063616C6CE7
:1005D0006564210A006563686F3A004572726F7244
:1005E0003A0042696C696E656172204C6576656C93
:1005F000696E6720477269643A0A002F2F6163743D
:10060000696F6E3A006E6F74696669636174696FD1
:100610006E2000656E640073686F77006275747495
:100620006F6E00486F74656E6420746F6F20636F27
:100630006C640A0053656E64204D31303820746F4D
:1006400020726573756D650A00496E73657274205A
:1006500066696C616D656E7420616E642073656E91
:1006600064204D3130380A00526568656174204459
:100670006F6E6500526568656174696E672E2E2E17
:100680000052656865617400486561746572205444
:10069000696D656F75740053656E64204D31303837
:1006A00020746F2068656174206E6F7A7A6C650AB9
:1006B000004E6F7A7A6C65205061726B65640070D1
:1006C000617573656400486561642063616E6E6F77
:1006D00074206265207061726B656400506175738F
:1006E0006500726573756D656400526573756D693B
:1006F0006E67004F46460A0046616465204865699A
:100700006768742000426564204C6576656C696E8C
:100710006720004661696C656420746F20656E61B6
:10072000626C6520426564204C6576656C696E6715
:100730000A00496E76616C6964206D6573682E0AE3
:10074000004731205A3130204631323030300A47AC
:100750003120583435205933300A4731205A31304E
:100760000050726F62696E6720506F696E74002569
:10077000532025692F2569002E0A002F0050726F23
:1007800062696E67206D65736820706F696E742092
:1007900000202844525952554E29004732392041F1
:1007A00075746F20426564204C6576656C696E6770
:1007B000003F20284C2C522C462C4229206F757467
:1007C000206F6620626F756E64732E0A003F285694
:1007D000296572626F7365206C6576656C20696D42
:1007E000706C61757369626C652028302D34292E18
:1007F0000A00426164205A2076616C75650A004ED9
:100800006F2062696C696E65617220677269640A43
:10081000005A2050726F62652050617374204265E7
:10082000640A005A2050726F626520506173742010
:1008300042656400446576696174696F6E00255392
:100840003A2025730046696E6973686564210A0061
:100850003A207A3A2000206F662000476F696E6761
:1008600020746F3A20580043570A00206469723A96
:100870000020616E676C653A005374617274207277
:1008800061646975733A004D343820506F696E7435
:100890000025533A2025642F256400506F73697436
:1008A000696F6E696E67207468652070726F62652B
:1008B0002E2E2E0A003F4C656773206F66206D6FE9
:1008C00076656D656E7420696D706C6175736962B3
:1008D0006C652028302D3135292E0A003F202858FC
:1008E0002C5929206F7574206F6620626F756E64B5
:1008F000732E0A0050726F6265206F7574206F66E8
:1009000020626F756E6473003F53616D706C65207B
:1009100073697A65206E6F7420706C61757369629B
:100920006C652028342D3530292E0A004D343820AE
:100930005A2D50726F6265205265706561746162F4
:10094000696C69747920546573740A003F285629CC
:100950006572626F7365206C6576656C20696D7079
:100960006C61757369626C652028302D34292E0AFC
:10097000005374616E6461726420446576696174C9
:10098000696F6E3A20002052616E67653A20002040
:100990004D61783A2000204D696E3A20002053695D
:1009A000676D613A20004D65616E3A200020440079
:1009B00020204D323030205300202844697361627A
:1009C0006C6564293A0046696C616D656E742073CC
:1009D000657474696E67730020204D323031205881
:1009E000004D617820416363656C65726174696F65
:1009F0006E2028756E6974732F7332290020204D84
:100A00003230332058004D6178206665656472612C
:100A10007465732028756E6974732F7329002052D2
:100A20000020204D323034205000416363656C65F6
:100A3000726174696F6E2028756E6974732F7332DA
:100A4000292028503C7072696E742D616363656C57
:100A50003E20523C726574726163742D61636365FC
:100A60006C3E20543C74726176656C2D61636365E5
:100A70006C3E2900204A0020540020530020204DC5
:100A8000323035204200416476616E63656420280F
:100A9000423C6D696E5F7365676D656E745F746906
:100AA0006D655F75733E20533C6D696E5F6665656D
:100AB00064726174653E20543C6D696E5F7472614E
:100AC00076656C5F66656564726174653E204A3C5C
:100AD0006A756E635F6465763E2900204400204994
:100AE0000020204D333031205000486F74656E6413
:100AF000205049440020440020490020204D33303C
:100B0000342050004265642050494400203B0020BE
:100B1000550020204D363033204C0046696C616D05
:100B2000656E74206C6F61642F756E6C6F6164000C
:100B30004D323453256C6454256C64004739322E91
:100B4000394525730047314625640047315A2573DE
:100B500046363030004731582573592573463330B7
:100B60003030004D313036502569532569004D3104
:100B70003039532569004D323030442573004739F0
:100B8000322E395A2573004D3432305325635A259D
:100B90007300473238523058590047315A2573464E
:100BA000363030004739322E395A257300473932F2
:100BB0002E394530004D313039532569004D3139DA
:100BC00030532569004D343230533000203B200033
:100BD00020204D343133205300506F7765722D6CD7
:100BE0006F7373207265636F76657279003B2000C6
:100BF00020496E76616C69642065787472756465ED
:100C000072200047322F4733206261642070617286
:100C1000616D65746572730A00536C6565702E2E84
:100C20002E004732384C300070726F62655F72651B
:100C300077697065004D3131372050726F626520E1
:100C40006661696C65642E205265776970696E67AC
:100C50002E0A4732380A4731322050302053313281
:100C600020543000473239205265747279696E67BA
:100C70000070726F62655F6661696C6564005072D6
:100C80006F62696E67204661696C6564004D313141
:100C90003720426564206C6576656C696E672066F6
:100CA00061696C65642E0A4730205A31300A4D3331
:100CB00030302050323520533838300A4D33303000
:100CC000205035302053300A4D33303020503235EB
:100CD00020533838300A4D333030205035302053CF
:100CE000300A4D3330302050323520533838300AF6
:100CF0004D333030205035302053300A47342053A4
:100D000031004D31313720426564206C6576656C69
:100D1000696E6720646F6E652E005A2050726F6294
:100D20006520506173742042656400205A3A2000A7
:100D300020593A200042656420583A2000206D690D
:100D40006E757465730020616E6420002074757286
:100D50006E7300206279200020005475726E2000AE
:100D60004733352061626F727465642E0A00202853
:100D700000473335206661696C65642061742070BA
:100D80006F696E7420004732385A003F2853296338
:100D900072657720746872656164206D7573742064
:100DA00062652033302C2033312C2034302C203419
:100DB000312C2035302C206F722035312E0A004D19
:100DC00065736820706F696E74206F7574206F662C
:100DD0002072616E67650A004E6F204D6F76652E3A
:100DE00000456E642066696C65206C6973740A0046
:100DF000426567696E2066696C65206C6973740A68
:100E0000004E6F206D656469610A00286E6F206670
:100E1000696C65290043757272656E742066696C31
:100E2000653A200043616E6E6F74206F70656E20AE
:100E300073756264697220005072696E74207469FF
:100E40006D653A20006F6B006F6666001603110334
:100E50000A030303F50244454255473A004D313138
:100E6000332053003344205072696E746572204FF2
:100E700046462E002F2F004D31343520533C696EED
:100E80006465783E206F7574206F662072616E67AE
:100E9000652028302D31290A003F4A206F757420C3
:100EA0006F662072616E67652028302E30312074A5
:100EB0006F20302E33290A0020580020204D617801
:100EC0003A2000200020204D696E3A2000203B206F
:100ED0000020204D323131205300536F667420655D
:100EE0006E6473746F707300250A0046523A0020D6
:100EF000466C6F773A20003A200020536572766F77
:100F00002000206F7574206F662072616E67650A1D
:100F100000536572766F200050726F6265204F66D5
:100F200066736574205A0050726F6265204F666662
:100F3000736574205A0064697300656E0043290A62
:100F40000061626C656420286D696E2074656D7047
:100F50002000436F6C64206578747275646573203B
:100F60006172652000424C546F75636820485320BD
:100F70006D6F646520004F4646004F4E00203B20B9
:100F8000486F73742068616E646C696E6720006DD1
:100F90006D00203B2044697374616E6365200046D8
:100FA000696C616D656E742072756E6F757420006A
:100FB0004D34323120696E636F72726563742070D4
:100FC0006172616D657465722075736167650A0091
:100FD0004D65736820706F696E74206F7574206F33
:100FE000662072616E67650A00454550524F4D207C
:100FF0004F4B0A00290A0020746F20003F5A206FCF
:101000007574206F662072616E6765202800290A5A
:101010000020746F20003F59206F7574206F662088
:1010200072616E676520282D00290A0020746F20E8
:10103000003F58206F7574206F662072616E67657F
:1010400020282D004D383400446F6E652070726981
:101050006E74696E672066696C650A004D373700EB
:101060004D333100496E76616C6964206578747225
:10107000756465720A0020204D32303620580048D1
:101080006F6D65206F6666736574004F6666736585
:101090007473204170706C696564004572723A2007
:1010A000546F6F206661722100546F6F2066617209
:1010B0002066726F6D207265666572656E6365206D
:1010C000706F696E740A004361703A00434F4E4678
:1010D00049475F4558504F5254004D454154504187
:1010E000434B00434F4F4C45525F54454D50455282
:1010F0004154555245004348414D4245525F544585
:101100004D50455241545552450045505F42414271
:101110005953544550004241425953544550504947
:101120004E470041524353004D4F54494F4E5F4D7F
:101130004F44455300544845524D414C5F50524F27
:1011400054454354494F4E00455854454E44454438
:101150005F4D323000435553544F4D5F4649524D19
:10116000574152455F55504C4F4144004C464E5FED
:101170005752495445004C4F4E475F46494C454EE7
:10118000414D45004155544F5245504F52545F53C5
:10119000445F5354415455530053445F575249548C
:1011A0004500524550454154004D554C54495F56F9
:1011B0004F4C554D45005344434152440050524F0B
:1011C0004D50545F535550504F525400484F535454
:1011D0005F414354494F4E5F434F4D4D414E445341
:1011E00000454D455247454E43595F504152534586
:1011F0005200434153455F4C494748545F4252496E
:101200004748544E45535300544F47474C455F4C55
:10121000494748545300534F4654574152455F5035
:101220004F574552004255494C445F504552434543
:101230004E54004C4556454C494E475F444154413D
:10124000005A5F50524F42450052554E4F55540080
:101250004155544F4C4556454C005052494E545FF1
:101260004A4F420050524F47524553530041555444
:101270004F5245504F52545F54454D5000415554C4
:101280004F5245504F52545F504F5300564F4C559C
:101290004D455452494300454550524F4D00424937
:1012A0004E4152595F46494C455F5452414E534658
:1012B00045520053455249414C5F584F4E5F584F7D
:1012C0004646004649524D574152455F4E414D45B5
:1012D0003A4D61726C696E2056322E312E324D5F5E
:1012E0004E494320284A756E203130203230323347
:1012F0002031303A31363A35382920534F55524350
:10130000455F434F44455F55524C3A676974687571
:10131000622E636F6D2F4D61726C696E4669726DDE
:10132000776172652F4D61726C696E2050524F5417
:101330004F434F4C5F56455253494F4E3A312E3032
:10134000204D414348494E455F545950453A334436
:10135000205072696E746572204558545255444548
:10136000525F434F554E543A3120555549443A63E4
:10137000656465326132662D343161322D34373423
:10138000382D396231322D63353563363266333666
:1013900037666600626567696E004D302053746F72
:1013A00070004D312053746F7000436C69636B2083
:1013B000746F20526573756D652E2E2E00203B00D4
:1013C00020204D3835312058005A2D50726F6265FB
:1013D000204F666673657400526573756D696E673C
:1013E000205344002569730025696D202569730029
:1013F0002569682025696D202569730025696420A9
:101400002569682025696D20256973002569792083
:10141000256964202569682025696D202569730088
:101420000A53746174733A2046696C616D656E7419
:1014300020757365643A20002C204C6F6E676573CD
:1014400074206A6F623A2000546F74616C20746972
:101450006D653A200053746174733A20002C204665
:1014600061696C65643A20002C2046696E69736876
:1014700065643A20005072696E74733A20005374A8
:101480006174733A2000436F6F6C696E672E2E2E65
:101490000045312025530020573A0042656420431F
:1014A0006F6F6C696E672E2E2E0042656420486552
:1014B0006174696E672E2E2E0023646566696E6501
:1014C0002044454641554C545F0000626564004B22
:1014D0006420004B6920004B702000504944207468
:1014E000756E696E6720646F6E65002066696E694F
:1014F00073686564212050757420746865206C6180
:101500007374204B702C204B6920616E64204B64F7
:1015100020636F6E7374616E74732066726F6D20DA
:1015200062656C6F7720696E746F20436F6E6669B9
:101530006775726174696F6E2E680A0050494420A5
:101540004175746F74756E6500206661696C6564C1
:10155000212074696D656F75740A005049442041FB
:1015600075746F74756E65004175746F74756E6512
:10157000206661696C6564212054696D656F7574BE
:101580002E00206661696C6564212054656D70656C
:1015900072617475726520746F6F20686967680A7C
:1015A00000504944204175746F74756E6500504950
:1015B00044204379636C65730025532025692F25EA
:1015C0006900204B643A2000204B693A2000204BF0
:1015D000703A200020436C61737369632050494462
:1015E000200A00204E6F206F76657273686F6F74EB
:1015F0000A002054753A2000204B753A2000206DD7
:1016000061783A2000206D696E3A200020643A200B
:101610000020626961733A200048656174696E67F1
:101620002E2E2E002073746172740A0050494420DB
:101630004175746F74756E65004175746F74756E65
:1016400065206661696C6564212054656D70657202
:10165000617475726520746F6F20686967682E0009
:10166000206661696C6564212054656D70657261E6
:101670007475726520746F6F20686967680A00501E
:101680004944204175746F74756E6500504944205B
:101690004175746F74756E6500206661696C656470
:1016A0002120426164206865617465722069640A62
:1016B00000504944204175746F74756E6500457221
:1016C000723A207574663820666F6E74206E6F747F
:1016D00020696E697469616C697A65642E0045726F
:1016E000723A207574663820666F6E74206E6F745F
:1016F00020696E697469616C697A65642E00554E63
:101700004C4F41442046494C414D454E54004C4FAE
:1017100041442046494C414D454E540046494C41B8
:101720004D454E54204348414E4745004572723A5C
:10173000207574663820666F6E74206E6F74206931
:101740006E697469616C697A65642E0020002000FE
:101750003A00200020003A003A002568753A25300A
:101760003268750025303268753A25303268750068
:101770002530326875272530326875002568756414
:101780002025303268753A2530326875004265642C
:1017900000456E636C6F7375726500450020002014
:1017A00000200020002000250020202020202020D4
:1017B000002020202000657272001FE02010201001
:1017C00020101020102020102010303008400480FD
:1017D00003001FE03FF03FF03FF01FE01FE03FF04D
:1017E0003FF03FF00FC0078003003FFFF03800706C
:1017F00030FC3020FC102078102030102C00D02E2F
:1018000031D02F7BD02F7BD02E31D02C00D0203068
:101810001020781020FC1030FC303800703FFFF0B2
:101820003FFFF03800703186302387102787902FD4
:1018300087D02F03D020301020781020781020304F
:10184000102F03D02F87D027879023871031863021
:101850003800703FFFF01FFFF81FFFF80410400230
:101860000820020820041040082080104100104188
:10187000000820800410400000001FFFF81FFFF840
:101880000000007BC08C8A219282209283DE9282AB
:1018900080928A40927221CC0000000000000089F2
:1018A00080008840008980008840005040002180EE
:1018B00000000000000063616E63656C0050726997
:1018C0006E742041626F72746564004469736D695F
:1018D00073730055492041626F72746564004D3224
:1018E0003520500A4D323400526573756D650055D0
:1018F000492050617573650050617573696E672E7C
:101900002E2E00726573756D65004D32340000FE39
:101910000003FF8007C7C00701E00000E00000F0FF
:101920000000700400700E00701F00703F80F00E09
:1019300000E00F01E007C7C003FF8000FE0000FECB
:101940000003FF8007C7C00F01E00E00E03F80F0FA
:101950001F00700E00700400700000700000F000A6
:1019600000E00701E007C7C003FF8000FE000E0093
:101970000E000E000E000E000E000E000E007FC0C6
:101980003F801F000E00040004000E001F003F8077
:101990007FC00E000E000E000E000E000E000E00A6
:1019A0000E00FFFFFF7F80FFC0FFC0FFC07F807F72
:1019B00080FFC0FFC0FFC03F001E000C0050726FD0
:1019C0006265205A204F66667365740052756E6FAB
:1019D00075742044697374206D6D004C6F616420D0
:1019E0006D6D00556E6C6F6164206D6D0046696CA5
:1019F0002E204469612E004F6666004F6E00452020
:101A0000696E206D6D5E33004D33303320553120CB
:101A10004525692053256900504944204175746F5C
:101A200074756E65202A005049442D44202A0050C8
:101A300049442D49202A005049442D50202A002095
:101A4000082046616374002008204D61780020085A
:101A5000204D696E004D696E2054726176656C2070
:101A60005370656564004D696E2056656C6F6369DF
:101A70007479004D61782040205370656564004D95
:101A80006178204520416363656C004D617820409A
:101A900020416363656C0054726176656C2041631C
:101AA00063656C00526574726163742041636365A1
:101AB0006C00416363656C005A2050726F62652050
:101AC00057697A6172640050726F6265205A204FC4
:101AD00066667365740050726F62652059204F66A8
:101AE000667365740050726F62652058204F666699
:101AF00073657400402073746570732F6D6D0041C1
:101B00006476616E6365642053657474696E67738F
:101B1000003F0043616E63656C00496E6974004D5F
:101B200034323800496E697469616C697A652045A0
:101B30004550524F4D0046696C616D656E7400549E
:101B4000656D70657261747572650053746570734C
:101B50002F6D6D0050726F6265204F6666736574FD
:101B600073004A756E6374696F6E20446576004138
:101B70006363656C65726174696F6E004D61782096
:101B8000537065656420286D6D2F7329005365744B
:101B900020486F6D65204F66667365747300436FF0
:101BA0006E66696775726174696F6E003F004361AC
:101BB0006E63656C204F626A656374004E4F005916
:101BC00045530043616E63656C204F626A656374C0
:101BD000207B004D61696E204D656E7500424C544E
:101BE0006F756368204D6F64653A200044414E472D
:101BF00045523A204261642073657474696E67735C
:101C00002063616E2063617573652064616D616737
:101C100065212050726F6365656420616E7977611C
:101C2000793F0043616E63656C005265706F72743A
:101C300020447261696E0053657420424C546F7584
:101C4000636820746F204F440053657420424C54E5
:101C50006F75636820746F203556004D6F64652D75
:101C600053746F7265004F442D4D6F646500355697
:101C70002D4D6F6465004869676820537065656421
:101C80000053572D4D6F64650053746F77004465A2
:101C9000706C6F790053656C662D546573740052D7
:101CA0006573657400426564004E6F7A7A6C6500F6
:101CB00046616E20537065656400436F6E666967A8
:101CC00075726174696F6E00526573746F7265200E
:101CD00044656661756C7473004C6F616420536574
:101CE0007474696E67730053746F72652053657402
:101CF00074696E6773005072656865617420242092
:101D0000436F6E6600506F776572204F7574616720
:101D100065004F6666004F6E0052756E6F757420D9
:101D200053656E736F7200424C546F756368005058
:101D3000726F6265205A204F666673657400416455
:101D400076616E6365642053657474696E677300B1
:101D50004D61696E204D656E75004D3730322054EF
:101D60002564004D36303020423020542564004D2B
:101D7000373032203B2564004D3730312054256404
:101D8000004D373032004D373031004D3630302085
:101D90004230004D61696E204D656E7500436F6E77
:101DA00074696E7565004F6666004F6E0052756E01
:101DB0006F75742053656E736F720050757267652E
:101DC000206D6F726500524553554D45204F50545C
:101DD000494F4E533A005052494E542050415553AA
:101DE0004544002F00200020204E6F7A7A6C653A1F
:101DF00020005061726B696E672E2E2E0000005716
:101E000061697420666F720066696C616D656E74DD
:101E1000206368616E676500746F2073746172740B
:101E2000005761697420666F720066696C616D6548
:101E30006E7420756E6C6F616400004E6F7A7A6C00
:101E4000652068656174696E6700506C65617365D3
:101E500020776169742E2E2E0000507265737320F6
:101E6000627574746F6E00746F2068656174206EA3
:101E70006F7A7A6C650000496E73657274206669CA
:101E80006C616D656E7400616E6420707265737351
:101E900020627574746F6E00746F20636F6E746966
:101EA0006E7565005761697420666F720066696CB3
:101EB000616D656E74206C6F6164000050726573B3
:101EC0007320427574746F6E00746F207265737541
:101ED0006D65207072696E740000576169742066C8
:101EE0006F72207072696E7400746F207265737502
:101EF0006D652E2E2E00005761697420666F72008A
:101F000066696C616D656E7420707572676500003E
:101F1000256C642E25696D0045787472756465645E
:101F200020546F74616C004C6F6E67657374204A47
:101F30006F622054696D65005072696E7420546937
:101F40006D6500436F6D706C65746564003A2000C8
:101F50005072696E7420436F756E74003A200031C0
:101F600032300035004245443A204154432031305C
:101F70003447542D320052756E6177617920576174
:101F80007463683A204F4E004D61782054656D703F
:101F900000323735004D696E2054656D7000350094
:101FA00045313A204550434F53203130304B00509B
:101FB00053550047656E657269630050726F746FA8
:101FC000636F6C00312E3000426175640032353031
:101FD00030303000437265616C697479334420524B
:101FE000414D50530042696C696E656172204C65C9
:101FF00076656C696E670045787472756465727396
:102000000031006D61726C696E66772E6F726700C9
:102010003344205072696E74657200323032332D51
:1020200030352D32390056322E312E324D5F4E4929
:1020300043004D61726C696E005072696E74657216
:1020400020537461747300546865726D6973746FA2
:10205000727300426F61726420496E666F00507245
:10206000696E74657220496E666F004D61696E20FD
:102070004D656E75004D313030300053746F7020F7
:102080005072696E7400526573756D652050726987
:102090006E7400506F776572204F757461676500CC
:1020A0003F004261636B0053746F70004368616E60
:1020B00067652046696C616D656E74004E6F204DDA
:1020C00065646961005072696E742066726F6D207C
:1020D0004D65646961004368616E6765204D6564A4
:1020E0006961004D32310041626F75742050726930
:1020F0006E74657200436F6E6669677572617469AC
:102100006F6E0054656D7065726174757265004D17
:102110006F74696F6E00526573756D6520507269DA
:102120006E740043616E63656C204F626A65637410
:102130000054756E650053746F70205072696E7430
:10214000005061757365205072696E7400496E6647
:102150006F2053637265656E003F00537461727443
:10216000205072696E740043616E63656C0050723A
:10217000696E740043616E6E6F7420656E74657273
:10218000207375626469723A200002202E2E00428C
:1021900061636B004D61696E204D656E75002100B5
:1021A000486F74656E6420746F6F20636F6C640099
:1021B0004261636B0050726F63656564004D6F76BA
:1021C0006520457874727564657200536F6674207B
:1021D000456E6473746F7073004732385A0047322B
:1021E000385900486F6D652040004732385800412B
:1021F00075746F20486F6D65004D6F74696F6E0068
:1022000044697361626C65205374657070657273A4
:10221000004D3834004D34382050726F62652054C0
:10222000657374004732384F0A4D343820503130CE
:102230000053746F77205A2D50726F6265004D34D1
:102240003032004465706C6F79205A2D50726F6285
:1022500065004D343031005472616D6D696E6720D8
:1022600057697A61726400466164652048656967F0
:102270006874004F6666004F6E00426564204C65CE
:1022800076656C696E67004C6576656C20426564A6
:10229000004732394E00486F6D696E67004D6169C5
:1022A0006E204D656E7500000C0F00FE07022503C1
:1022B000BB017FFE08FE08FE05080806000040F08E
:1022C000C88888987810050808060000C0F8888833
:1022D000888888F80505050600012030F8302005BB
:1022E00008080600002070F820202020E0050909D9
:1022F0000600FF2070A8A8B8888870200705050789
:102300000001D86C366CD80509090600FFF8A888CA
:1023100088888888A8F8050A0A0600FE20505050D0
:102320005088A8A8887003030306000340A040FF5C
:10233000FFFFFFFFFFFFFFFFFFFFFFFFFFFFFFFFAD
:10234000FFFFFFFFFF0000000605FF010707060271
:102350000080808080800080030303060105A0A028
:10236000A005060606000050F85050F8500509096F
:102370000600FF2070A8A07028A870200507070697
:102380000000C8C8102040989805070706000040C4
:10239000A0A040A890680103030602058080800386
:1023A00009090601FF204040808080404020030949
:1023B000090601FF8040402020204040800507079B
:1023C00006000020A8702070A82005050506000161
:1023D0002020F820200203030601FFC040800501F1
:1023E00001060003F8020202060100C0C00507074B
:1023F0000600000810102040408005070706000076
:10240000708898A8C8887003070706010040C0407C
:10241000404040E005070706000070880810204093
:10242000F8050707060000F808103008887005074F
:102430000706000010305090F8101005070706003E
:1024400000F880F008088870050707060000304093
:1024500080F0888870050707060000F80810102033
:10246000202005070706000070888870888870059E
:1024700007070600007088887808106002050506C6
:102480000100C0C000C0C00206060601FFC0C000B7
:10249000C04080030505060101204080402005035F
:1024A00003060002F800F80305050601018040203C
:1024B00040800507070600007088102020002005D6
:1024C00007070600007088B8A8B8807005070706DF
:1024D0000000708888F8888888050707060000F0E3
:1024E0004848704848F0050707060000708880805B
:1024F000808870050707060000F04848484848F003
:10250000050707060000F88080F08080F8050707BF
:10251000060000F88080F080808005070706000034
:102520007088808098887005070706000088888872
:10253000F8888888030707060100E04040404040D3
:10254000E00507070600003810101010906005071E
:10255000070600008890A0C0A09088050707060025
:1025600000808080808080F805070706000088D8FA
:10257000A8888888880507070600008888C8A89862
:102580008888050707060000708888888888700595
:102590000707060000F08888F0808080050707069E
:1025A000000070888888A89068050707060000F07A
:1025B0008888F0A090880507070600007088807062
:1025C000088870050707060000F82020202020203A
:1025D000050707060000888888888888700507072F
:1025E00006000088888888505020050707060000EC
:1025F00088888888A8A850050707060000888850A2
:102600002050888805070706000088885020202071
:1026100020050707060000F80810204080F803098D
:10262000090601FFE080808080808080E005070748
:10263000060000804040201010080309090601FF31
:10264000E020202020202020E005030306000520B4
:1026500050880501010600FEF8030303060105800A
:1026600040200505050600007008788878050707F2
:102670000600008080F0888888F0050505060000C7
:102680007080808870050707060000080878888831
:1026900088780505050600007088F080700507073A
:1026A000060000304840E04040400507070600FEB5
:1026B000708888887808700507070600008080F019
:1026C000888888880307070601004000C040404012
:1026D000E00409090601FE1000301010101090608F
:1026E00005070706000080808890E09088030707B0
:1026F000060100C04040404040E0050505060000DE
:10270000D0A8A8A8A8050505060000B0C888888834
:102710000505050600007088888870050707060013
:10272000FEF0888888F080800507070600FE78881C
:102730008888780808050505060000B0C8808080F4
:1027400005050506000078807008F00507070600FB
:10275000002020F8202020180505050600008888A4
:1027600088986805050506000088888850200505BA
:10277000050600008888A8A8500505050600008801
:10278000502050880507070600FE888888502040A2
:1027900080050505060000F8102040F80309090629
:1027A00001FF2040404080404040200109090602CE
:1027B000FF8080808080808080800309090601FF7F
:1027C000804040402040404080050303060002480E
:1027D000A890FF4261636B2D4C6566740042616393
:1027E0006B2D52696768740046726F6E742D526962
:1027F0006768740046726F6E742D4C6566740020B5
:1028000001400130013B014001360160013101709E
:10281000012C0190012701B0012201C0011D01F02E
:102820000118011002130130020E0160020901902B
:10283000020401C002FF000003FA004003F500801B
:1028400003F000D003EB002004E6007004E100E098
:1028500004DC004005D700C005D2004006CD00D002
:1028600006C8008007C3003008BE00F008B900C0E9
:1028700009B400B00AAF00B00BAA00D00CA500004C
:102880000EA000500F9B00C0109600501291000047
:10289000148C00C0158700B0178200B0197D00D0DD
:1028A0001B7800001E730040206E0090226900F02B
:1028B00024640040275F0090295A00E02B55001047
:1028C0002E500020304B0010324600E03341009083
:1028D000353C001037370070383200A0392D00B079
:1028E0003A2800A03B2300603C1E00103D190090D8
:1028F0003D1400103E0F00703E0A00C03E0500006F
:102900003F0000403FFBFF803FF6FFC03FF1FF4725
:1029100032385A0043616E63656C00446F6E650027
:102920004D6F766520246D6D00302E303235004DB0
:102930006F766520302E316D6D004D6F76652031DC
:102940006D6D0050726F6265205A204F6666736528
:1029500074005A004D6F7665204E6F7A7A6C652050
:10296000746F20426564004D6F76696E6720746FE6
:102970002050726F62696E6720506F730050726FE3
:1029800062696E67205A205265666572656E63657E
:102990000047323800507265686561742024204217
:1029A00065640050726568656174202420456E641A
:1029B0000054656D706572617475726500436F6F68
:1029C0006C646F776E0050726568656174202400D6
:1029D00046616E20537065656400426564004E6F09
:1029E0007A7A6C65004D61696E204D656E75004D9B
:1029F000656173757265004C6173742076616C75E6
:102A0000652000426564205472616D6D696E6700D7
:102A1000446F6E6500F427E827DD27D32753656CE4
:102A2000656374204F726967696E00486F6D696EE7
:102A3000672058595A004732384C300050726F6244
:102A400065205A204F666673657400466C6F770088
:102A500046616E20537065656400426564004E6F88
:102A60007A7A6C65005370656564004D61696E200B
:102A70004D656E7500486F6D696E67204661696CC3
:102A80006564006F70656E00545249474745524572
:102A900044003A200066696C616D656E74007A5F6F
:102AA0006D696E00795F6D696E00785F6D696E00AB
:102AB0005265706F7274696E6720656E6473746FAF
:102AC00070207374617475730A0020746F6F206CCA
:102AD0006F6E6720657874727573696F6E2070729F
:102AE0006576656E7465640A0020636F6C642065AA
:102AF0007874727573696F6E2070726576656E7426
:102B000065640A00486F6D652025732046697273FD
:102B10007400000000000000000000000000576189
:102B2000726E696E673A20486F6D696E67204275F4
:102B30006D702044697669736F72203C20310A0001
:102B400002020400009B4300009B430000E143009D
:102B500000A0400000A04000000040000000010074
:102B60000000010000800055555500000040003372
:102B7000333300AAAA2A004992240000002000C78B
:102B8000711C0099991900D1451700555515003B46
:102B9000B113002449120011111100000010000FA0
:102BA0000F0F00E3380E0043790D00CCCC0C00C3AE
:102BB000300C00E8A20B0064210B00AAAA0A0070E6
:102BC0003D0A009DD80900427B090092240900DCDF
:102BD000D30800888808001042080000000800F0B0
:102BE000C107008787070075500700711C07003E6A
:102BF000EB0600A1BC060069900600666606007040
:102C00003E06006118060017F4050074D105005B4C
:102C1000B00500B2900500627205005555050078B8
:102C2000390500B81E0500050505004EEC040087B7
:102C3000D40400A1BD040090A7040049920400C17F
:102C40007D0400EE690400C7560400444404005C9F
:102C50003204000821040041100400000004003F79
:102C6000F00300F8E0030026D20300C3C30300CC46
:102C7000B503003AA803000A9B0300388E0300C086
:102C80008103009F750300D0690300505E03001D9F
:102C900053030034480300913D030033330300160F
:102CA000290300381F030097150300300C030003AD
:102CB0000303000BFA020049F10200BAE802005CCB
:102CC000E002002DD802002DD0020059C80200B049
:102CD000C0020031B90200DAB10200AAAA0200A0C3
:102CE000A30200BC9C0200FA9502005C8F0200DF88
:102CF00088020082820200457C02002776020027BB
:102D0000700200436A02007C640200D05E02003F51
:102D1000590200C8530200FFFDFCFAF8F6F4F2F085
:102D2000EEECEAE9E7E5E3E1E0DEDCDAD9D7D5D499
:102D3000D2D0CFCDCBCAC8C7C5C3C2C0BFBDBCBA35
:102D4000B9B7B6B4B3B2B0AFADACAAA9A8A6A5A4A2
:102D5000A2A1A09E9D9C9A99989795949392908FEA
:102D60008E8D8B8A8988878684838281807F7E7D11
:102D70007B7A797877767574737271706F6E6D6C1B
:102D80006B6A696867666564636261605F5E5D5C0B
:102D90005B5A5958585756555453525150504F4EEC
:102DA0004D4C4B4A4A4948474646454443424241B6
:102DB000403F3E3E3D3C3B3B3A393838373635356F
:102DC000343332323130302F2E2E2D2C2B2B2A291A
:102DD0002928272726252524232322212120201FB7
:102DE0001E1E1D1C1C1B1B1A191918181716161548
:102DF0001514131312121111100F0F0E0E0D0D0CCE
:102E00000C0B0A0A09090808070706060505040449
:102E10000303020201000053544F505045442E203A
:102E2000005072696E7465722073746F707065649F
:102E30002064756520746F206572726F72732E2026
:102E400046697820746865206572726F7220616EC1
:102E50006420757365204D39393920746F2072658F
:102E600073746172742E202854656D70657261747C
:102E70007572652069732072657365742E205365C1
:102E80007420697420616674657220726573746160
:102E90007274696E67290A00206572726F72202D44
:102EA00020726573746172742077697468204D397B
:102EB00039390A00424C546F756368002121205350
:102EC000544F502063616C6C65642062656361756A
:102ED0007365206F66200000009B4300009B430049
:102EE00000E143000000000000000000000000536B
:102EF000657474696E67732053746F72656400291A
:102F00000A002062797465733B206372632000536A
:102F1000657474696E67732053746F7265642028DA
:102F200000454550524F4D20496E697469616C6986
:102F30007A65640A0048617264636F646564204462
:102F4000656661756C742053657474696E6773206F
:102F50004C6F616465640020286D6D2900203B2062
:102F60004C6576656C696E67200020204D343230E8
:102F70002053004175746F20426564204C6576656E
:102F80006C696E670020460020480020204D3134D7
:102F9000352053004D6174657269616C206865610C
:102FA00074757020706172616D6574657273002054
:102FB0003B2053656E736F72200020440020204D2B
:102FC00034313220530046696C616D656E74207235
:102FD000756E6F75742073656E736F7200204A0092
:102FE0002020473239205720490020204D313439E4
:102FF0002043203B20556E69747320696E20436521
:103000006C736975730A0054656D706572617475CF
:10301000726520556E697473002020473231203B61
:10302000004C696E65617220556E69747300454588
:1030300050524F4D206461746173697A65206572E6
:10304000726F722E0A004572723A20454550524FF7
:103050004D2043524300202863616C63756C61749A
:10306000656429210A0020213D2000454550524F2A
:103070004D20435243206D69736D61746368202D48
:10308000202873746F726564292000454550524FA3
:103090004D20436F72727570740A002053697A650F
:1030A0003A2000496E6465783A200053746F726567
:1030B000642073657474696E6773207265747269D5
:1030C0006576656400290A002062797465733B2087
:1030D00063726320002073746F726564207365747B
:1030E00074696E67732072657472696576656420B1
:1030F000280000803B4400803B44000070410000F9
:1031000096420000A0420000A0420000C843008098
:10311000C543E8030000E8030000640000008813D2
:103120000000204D61726C696E3D563838290A00E6
:10313000454550524F4D2076657273696F6E206D14
:1031400069736D617463682028454550524F4D3D49
:103150000024F4D43050C38D20C3A24117828B7059
:1031600011127A900D826CDA0AA861E108C75866DC
:1031700007615142061F4B5E05C145A6041B411263
:1031800004093D9703723931034136DB02663392FD
:1031900002D4305302812E1D02642CEE01762AC522
:1031A00001B128A101102781018F2564012B244A38
:1031B00001E1223401AD2120018D200C01811FFC91
:1031C00000851EED00981DDF00B91CD200E71BC76B
:1031D00000201BBB00651AB200B319A9000A19A090
:1031E000006A189800D217920040178A00B6168419
:1031F0000032167E00B41579003B157400C7146FB9
:103200000058146A00EE1366008813620026135EED
:1032100000C8125B006D12570016125500C1115103
:103220000070114E0022114C00D61049008D10463E
:10323000004710450002104200C00F4000800F3EC2
:1032400000420F3C00060F3A00CC0E3900930E37B7
:10325000005C0E3500270E3400F30D3200C10D3135
:1032600000900D2F00610D2F00320D2D00050D2C4B
:1032700000D90C2A00AF0C2A00850C28005D0C2810
:1032800000350C27000E0C2500E90B2500C40B248B
:1032900000A00B23007D0B22005B0B21003A0B21C9
:1032A00000190B2000F90A1F00DA0A1F00BB0A1ED2
:1032B000009D0A1D00800A1C00640A1C00480A1CAC
:1032C000002C0A1B00110A1A00F7091A00DD09195F
:1032D00000C4091900AB091800930918007B0917ED
:1032E00000640917004D091700360916002009155A
:1032F000000B091500F6081500E1081500CC0814AC
:1033000000B8081400A4081300910813007E0813E5
:10331000006B081200590812004708120035081205
:1033200000230811001208110001081000F1071114
:1033300000E0071000D0071000C0070F00B1071011
:1033400000A1070F0092070F0083070F0074070EFC
:103350000066070E0058070E004A070E003C070ED5
:10336000002E070D0021070D0014070D0007070DA3
:1033700000FA060D00ED060C00E1060D00D4060C67
:1033800000C8060C00BC060C00B0060B00A5060C1D
:103390000099060B008E060B0083060B0078060BC7
:1033A000006D060B0062060B0057060A004D060A68
:1033B0000043060B0038060A002E060A0024060900
:1033C000001B060A0011060A0007060900FE050A8E
:1033D00000F4050900EB050900E2050900D905091B
:1033E00000D0050900C7050800BF050900B605099A
:1033F00000AD050800A50508009D05080095050914
:10340000008C050800840508007C05070075050888
:10341000006D050800650507005E050800560507F4
:10342000004F05080047050700400507003905075C
:1034300000320507002B050700240507001D0507BE
:1034400000160507000F050600090507000205061E
:1034500000FC040700F5040600EF040700E804067A
:1034600000E2040600DC040600D6040600D00407CF
:1034700000C9040500C4040600BE040600B8040622
:1034800000B2040600AC040600A6040500A1040670
:10349000009B04050096040600900405008B0406BA
:1034A0000085040500800405007B04050076040601
:1034B00000700405006B0405006604050061040546
:1034C000005C04050057040500520405004D040586
:1034D0000048040400440405003F0405003A0404C5
:1034E0000036040500310405002C040400280405FE
:1034F00000230404001F0405001A04040016040439
:1035000000120405000D040400090404000504046D
:103510000001040500FC030400F8030400F40304A4
:1035200000F0030400EC030400E8030400E40304D7
:1035300000E0030400DC030400D8030400D4030308
:1035400000D1030400CD030400C9030400C5030433
:10355000000000000000000000000000000000006B
:10356000000000000000000000D1036D6403570D4F
:103570000347C6023B8B023259022B2E0225090259
:1035800021E8011CCC011AB201179B011487011319
:1035900074011163010F54010E46010D39010D2C08
:1035A000010B21010A17010A0D0109040108FC00A1
:1035B00008F40007ED0007E60007DF0006D9000663
:1035C000D30005CE0006C80005C30004BF0005BA3D
:1035D0000004B60004B20004AE0004AA0004A60071
:1035E00003A300049F00039C0003990003960003BB
:1035F0009300029100038E00028C00038900028771
:1036000000038400028200028000027E00027C002F
:10361000027A00027800027600017500027300024F
:103620007100017000026E00016D00026B00016A02
:103630000002680001670002650001640001630088
:10364000016200026000015F00015E00015D000197
:103650005C00015B00015A0001590001580001574C
:1036600000015600015500015400015300015200B1
:10367000015100005100015000014F00014E0001B6
:103680004D00004D00014C00014B00014A00004A72
:1036900000014900014800004800014700014600C0
:1036A00000460001450000450001440001430000C0
:1036B000430001420000420001410000410001407E
:1036C00000004000013F00003F00013E00003E00BE
:1036D000013D00003D00013C00003C00013B0000BA
:1036E0003B00013A00003A0001390000390000397E
:1036F00000013800003800013700003700003700B3
:1037000001360000360000360001350000350001AA
:103710003400003400003400013300003300003373
:10372000000132000032000032000131000031009F
:103730000031000031000130000030000030000195
:103740002F00002F00002F00002F00012E00002E60
:1037500000002E00012D00002D00002D00002D0086
:10376000012C00002C00002C00002C00012B00007C
:103770002B00002B00002B00012A00002A00002A49
:1037800000002A00002A0001290000290000290069
:10379000002900012800002800002800002800005F
:1037A000280001270000270000270000270000272D
:1037B000000126000026000026000026000026004A
:1037C000002600012500002500002500002500003E
:1037D000250000250001240000240000240000240E
:1037E0000000240000240001230000230000230027
:1037F000002300002300002300012200002200001B
:1038000022000022000022000022000022000121EC
:103810000000210000210000210000210000210003
:1038200000210001200000200000200000200000F6
:103830002000002000002000002000011F00001FC9
:1038400000001F00001F00001F00001F00001F00DD
:103850000020436F756E7420583A0042656400453D
:1038600031004500626564002C2073797374656DC6
:103870002073746F7070656421204865617465728F
:103880005F49443A20004572723A204D41585445F0
:103890004D50004D415854454D5020747269676732
:1038A000657265640048656174696E672046616988
:1038B0006C65640048656174696E67206661696C57
:1038C0006564004D353234004D3131322053687516
:1038D00074646F776E001000C90210012C01400162
:1038E000220170011801B0010E01F0010401500223
:1038F000FA00B002F0003003E600D003DC009004D0
:10390000D2007005C800A006BE000008B400B009CF
:10391000AA00D00BA000600E960060118C0000156C
:10392000820020197800C01D6E00A0226400B0271C
:103930005A00902C500000314600E0343C00103812
:103940003200903A2800603C1E00A03D1400803EEA
:103950000A00203F00004572723A204D494E5445FE
:103960004D50004D494E54454D5020747269676763
:103970006572656400544845524D414C2052554E85
:103980004157415900546865726D616C2052756EE3
:103990006177617900202F002042403A0020403AB0
:1039A0000020573A007C3C3E5E2B3D3F2F5B5D3B49
:1039B0002C2A225C0043616E6E6F74206F70656EFE
:1039C0002073756264697220004D656469612049E5
:1039D0006E6974204661696C0053442063617264AF
:1039E000206F6B0A006F70656E526F6F7420666196
:1039F000696C65640A00766F6C756D652E696E6919
:103A000074206661696C65640A004E6F205344201F
:103A1000636172640A0053442063617264207265BA
:103A20006C65617365640A000A4D3234004D3233AF
:103A3000202573002E0A006F70656E206661696C28
:103A400065642C2046696C653A200046696C6520E7
:103A500073656C65637465640A002053697A653A1E
:103A6000200046696C65206F70656E65643A2000C1
:103A7000454E4420535542524F5554494E450A0035
:103A80002220706F73002220706172656E743A227A
:103A900000535542524F5554494E452043414C4CDA
:103AA000207461726765743A220053756263616CB9
:103AB0006C204F766572666C6F770045786365653C
:103AC000646564206D617820535542524F555449C6
:103AD0004E452064657074683A0041425300504579
:103AE000544700504C41002E0A0044656C657469CF
:103AF0006F6E206661696C65642C2046696C653A5E
:103B0000200046696C652064656C657465643A00E4
:103B10004E6F74205344207072696E74696E670A28
:103B2000005344207072696E74696E672062797404
:103B300065200057726974696E6720746F2066692A
:103B40006C653A2000667265736800646F696E6721
:103B5000002066696C653A20004E6F7720002F6167
:103B600075746F25632E67000000000000000000E0
:103B70000000000000000000000000000000000045
:103B80000000000000000000000000000000000035
:103B90000000000000000000000000000000000025
:103BA0000000000000000000000000000000000015
:103BB0000000000000000000000000000000000005
:103BC00000000000000000000000000000000000F5
:103BD00000000000000000000000000000000000E5
:103BE000000000000000000000000080000008004D
:103BF000000000000000000000000080000008003D
:103C0000000000000000000000209E9DE773C80037
:103C1000000000000000000000359291249248004E
:103C2000000000000000000000151E912493C80051
:103C30000000000000000000001B10912492000012
:103C40000000000000000000000A1E9DE493C80070
:103C50000000000000000000000000000000000064
:103C60000000000000000000000000000000000054
:103C70000000000000000000000000000000000044
:103C80000000000000000000000000000000000034
:103C90000000000000000000000000000000000024
:103CA0000000000000000000000000000000000014
:103CB0000000000000000000000000000000000004
:103CC00000000000000000000000000000000000F4
:103CD00000000000000000000000000000000000E4
:103CE00000000000000000000000000000000000D4
:103CF00000000000000000000000000000000000C4
:103D000000000000000000000000000000000000B3
:103D100000000000000000000000000000000000A3
:103D20000000000000000000000000000000000093
:103D30000000000000000000000000000000000083
:103D4000000000000000000000000FFDFFC0FF8029
:103D5000C0600FFFF80F000000001FFDFFE3FF80B1
:103D6000C0600FFFF81E000000003C01806780016A
:103D7000C0600E0E1E3C0000000070018067000154
:103D8000E0600E0E0F78000000006001806E0003FE
:103D9000E0600E0E07F0000000006001BFEFFF833F
:103DA00070600E0E03E00000000060019FCFFF87EF
:103DB00038600E0E01C00000000060018E0E00078A
:103DC00018600E0E01C00000000070018707000E91
:103DD0001E600E0E01C0000000003C018387800CB5
:103DE0000E600E0E01C0000000001FFD81C3FF9C8D
:103DF000FE7FEE0E01C0000000000FFD80E0FFBD61
:103E0000FF7FEE0E01C00000000000000000000077
:103E100000000000000000000000000000000000A2
:103E20000000000000000000000000000000000092
:103E30000000000000000000000000000000000082
:103E40000000000000000000000000000000000072
:103E50000000000000000000000000000000000062
:103E60000000000000000000000000000000000052
:103E70000000000000000000000000000000000042
:103E80000000000000000000000000000000000032
:103E90000000000000000000000000000000000022
:103EA0000000000000000000000000000000000012
:103EB0000000000000000000000000000000000002
:103EC00000000000000000000000000000000000F2
:103ED00000000000000000000000000000000000E2
:103EE00000000000000000000000000000000000D2
:103EF00000000000000000000000000000000000C2
:103F000000000000000000000000000000000000B1
:103F100000000000000000000000000000000000A1
:103F20000000000000000000000000000000000091
:103F30000000000000000000000000000000000081
:103F40000000000000000000000000000000000071
:103F50000000000000000000000000000000000061
:103F600000000000000000006D61726C696E6677F1
:103F70002E6F72670056322E312E324D5F4E4943FE
:103F8000001FFFFFFFFFFFFF600000000001FF4078
:103F90000000000000FF8000000000007F83CF00D1
:103FA000000C303F87FF80000C301F867980000CAA
:103FB000000F8C30C7838C30E78C30CFC7CC31F307
:103FC0008C30DCECEC33B98C30D86C6C33198C3021
:103FD000D06C0C33198C30D86C0C33198C30DC6CF1
:103FE0000E3B198C30CF7C079F198C30C77C038F18
:103FF0001940000000000002600000000000061FE1
:10400000FFFFFFFFFFF82020506C616E6E6572426B
:10401000756666657242797465733A20002046724F
:104020006565204D656D6F72793A200020436F6D94
:1040300070696C65643A204A756E203130203230E8
:1040400032330A00204C61737420557064617465CA
:10405000643A20323032332D30352D3239207C20F5
:10406000417574686F723A204E69632057696C73AA
:104070006F6E0A004D61726C696E2056322E312EC1
:10408000324D5F4E49430A0020536F667477617268
:10409000652052657365740A002057617463686413
:1040A0006F672052657365740A002042726F776EE5
:1040B000206F75742052657365740A00204578740A
:1040C00065726E616C2052657365740A00506F777B
:1040D000657255700A0073746172740A0047323851
:1040E00058590A4D31380A004D313030310065726F
:1040F000726F722077726974696E6720746F2066C0
:10410000696C650A00446F6E6520736176696E673D
:104110002066696C652E0A004D323900456E647365
:10412000746F707300255320256320256320256359
:1041300020256300205A3A0020593A0020583A00BE
:10414000656E6473746F7073206869743A20000040
:10415000000A0B02090C0D0E080703040100000001
:10416000000000000000000000000000000000004F
:10417000000000000000000000000012111000000C
:10418000000000000000000000000000000000002F
:1041900000000000004D6F766520246D6D00302E0C
:1041A000303235004D6F766520302E316D6D004D0B
:1041B0006F766520316D6D004D6F76652031306D05
:1041C0006D004D6F76652041786973004D6F76659F
:1041D000202A004D6F7665204000E33ADE3ADA3A55
:1041E0004368616E67652046696C616D656E740039
:1041F000556E6C6F61642046696C616D656E74000C
:104200004C6F61642046696C616D656E740050721C
:10421000656865617420437573746F6D00507265D5
:10422000686561742024004261636B002000507255
:10423000696E742066726F6D204D6564696100203F
:10424000002000DB0FC93F45BCDA3F8FB30240FCC2
:10425000F0274056946140FE4B9B4084A5D840E037
:10426000231841346A5641E859974164DBD5416EC1
:10427000271742B4B75542CE1A9742C8AED542B5B9
:10428000885A43D40684BFA65FA7BF7443E0BF101B
:10429000B11AC01C2C58C0E8F697C0B849D6C04E19
:1042A0004E17C124D355C1802497C1A0B5D5C112E2
:1042B0001A17C244AE55C2781797C26CACD5C26704
:1042C000885AC320746F6F206C6F6E672065787496
:1042D000727573696F6E2070726576656E74656451
:1042E0000A0020636F6C6420657874727573696F5F
:1042F0006E2070726576656E7465640A0070726F08
:104300006D70745F00626567696E00446973616215
:104310006C6552756E6F75740050757267654D6F80
:1043200072650050617573656400436F6E74696EE9
:104330007565004C6F61642046696C616D656E74D3
:10434000205400496E736572742066696C616D65F6
:104350006E7420616E642073656E64204D31303858
:104360000A00205A3A200020593A20004265642071
:10437000583A200050726F62696E67204661696C1E
:10438000656400FFFFFF00002200250028002B00CD
:104390002E003100340002010000050108010B016C
:1043A00000002100240027002A002D0030003300E7
:1043B00001010000040107010A01050505050705C3
:1043C00008080808020202020A0A08080404040491
:1043D00001010101010101010303030303030303BD
:1043E000040707070C0C0C0C0C0C0C0C020202024C
:1043F00006060606060606060B0B0B0B0B0B0B0B35
:1044000001021020200808102040102040800201E6
:1044100002010804020101020408102040808040CB
:1044200020100804020180040201804020100804CA
:104430000201080402010102040810204080010268
:10444000040810204080204500205A0020590020F8
:10445000204D393220580053746570732070657296
:1044600020756E697400220A00556E6B6E6F776E50
:1044700020636F6D6D616E643A202200204200203F
:1044800050006F6B0020453A00205A3A0020593AFC
:1044900000583A006F6B0A00526573656E643A20EB
:1044A000003344205072696E7465722052656164F5
:1044B000792E005072696E74696E672E2E2E005030
:1044C00072696E7420506175736564006E6F7469F3
:1044D0006669636174696F6E2000B600C8001124BC
:1044E0001FBECFEFD1E2DEBFCDBF00E00CBF84B76F
:1044F0008093F41A14BE0FB6F894A89580916000CA
:10450000886180936000109260000FBE14E0A0E00C
:10451000B2E0E8E5FFED02E00BBF02C007900D92AC
:10452000A630B107D9F72AE1A6E0B4E001C01D9298
:10453000A43FB207E1F712E2CEE6D2E200E006C005
:1045400021970109802FFE010F94396CCD36D107D8
:1045500080E00807A9F70F9461590D949B6F0C94A4
:104560000000CF93DF93C091CE10D091CF1081E0A7
:10457000CE31D105E4F020E030E040E05FE360912F
:10458000CA107091CB108091CC109091CD100F94E7
:10459000546C0F94986D6C1B7D0B77FF03C0719565
:1045A0006195710981E0633071050CF080E0DF9165
:1045B000CF910895CF93DF93DB01F9019C91913066
:1045C000C1F0943080F094509C938830D1F4808175
:1045D0009181009771F0019791838083480F591F53
:1045E000EA01188206C08C3539F49C5F9C939430A4
:1045F00041F4DF91CF9108958B3339F781E08C93AB
:10460000F8CF20813181B9016F5F7F4F7183608363
:10461000420F531FEA018883808191818F35910574
:104620006CF7E7CF0F931F9381E00091EC18109186
:10463000ED182091EE183091EF184091E818509144
:10464000E9186091EA187091EB180417150726070E
:10465000370708F480E01F910F91089590E080E003
:1046600008952091E318833021F425FD0CC024FD2A
:104670000CC030E0A90102C0559547958A95E2F734
:10468000CA018170089581E0089580E008958091C5
:10469000AB0484FD0BC08091AD0487FD07C09091F1
:1046A000AE04937081E019F480E0089581E00895EC
:1046B0002FEB280F2A3108F047C0E22FF0E080915D
:1046C000AB049091AC04A091AD04B091AE0404C0D1
:1046D000B695A795979587952A95D2F780FD02C044
:1046E00081700895EF56FB4FE081EE2341F18091F8
:1046F0004C0B90914D0BE80FF92FF11D808190ED3F
:10470000980F9A3030F08E3251F4818180538A3084
:1047100098F4F0938004E0937F0481E008958D3253
:1047200011F08B3249F4818190ED980F9A3088F323
:104730008E3211F48281EACFF0E0E0E0EACF10920D
:10474000800410927F04E9CF80E00895B1DF8823D0
:1047500041F081E020917F0430918004232B09F403
:1047600080E00895282F80931F02803240F58091C9
:10477000BE04281724F081E0820F8093BE0481E0FC
:1047800090E002C0880F991F2A95E2F7092E000CCD
:10479000AA0BBB0B4091BA045091BB046091BC04BE
:1047A0007091BD0484239523A623B72321E0892B90
:1047B0008A2B8B2B09F420E02093F60A089510929F
:1047C000F60A08951092F80A80914B0290914C02DB
:1047D000A0914D02B0914E0280930E0890930F0865
:1047E000A0931008B09311080895269A2E9A089560
:1047F0008F929F92AF92BF92CF92DF92EF92FF92F1
:10480000FC01828158E5C52E52E0D52EC81AD10888
:1048100087FDD394CC0CDD1CCC0CDD1C0D2C000CC6
:10482000EE08FF08818178E8872E912C881A91087C
:1048300087FD9394880C991C880C991C092C000CFA
:10484000AA08BB0880818F3FD1F190E0FC01EE0FF8
:10485000FF1FE80FF91FE05EFE4E8181928133E079
:10486000880F991F3A95E1F7B0E0A0E044E0B595D4
:10487000A795979587954A95D1F702969C012F5F4A
:104880003F4F032E000C440B550B281939094A09D8
:104890005B09A4EBB0E00F94DA6BA701960128192D
:1048A00039094A095B090F94BE6BC901FF90EF906B
:1048B000DF90CF90BF90AF909F908F90089590E041
:1048C00080E0DCCFCF93DF93C091CE10D091CF109A
:1048D000209729F16091CA107091CB108091CC1073
:1048E0009091CD100F94986D6E5F7F4F24976C1749
:1048F0007D07ACF47093C7086093C6080F94D04D41
:10490000605E70448D4F9F4F6093C8087093C908D4
:104910008093CA089093CB08DF91CF9108951092AD
:10492000C8081092C9081092CA081092CB08F4CF98
:10493000AB01BC014093EC185093ED186093EE1856
:104940007093EF1885E59AE10C944DE4CF93DF93D3
:1049500000D01F92CDB7DEB780E090E0A0EAB0E4CF
:1049600089839A83AB83BC8341E061E0CE010196E9
:104970000F9449040F900F900F900F90DF91CF91FB
:1049800008950F931F93CF93DF9300D01F92CDB75D
:10499000DEB79C010CE716E090E1EEE4FBE0D80105
:1049A00001900D929A95E1F7F901208131814281C0
:1049B0005381F80160857185828593850F94546CCD
:1049C000F801608771878287938780E090E0A0E696
:1049D000B1E489839A83AB83BC83CE0101960F94A3
:1049E000F3290F900F900F900F90DF91CF911F91AF
:1049F0000F91089580917F0490918004009731F089
:104A00004AE050E070E060E00D94936360E070E095
:104A1000CB0108950F931F93CF9380917F049091C2
:104A20008004009709F1FC018F01C1912C2F2F7D8B
:104A3000A1F0C53431F0C53621F0C83511F0C837C2
:104A400099F7F801108270E060E00F941061F801AE
:104A5000C083CF911F910F91089570E060E0CF91D6
:104A60001F910F910D94106160E070E0CB01F1CFC8
:104A7000CF92DF92EF92FF926A017B0167DE88237B
:104A800029F0FF90EF90DF90CF90C4CFC701B6011F
:104A9000FF90EF90DF90CF9008950F931F93CF93E7
:104AA00083E554DE8823F9F00F94D04D6093DD0840
:104AB0007093DE088093DF089093E008ABDF20E07E
:104AC00030E04AE754E40F94D7650F949D6D6093EE
:104AD0000202709303028093040290930502CF9127
:104AE0001F910F910895D3DD882331F10E94BFF209
:104AF00085E4DEDD81110E949EEC0AEC12E0C0E04C
:104B0000F80121918F0121548091AB049091AC0464
:104B1000A091AD04B091AE0404C0B695A795979549
:104B200087952A95D2F780FF03C08C2F0E94ADECA9
:104B3000CF5FC33029F7D3CFCF911F910F910C9442
:104B4000D0F280917F0490918004009731F04AE088
:104B500050E070E060E00D94666260E070E0CB01D0
:104B60000895CF93DF93EB01F1DD882311F0E9DFA6
:104B7000EB01CE01DF91CF910895E3DFCB010895E2
:104B8000CF93DF93EB01E2DD882319F0DF91CF9122
:104B9000F4CFCE01DF91CF910895D3DF97FD0AC006
:104BA000D0DF6F3F71058105910509F02CF4C9DF55
:104BB000862F089580E008958FEF089580917F04F7
:104BC00090918004892B39F0E8DF91E0811101C0D8
:104BD00090E0892F089591E0FCCFCF93DF93C82F09
:104BE000D62FB4DD882319F0DF91CF91E7CF8C2F3A
:104BF0005FDD811101C08D2FDF91CF910895CF939B
:104C0000C62FA4DD882311F0CF91C7CF8C2FCF9171
:104C10000895CF92DF92EF92FF92CF936B017C01C8
:104C2000C42F809112088F5F09F4B5C080931208D9
:104C3000809112088093C10820E030E040E752E400
:104C400060912702709128028091290290912A0296
:104C50000F94D7650F949D6D70932408609323087B
:104C6000C0922508D0922608E0922708F0922808E2
:104C70008091C008C0FB80F98093C0088CE0EDE310
:104C8000FAE0A9E2B8E001900D928A95E1F78CE094
:104C9000E0E7F6E0A5E3B8E001900D928A95E1F730
:104CA0008091C3069091C00880FB94F99093C0084E
:104CB000882381F08091BF069091C006A091C10623
:104CC000B091C2068093410890934208A093430894
:104CD000B09344088091FA109091FB10909346088D
:104CE000809345088091CE109091CF109093480802
:104CF000809347088091E50A809349088091C00815
:104D00009091AE0690FB83F98093C0088091AA062B
:104D10009091AB06A091AC06B091AD0680934A0885
:104D200090934B08A0934C08B0934D080F94AC0A95
:104D30006093BB087093BC088093BD089093BE0835
:104D40008091E3188093BF089091F70A8091C00882
:104D500093FB81F990918F0490FB82F98093C008B6
:104D600080E00F94E45440E050E0BA0186EF98E10F
:104D70000E944DE440EB50E062E178E086EF98E17C
:104D80000E9423E686EF98E1CF91FF90EF90DF90AD
:104D9000CF900C949DE781E049CF4F925F926F9244
:104DA0007F928F929F92AF92BF92CF92DF92EF92BB
:104DB000FF920F931F93CF93DF9300D01F92CDB735
:104DC000DEB719821A821B821C829AEC892E92E02D
:104DD000992ECE0101965C012EE4C22E2BE0D22E3C
:104DE0003CE7E32E36E0F32E10E000E0F401819181
:104DF0004F01ACDCF50181935F01882339F00ADEB5
:104E00002B013C018091F60A882359F0F60180813C
:104E10009181A281B381F70180839183A283B383BF
:104E200013C0802F1EDC882309F4D1C0F601208135
:104E3000318142815381C301B2010F94546CF70157
:104E400060837183828393830F5F1F4FF4E0CF0EE3
:104E5000D11C84E0E80EF11C0330110539F685E41D
:104E600075DC8C83882309F4C2C0D4DD6B017C011E
:104E700083E0F7DB882371F020915A0B30915B0BB4
:104E800040915C0B50915D0BC701B6010F94546CBF
:104E90006B017C01C0928806D0928906E0928A0656
:104EA000F0928B068091C406882389F18091F018D6
:104EB00082FF2DC087FD2BC08C81882341F1898121
:104EC000811103C08A81882311F12AE939E949E176
:104ED0005EE360911B0870911C0880911D08909101
:104EE0001E080F94546C9B01AC016091560B70919D
:104EF000570B8091580B9091590B0F947B6E18169D
:104F000034F440E060E070E080E090E482DE40E075
:104F100050E0BA0186E4ACDD20E030E0A9010F9456
:104F20007B6E18167CF476DD20E030E040E752E43A
:104F30000F94306D609327027093280280932902AA
:104F400090932A028091F70A83FD2CC08091F60A83
:104F5000811128C08091280A882321F120915A0BC1
:104F600030915B0B40915C0B50915D0B609188061A
:104F70007091890680918A0690918B060F94536CEC
:104F80002091350A3091360A4091370A5091380AFB
:104F90000F94546C6093350A7093360A8093370AE5
:104FA0009093380A0F900F900F900F90DF91CF9150
:104FB0001F910F91FF90EF90DF90CF90BF90AF9037
:104FC0009F908F907F906F905F904F900895F80121
:104FD000EE0FFF1FEE0FFF1FE25AF44F20813181C9
:104FE00042815381C301B2010F94536C28CF809149
:104FF0005A0B90915B0BA0915C0BB0915D0B809371
:10500000880690938906A0938A06B0938B064ACFB0
:10501000AF92BF92CF92DF92EF92FF920F931F93C6
:10502000CF935C016B018A01885E9B4F7C01DC01A0
:10503000CC91C7FF3DC0FB0111821082CF5FD70129
:10504000CC93CC300CF053C08CE08A9DF0018B9D4A
:10505000F00D1124CF018C0F911DC7FD9A95209161
:1050600068112817190609F00CF441C0F6012081D7
:105070003181FC01EE0FFF1FE80FF91FE05EFE4ECD
:1050800081819281820F931FD80111969C938E93F8
:10509000808187FF3DC061E08F77CF911F910F9195
:1050A000FF90EF90DF90CF90BF90AF900D94114D97
:1050B0008CE08A9DF0018B9DF00D1124CF018C0FA7
:1050C000911DC7FD9A95209168112817190609F0BE
:1050D0000CF4B4CFFC01EE0FFF1FE80FF91FE05EE8
:1050E000FE4E808160E08F770F94114DA7CFF601BF
:1050F0008081918104968034FCE99F0710F480E45C
:105100009CE9D80111969C938E938FEFF7018083D1
:10511000CF911F910F91FF90EF90DF90CF90BF90B4
:10512000AF900895CF92DF92EF92FF920F931F936B
:10513000CF93DF93CDB7DEB72C970FB6F894DEBFD1
:105140000FBECDBFF090E018E090E1182091B504BB
:1051500021111DC04EED56E16E2D8F2D0F94295259
:1051600090E080E0F80EF092E018E092E1189927C4
:105170002C960FB6F894DEBF0FBECDBFDF91CF9156
:105180001F910F91FF90EF90DF90CF900895C09006
:10519000AD18D090AE1829EA38E13A8329832F2D33
:1051A00030E03C832B832E2D30E03E832D83188608
:1051B0001F827A8769871C861B8607EA1FE89E0183
:1051C0002F5F3F4F4AE458EDBC01C6010F94A33D49
:1051D000B60189EA98E10F9466518F819885C2CF14
:1051E000CF92DF92EF92FF920F931F93CF93DF93B3
:1051F000CDB7DEB72C970FB6F894DEBF0FBECDBF8C
:10520000F090E018E090E1182091B50421111DC044
:105210004EEB56E16E2D8F2D0F94295290E080E0D9
:10522000F80EF092E018E092E11899272C960FB64C
:10523000F894DEBF0FBECDBFDF91CF911F910F91CC
:10524000FF90EF90DF90CF900895C090AD18D09070
:10525000AE1829EA38E13A8329832F2D30E03C83C8
:105260002B832E2D30E03E832D8318861F827A8774
:1052700069871C861B8607EA1FE89E012F5F3F4F48
:105280004DE458EDBC01C6010F94A33DB60189EA77
:1052900098E10F9466518F819885C2CF2F923F92EB
:1052A0004F925F926F927F928F929F92AF92BF9236
:1052B000CF92DF92EF92FF920F931F93CF93DF93E2
:1052C000D62FC72FFC0180809180A280B380C501BA
:1052D000B40120E831E541E050E00F949C6BC90136
:1052E0006DE671E00F94126C6B017C01C501B40195
:1052F00020E13EE040E050E00F949C6BCA01B90110
:1053000028E130E040E050E00F949C6B362E272ED1
:10531000062F172F8CE3482E512C612C712CC501C0
:10532000B401A30192010F949C6BB62EA72ECA0163
:10533000B901A30192010F949C6BCB01C114D1045C
:1053400079F1AF92BF927F936F932F923F92FF922A
:10535000EF92DF92CF928CE094E19F938F93CF9363
:10536000DF930F940B658DB79EB70E960FB6F8942A
:105370009EBF0FBE8DBF8D2F9C2FDF91CF911F91B0
:105380000F91FF90EF90DF90CF90BF90AF909F90E4
:105390008F907F906F905F904F903F902F900895E7
:1053A000E114F104C9F0AF92BF927F936F932F92F3
:1053B0003F92FF92EF928CEF93E19F938F93CF9365
:1053C000DF930F940B65EDB7FEB73C960FB6F894DC
:1053D000FEBF0FBEEDBFCFCF012BB9F0AF92BF9292
:1053E0007F936F932F923F9280EF93E19F938F93E0
:1053F000CF93DF930F940B658DB79EB70A960FB6C8
:10540000F8949EBF0FBE8DBFB6CF892BA9F0AF9287
:10541000BF927F936F9388EE93E19F938F93CF9387
:10542000DF930F940B65EDB7FEB738960FB6F8947F
:10543000FEBF0FBEEDBF9FCFAF92BF9284EE93E150
:105440009F938F93CF93DF930F940B650F900F90E3
:105450000F900F900F900F908ECF8F929F92AF92E0
:10546000BF92CF92DF92EF92FF920F931F93CF9351
:10547000DF931092B0041092AF042FE32093B40492
:105480001092B3041092B2041092B1041092AB04C3
:105490001092AC041092AD041092AE049C01F9017C
:1054A00090812F5F3F4F9032D1F39E34C9F48181B8
:1054B00090ED980F9A3020F08D3211F08B3281F4FC
:1054C00032969F012F5F3F4F808180538A3008F4CE
:1054D0007BC09F012F5F3F4F8081803209F476C0EF
:1054E000F0934D0BE0934C0B8F010F5F1F4FC0816A
:1054F0006AE270E0C8010F94616F009731F0FC011F
:10550000319780818032E1F31182CD3429F0C435A6
:1055100019F0C73409F04BC0F80180810F5F1F4FAD
:105520008032D1F380538A3008F041C0C093B40474
:1055300030E020E04AE0DF011196429FC001439F26
:10554000900D11249C01205331098081280F311DB9
:1055500087FD3A95818190ED980F9A30C8F130938C
:10556000B3042093B2048E3261F4329690E04AE0A4
:10557000DF0131968C9150ED580F5A3058F19093CD
:10558000B104CD01DC0101964C914032D9F3CD3408
:1055900089F52E31310539F018F52731310519F02B
:1055A0002C31310539F5B093B004A093AF04DF91ED
:1055B000CF911F910F91FF90EF90DF90CF90BF9010
:1055C000AF909F908F900895F9017BCFF90181CF23
:1055D000FD01B1CF949F800D112490ED980FC8CF9D
:1055E0002537310538F027373105E8F2203A83E0D6
:1055F0003807C9F2D0914C0B40E050E0BA0110E0FE
:1056000000E0C12CD12C7601C394FD0131968C9120
:10561000882309F47FC08132E1F4CD34D1F4203203
:105620003105B9F44093AB045093AC046093AD04DE
:105630007093AE04F093B004E093AF0463E270E0C3
:10564000CF010F94616F009709F4B1CFFC01108274
:10565000AECF81548A3108F058C0DF019D9190325D
:1056600091F0A0EDA90FAA30E8F09E3271F491817B
:1056700090539A30B8F00115110519F48F010150BB
:10568000110990E013C0FD01E8CF9D3211F09B326B
:1056900091F79181A0EDA90FAA3020F09E3259F721
:1056A0009281E6CF9E2F9D1B309759F3A82FB0E033
:1056B0004601570104C0880C991CAA1CBB1C8A9582
:1056C000D2F7482959296A297B29AF56BB4F9C93A9
:1056D00080818154DF018A3108F497CFDF01819105
:1056E000882309F492CF90ED980F9A30B8F393ED98
:1056F000980F923098F38B3289F3CD010196EC919B
:10570000E03209F082CFDC01F8CF0115110501F775
:105710008D01DECF1093B0040093AF044093AB042F
:105720005093AC046093AD047093AE0440CF81E01D
:105730008093FD100895FC01659175918591949178
:1057400008959091FC0A992321F0682F80E00F942E
:10575000FA0880E00895E2E1F8E080EBDF011D92B5
:105760008A95E9F708958091C406811103C0F3DF9B
:105770000D946E558091F01882FF08C087FD06C019
:1057800040E060E070E080E090E443CA08958091DA
:105790001208882361F09091C108891308C0809194
:1057A000F01884FF04C08EE498E00D946A5380E002
:1057B0000895FC01238121110C949DE70895CF9257
:1057C000DF92EF92FF920F931F93CF93909120025D
:1057D000913009F461C0662351F010926E0410926A
:1057E0006A0410926B0410926C0410926D04C82F1E
:1057F0000F94D04DC0906A04D0906B04E0906C047C
:10580000F0906D049B01AC012C193D094E095F0914
:1058100069017A01F7FC40C020916E04C7FD15C0F4
:105820004C2F0C2E000C550B4C5F5F4FE22F022EBD
:10583000000CFF0B4E175F077CF144EFC42EDD24F4
:10584000D394E12CF12C2C1734F438EEC32E33E032
:10585000D32EE12CF12CC60ED71EE81EF91EC092E5
:105860006A04D0926B04E0926C04F0926D04022FF3
:10587000017010E084E2809FB001819F700D701B69
:10588000112460597C4F82E390E00F94612A80914B
:105890006E048F5F80936E04CF911F910F91FF90E4
:1058A000EF90DF90CF900895AC0180918F0481112B
:1058B0000EC09091C10491110BC02091090230914A
:1058C0000A022150310981E0421753070CF080E0B1
:1058D00008950F931F9341E050E0082E02C0440F3B
:1058E000551F0A94E2F7052E000C660B770B00910A
:1058F000BA041091BB042091BC043091BD04402B2C
:10590000512B622B732B4093BA045093BB046093CA
:10591000BC047093BD0490911F02891303C081E001
:105920008093F60A1F910F910895CF93C82F882373
:1059300079F020E030E0A9016091AF067091B006E7
:105940008091B1069091B2060F9472658823C9F0D8
:105950008091AE068C17A9F00E94BFF28EE49BE006
:105960000E94E1F28091AE0691E089278093AE0615
:10597000882321F08EE49BE00E94BCF1CF910D942E
:105980007E05CF910895CF92DF92EF92FF9280E053
:10599000CCDF1092A6061092A7061092A8061092CD
:1059A000A9061092A2061092A3061092A4061092C5
:1059B000A5061092B3061092B4061092B506109286
:1059C000B6061092AF061092B0061092B106109271
:1059D000B20645EC56E029E0C12CD12C60ECE62E55
:1059E0006FE7F62E90E080E0FC01EE0FFF1FEE0F58
:1059F000FF1FE40FF51FC082D182E282F38201967D
:105A00008930910589F721504C5D5F4F2111EACF14
:105A1000FF90EF90DF90CF9008954F925F926F923A
:105A20007F928F929F92AF92BF92CF92DF92EF922E
:105A3000FF921F93CF93DF93EC01162F2091AA06BC
:105A40003091AB064091AC065091AD0668817981EA
:105A50008A819B810F947265882309F4ACC0B09051
:105A6000AE0680E062DFC880D980EA80FB8020E05B
:105A700030E0A901C701B6010F947B6E18161CF027
:105A8000C12CD12C7601C092AA06D092AB06E0922E
:105A9000AC06F092AD062DEB37E346E855EBC701B7
:105AA000B6010F947B6E87FD0BC02DEB37E346E804
:105AB00055E3C701B6010F94726518160CF077C054
:105AC000A701960160E070E080E89FE30F94306DDD
:105AD000609394067093950680939606909397062C
:105AE00080EF9FEFA9E7B4EC809390069093910626
:105AF000A0939206B0939306BB2009F45CC040903B
:105B00004E0B50904F0B6090500B7090510B80904B
:105B1000520B9090530BA090540BB090550BC0902B
:105B2000560BD090570BE090580BF090590B81E03A
:105B3000FCDE112309F43FC020914E0B30914F0B36
:105B40004091500B5091510BC301B2010F947265FB
:105B500081111CC02091520B3091530B4091540B7A
:105B60005091550BC501B4010F94726581110EC09F
:105B70002091560B3091570B4091580B5091590B77
:105B8000C701B6010F9472658823A9F0DF91CF9108
:105B90001F91FF90EF90DF90CF90BF90AF909F90BC
:105BA0008F907F906F905F904F900D94E00560E034
:105BB00070E0CB018DCFDF91CF911F91FF90EF90DF
:105BC000DF90CF90BF90AF909F908F907F906F901D
:105BD0005F904F9008954F925F926F927F928F9255
:105BE0009F92AF92BF92CF92DF92EF92FF920F936C
:105BF0001F93CF93DF93EC012091A2063091A3066F
:105C00004091A4065091A506688179818A819B8183
:105C10000F94536C6B017C012091A6063091A7066E
:105C20004091A8065091A9066C817D818E819F814B
:105C30000F94536C4B015C01A701960160916204C3
:105C40007091630480916404909165040F9472656F
:105C5000882309F459C0C0926204D0926304E09290
:105C60006404F092650420915A0430915B044091E1
:105C70005C0450915D04C701B6010F94D7652B01F8
:105C80003C010F94C96D6B017C0120E030E0A9015B
:105C90000F94726587FD79C020E030E040E051E468
:105CA000C701B6010F947B6E18162CF4C12CD12CB1
:105CB000E12CC1E4FC2EA7019601C301B2010F94AF
:105CC000536C2B013C0120E030E0A9010F94726578
:105CD00087FD5FC040925204509253046092540476
:105CE00070925504C701B6010F94986D60935004EB
:105CF000062E000C770B6F5F7F4F6830710514F034
:105D000068E070E060934E04D0914C041091500410
:105D1000A501940160916604709167048091680404
:105D2000909169040F94726581113CC0D11393C0A6
:105D30002091340430913504409136045091370459
:105D400060915204709153048091540490915504D1
:105D50000F94D765209138043091390440913A046A
:105D600050913B040F94546CDF91CF911F910F9190
:105D7000FF90EF90DF90CF90BF90AF909F908F906B
:105D80007F906F905F904F900895C12CD12C760139
:105D900092CF109252041092530410925404109215
:105DA0005504A0CF8092660490926704A092680484
:105DB000B092690420915E0430915F0440916004C8
:105DC00050916104C501B4010F94D7654B015C018A
:105DD0000F94C96D6B017C0120E030E0A9010F94A4
:105DE000726587FDFCC020E030E040E051E4C7016F
:105DF000B6010F947B6E18162CF4C12CD12CE12C1B
:105E0000B1E4FB2EA7019601C501B4010F94536CB8
:105E10004B015C0120E030E0A9010F94726587FD21
:105E2000E2C08092560490925704A0925804B09217
:105E30005904C701B6010F94986D60935104062E62
:105E4000000C770B6F5F7F4F6830710514F068E0CE
:105E500070E060934F04C0915104D11305C080914C
:105E60004D048C1709F470C0809150049091510436
:105E700090934D0480934C040C2E000CDD0B29E014
:105E80001203C0011124FC01EC0FFD1FEE0FFF1FD8
:105E9000EE0FFF1FEB53F94F208131814281538177
:105EA000209348043093490440934A0450934B0490
:105EB00000914F04002E000C110BFC01E00FF11FAC
:105EC000EE0FFF1FEE0FFF1FEB53F94F6081718143
:105ED000828193810F94536C6093440470934504C2
:105EE000809346049093470420914E0439E02303A5
:105EF000F0011124CE0FDF1FCC0FDD1FCC0FDD1FF3
:105F0000CB53D94F288139814A815B81209340044A
:105F1000309341044093420450934304E00FF11F37
:105F2000EE0FFF1FEE0FFF1FEB53F94F60817181E2
:105F3000828193810F94536C60933C0470933D0471
:105F400080933E0490933F048090560490905704B1
:105F5000A0905804B0905904209144043091450415
:105F60004091460450914704C501B4010F94D76590
:105F7000209148043091490440914A0450914B04C7
:105F80000F94546C6B017C01C0923804D092390498
:105F9000E0923A04F0923B0420913C0430913D049D
:105FA00040913E0450913F04C501B4010F94D76560
:105FB00020914004309141044091420450914304A7
:105FC0000F94546CA70196010F94536C60933404A2
:105FD000709335048093360490933704A9CEC12C76
:105FE000D12C76010FCF10925604109257041092C4
:105FF0005804109259041DCFE2E6F4E080EF9FEFC1
:10600000A9E7B4EC84839583A683B78380839183C7
:10601000A283B383ECE4F4E08DE981838083089567
:106020008F929F92AF92BF92CF92DF92EF92FF92A8
:10603000FC0198E0AFEAB6E001900D929A95E1F785
:1060400088E0FB01A2EAB6E001900D928A95E1F7A3
:10605000C090AF06D090B006E090B106F090B206C6
:1060600020E030E0A901C701B6010F9472658823D2
:10607000E1F1A701960160E070E080E89FE30F94F2
:10608000306D6B017C018090B3069090B406A090B7
:10609000B506B090B60620E030E0A901C501B40114
:1060A0000F947265882329F1A501940160E070E0E6
:1060B00080E89FE30F94306DC0925A04D0925B0445
:1060C000E0925C04F0925D0460935E0470935F0460
:1060D0008093600490936104FF90EF90DF90CF90E5
:1060E000BF90AF909F908F900895C12CD12C7601D6
:1060F000CACF60E070E0CB01DFCF20913204309155
:106100003304280F391F3093330420933204209135
:10611000DA083091DB08820F931F9093DB0880939D
:10612000DA080F94D04D6093DD087093DE088093F9
:10613000DF089093E0080895CF92DF92EF92FF92EC
:106140006B017C0183E3C816D104E104F10470F013
:1061500082E3C81AD108E108F10862E370E080E048
:1061600090E00F949D4D0F949925ECCFC701B60197
:106170000F949D4DFF90EF90DF90CF900D94992557
:106180008091E108811111C080913810813079F03F
:106190009091F01892FB882780F992FF09C097FB35
:1061A000882780F991E08927089580E0089581E0AB
:1061B000089580917D1190917E11891B8F7009F453
:1061C000DFCF81E008959091F01894FB882780F943
:1061D00094FF06C081E09091581A911101C080E0AF
:1061E0000895F1DF882339F08091F01882FB882729
:1061F00080F991E0892708958091E108811105C017
:1062000080913810823009F0ECCF81E00895F4DFFE
:1062100081110DC01092BA041092BB041092BC04FC
:106220001092BD041092BE048FEF0E94B2230D9411
:106230006B0B81E00D94DE0A81E00895DC01EC91A6
:106240008E2F90E0FC01EE0FFF1FE80FF91FE05EBC
:10625000FE4E80818F77808308958F929F92AF92B8
:10626000BF92CF92DF92EF92FF920F93CF93DF9383
:106270001F92CDB7DEB75C017B0149016B01C40EF3
:10628000D51EF501808191810F94776B898300235E
:1062900011F0F7018083BE016F5F7F4FC4010F943F
:1062A000C83CF50180819181019691838083FFEF45
:1062B000EF1AFF0AEC14FD0421F780E00F90DF9144
:1062C000CF910F91FF90EF90DF90CF90BF90AF9064
:1062D0009F908F900895009719F0019789F0089585
:1062E0001092900082E0809391001092950010929D
:1062F0009400C19A8091710082608093710008952A
:106300001092A00082E08093A1001092A50010924C
:10631000A40089BB8093720008957F928F929F9210
:10632000AF92BF92CF92DF92EF92FF920F931F93A3
:10633000CF93DF93EC017B018881883108F0C1C0E5
:1063400090E0FC01EE0FFF1FE80FF91FE05EFE4E2C
:1063500080818F770F948B4319821A8288812CE079
:10636000622F0F94F96B829FB001112430E020E07E
:10637000AB01420F531FFA01EE0FFF1FE40FF51F91
:10638000E05EFE4E908197FD07C02F5F3F4F2C309F
:10639000310571F790E09FDF7880072D10E06801EC
:1063A000CC0CDD1CF601E00FF11FE05EFE4E80819B
:1063B0008068808377FC85C080E2E81682E0F8067A
:1063C0000CF03FC08A8128E532E0281B310987FDA7
:1063D0003395220F331F220F331F032E000C440B63
:1063E000550B898178E8872E912C881A910887FDB2
:1063F0009394880C991C880C991C092C000CAA08F1
:10640000BB0860E070E0CB01F7FC0AC0B701653B58
:10641000710514F064EB70E0072E000C880B990BEB
:10642000281939094A095B090F948D6B24EB30E078
:1064300040E050E00F94BE6B820E931EA41EB51E6A
:10644000740187E18715D8F0298188E890E0821BE4
:10645000910927FD9395880F991F880F991FE816BA
:10646000F906FCF402972FB7F894E601C00FD11F8C
:10647000C05EDE4E880F991F9A8389832FBF62E327
:1064800070E080E090E0DF91CF911F910F91FF903D
:10649000EF90DF90CF90BF90AF909F908F907F90C4
:1064A0004BCE2A8188E592E0821B910927FD9395C6
:1064B000880F991F880F991FE816F9069CF6C701E7
:1064C000D1CFDF91CF911F910F91FF90EF90DF908F
:1064D000CF90BF90AF909F908F907F9008950F9333
:1064E0001F93CF93C82F8B0189E691E10E94F82377
:1064F000C817A9F06C2F70E089E691E10EDFF80172
:106500006081718182819381643FF1E07F07810521
:10651000910520F464EF71E080E090E00DDE89B138
:1065200082FB882780F9CF911F910F910895CF9317
:10653000DF9300D01F92CDB7DEB78EEE92E0A0E0E1
:10654000B0E089839A83AB83BC83BE016F5F7F4FCA
:106550008AE5C5DF0F900F900F900F90DF91CF91DC
:106560000895CF93DF9300D01F92CDB7DEB78EEEA4
:1065700092E0A0E0B0E089839A83AB83BC83BE0144
:106580006F5F7F4F8AE0ABDF0F900F900F900F90FF
:10659000DF91CF910895CF93DF9300D01F92CDB7B5
:1065A000DEB786E990E0A0E0B0E089839A83AB8310
:1065B000BC83BE016F5F7F4F82E891DF0F900F9029
:1065C0000F900F90DF91CF910895CF93DF9300D07C
:1065D0001F92CDB7DEB786E990E0A0E0B0E08983F6
:1065E0009A83AB83BC83BE016F5F7F4F86E977DF01
:1065F0000F900F900F900F90DF91CF910895CF9350
:10660000DF9300D01F92CDB7DEB786E990E0A0E01F
:10661000B0E089839A83AB83BC83BE016F5F7F4FF9
:106620008CE85DDF0F900F900F900F90DF91CF916E
:106630000895CF93DF9300D01F92CDB7DEB784EFDC
:1066400091E0A0E0B0E089839A83AB83BC83BE0174
:106650006F5F7F4F8CE343DF0F900F900F900F9091
:10666000DF91CF910895CF93DF9300D01F92CDB7E4
:10667000DEB784EF91E0A0E0B0E089839A83AB833A
:10668000BC83BE016F5F7F4F80EA29DF0F900F90C0
:106690000F900F90DF91CF910895CF92DF92EF92FC
:1066A000FF921F93CF93DF9300D01F92CDB7DEB739
:1066B0008EEEC82E82E0D82EE12CF12CC982DA822F
:1066C000EB82FC82BE016F5F7F4F8AE508DF81119C
:1066D0000EC010E0812F0F900F900F900F90DF9160
:1066E000CF911F91FF90EF90DF90CF900895BBDF87
:1066F000C982DA82EB82FC82BE016F5F7F4F8AE53E
:10670000EEDE182F882329F30E9438F1E3CFCF92D1
:10671000DF92EF92FF921F93CF93DF9300D01F92EF
:10672000CDB7DEB78EEEC82E82E0D82EE12CF12C4C
:10673000C982DA82EB82FC82BE016F5F7F4F8AE002
:10674000CEDE81110EC010E0812F0F900F900F90C0
:106750000F90DF91CF911F91FF90EF90DF90CF903E
:10676000089581DFE4DEFDDEE2DEC982DA82EB82BB
:10677000FC82BE016F5F7F4F8AE0B1DE182F882355
:1067800011F30E9438F1E0CF1F920F920FB60F92D3
:1067900011240BB60F922F933F934F935F936F93F8
:1067A0007F938F939F93AF93BF93EF93FF9348EAA9
:1067B00050E064EA70E081E090E00E940828FF91D8
:1067C000EF91BF91AF919F918F917F916F915F9169
:1067D0004F913F912F910F900BBE0F900FBE0F90D6
:1067E0001F9018951F920F920FB60F9211240BB69F
:1067F0000F922F933F934F935F936F937F938F935A
:106800009F93AF93BF93EF93FF9348E950E064E900
:1068100070E090E080E00E940828FF91EF91BF9126
:10682000AF919F918F917F916F915F914F913F9128
:106830002F910F900BBE0F900FBE0F901F901895C9
:106840009091C00095FFFCCF8093C6000895CF9330
:10685000DF93EC01FE0184912196882311F0F0DF93
:10686000F9CFDF91CF910895CF92DF92EF92FF920F
:106870006A017B01ECDFC701B601FF90EF90DF906A
:10688000CF900D944A3E0F931F93CF938C01C62F48
:1068900087EC90E1DCDFC801DADF8AE3D1DF80E357
:1068A0008C0FCEDF8AE0CF911F910F91C9CF83EC7F
:1068B00092E1CDDF8AE0C4DF60E083EB92E1E3DFC9
:1068C00060E08EE992E1DFDF61E087E992E1DBDF02
:1068D00061E08CE892E1D7DF60E08DE792E1D3DF01
:1068E00061E08DE692E1CFDF60E084E692E1CBDF0C
:1068F00061E08AE592E1C7DF61E080E592E1C3DF14
:1069000061E089E492E1BFDF61E081E492E1BBDF15
:1069100061E083E392E1B7DF60E085E292E1B3DF1B
:1069200060E086E192E1AFDF60E088E092E1ABDF1A
:1069300060E082EF91E1A7DF61E081EE91E1A3DF0A
:1069400061E08CEC91E19FDF61E08DEB91E19BDFF9
:1069500061E086EB91E197DF60E089EA91E193DF06
:1069600060E082EA91E18FDF61E089E991E18BDF0C
:1069700061E084E891E187DF61E086E791E183DF10
:1069800060E08CE691E17FDF60E085E591E17BDF0F
:1069900061E088E491E177DF61E085E391E173DF15
:1069A00060E088E291E16FDF61E083E291E16BDF1B
:1069B00061E086E191E167DF60E08AE091E163DF19
:1069C00060E086EF90E15FDF60E083EE90E15BDF07
:1069D00060E084EF98E10E942E23682F61708AEDB9
:1069E00090E151DF60E08CEC90E14DCFAF92BF922F
:1069F000CF92DF92EF920F931F93CF93DF935B01C0
:106A0000EA016901882309F45AC086EA99E01FDF88
:106A1000F501608171818281938146E00F94643E2B
:106A2000E1100AC08DE999E012DF688179818A81DD
:106A30009B8146E00F94643E86E999E008DFF60109
:106A4000608171818281938143E00F94643E8FE87D
:106A500099E0FDDEF801608171818281938143E0DC
:106A60000F94643E86E899E0F2DEF60120813181E0
:106A700042815381F80160817181828193810F94F9
:106A8000536C43E00F94643EEE20D9F08AE0D8DEE8
:106A900081E799E0DCDE688179818A819B8146E02B
:106AA0000F94643E8AE0CCDE8AE0DF91CF911F91A3
:106AB0000F91EF90DF90CF90BF90AF90C1CEE110DB
:106AC000E7CFDF91CF911F910F91EF90DF90CF90A3
:106AD000BF90AF9008950F931F93CF938C01C62F53
:106AE0008BEF95E0B4DEC801B2DECC2329F08AE05A
:106AF000CF911F910F91A4CECF911F910F91089527
:106B000060E08DEF92E4E7DF83E196E0A0DE8AE0CB
:106B100097CECF93DF93EC0160E08DEF92E4DBDF63
:106B20008CE196E094DE80E28BDECE0190DE8AE09E
:106B3000DF91CF9185CE60E08DEF92E4CCDF87E1ED
:106B400096E085DE8AE07CCEDF92EF92FF920F9393
:106B50001F93CF93DF93D82E7B018A01E901D0DF09
:106B6000D0924A0B60E08DEF92E4B5DF85E093E4CC
:106B70006EDE80E265DEC7016ADE8AE061DE011555
:106B8000110511F0C801C5DF209711F0CE01C1DF5A
:106B9000DF91CF911F910F91FF90EF90DF90CBCFBE
:106BA00030E020E04AE253E4BC0182E0CDCF811125
:106BB00005C086E79FE04BDE8AE042CE8AE79FE091
:106BC000FACFCF9369ED7BE00F943343C091C406B5
:106BD000C05D80ED9BE03BDE8C2F32DE8CEC9BE0D9
:106BE00036DE8091C406CF91E2CF8BED95E02FCEBB
:106BF0002F923F924F925F926F927F928F929F92CD
:106C0000AF92BF92CF92DF92EF92FF920F931F93BA
:106C1000CF93DF93CDB7DEB72E970FB6F894DEBFD4
:106C20000FBECDBF87E00F947E228111C0C092E1DC
:106C3000C92E9BE2D92E8EE49BE09E878D87FE01B4
:106C400031961F017F0110E000E0C6010E949B2BDE
:106C5000ED85FE8581909190A190B190FE87ED87A2
:106C6000A50194010F94536C2B013C01F701408264
:106C700051826282738220E030E040EA51EC0F944E
:106C80007B6E87FD0AC020E030E040EA51E4C3019A
:106C9000B2010F94726518167CF4F801ED57FC4BA5
:106CA000E4911E164CF4B7FAB094B7F8B094F7011B
:106CB00080829182A282B382F70181909190A1900B
:106CC000B1907F0120E030E040EA51ECC501B40111
:106CD0000F947B6E87FD42C020E030E040EA51E433
:106CE000C501B4010F9472651816C4F10F5F1F4FF0
:106CF000F4E0CF0ED11C0330110509F0A6CF8DE3CF
:106D0000E82E8AE0F82E10E0F10181919191A19195
:106D1000B1911F01F70181939193A193B1937F01E9
:106D2000812F0F94D8011F5F133071F70F94E00586
:106D300060E08BE890E10E94789663E972E084E677
:106D400090E00F94612A70E060E08AE090E00F9498
:106D5000612A6AEB72E084E690E00FC046DF89EAC0
:106D600090E175DD61E08BE990E10E9478960E94E8
:106D7000059468E270E080E991E02E960FB6F894F1
:106D8000DEBF0FBECDBFDF91CF911F910F91FF905E
:106D9000EF90DF90CF90BF90AF909F908F907F90BB
:106DA0006F905F904F903F902F900D94612A2E9698
:106DB0000FB6F894DEBF0FBECDBFDF91CF911F910C
:106DC0000F91FF90EF90DF90CF90BF90AF909F908A
:106DD0008F907F906F905F904F903F902F9008958D
:106DE00085ED95E034CD811101C0FACF0895CF93A0
:106DF00084E50E94A623C0E08823E9F00E94CD2507
:106E0000C82F1816C4F4ECDF8DE41ADD6091B204CB
:106E10007091B30490E080E00F94E03D80EF9BE040
:106E200016DD6C2FCC0F770B880B990B0F944A3E15
:106E30008AE006DDCFEF8C2FCF9108958F929F923D
:106E4000AF92BF92CF92DF92EF92FF920F931F9378
:106E5000CF93DF939091F70A93FDF1C0C82FC7DF5E
:106E6000082F87FDECC089E40E94A623882309F43B
:106E700068C00E94CD2590E08330910514F082E037
:106E800090E026E0289FF001299FF00D1124E357A0
:106E9000F54F80819181D0E00F94C01261E08C2F7A
:106EA0000E942AEB6091FA107091FB10072E000CE3
:106EB000880B990B0F9478656B017C018090F6101C
:106EC0009090F710A090F810B090F910A5019401DF
:106ED0000F947B6E18161CF01D2FD1113BC0C111F1
:106EE000A2C0A5019401C701B6010F947B6E1816CC
:106EF0000CF077C011E089E196E19F938F9381E9CF
:106F000094E19F938F931F920E94C7D30F900F908D
:106F10000F900F900F90112331F08BEC95ED909323
:106F20003B1080933A1011E015C082E50E94A62321
:106F3000882379F00E94BD25AFCF60E070E0CB01DF
:106F400026C083E50E94A623D82F8111F3CFC1115B
:106F5000ECCF10E083E50E94A623882331F00E9445
:106F6000BD25909357028093560282E40E94A62387
:106F7000882331F00E94BD259093590280935802D6
:106F800086E40E9458238823C1F20E940A25609358
:106F90005A0270935B0280935C0290935D02FF241F
:106FA000F39420E030E0A9010F947265811101C0D3
:106FB000F12CF0925E02CC2309F441C0112309F4B4
:106FC0003EC06D2F802FDF91CF911F910F91FF90C9
:106FD000EF90DF90CF90BF90AF909F908F900C94E8
:106FE0006DE986E894E19F938F9381E994E19F9303
:106FF0008F931F920E94C7D30F900F900F900F9006
:107000000F908BCF89E196E19F938F9381E994E173
:107010009F938F931F920E94C7D30F900F900F9052
:107020000F900F9080CFA5019401C701B6010F9476
:107030007B6E18163CF310E086E894E15ECFDF919A
:10704000CF911F910F91FF90EF90DF90CF90BF9065
:10705000AF909F908F9008954F925F926F927F9222
:10706000AF92BF92CF92DF92EF92FF920F931F9356
:10707000CF93BDDE87FD97C08091AB0484FD09C02E
:107080008091AD0487FD05C08091AE04837009F442
:107090007AC08AECA82E82E0B82E02E01BE0C0E0A5
:1070A000F50181915F010E94A623882349F0C33036
:1070B000D9F00E940A25F801648B758B868B978B1B
:1070C000CF5F0C5F1F4FC43059F7CF911F910F91C5
:1070D000FF90EF90DF90CF90BF90AF907F906F9038
:1070E0005F904F900C949CF20E940A256B017C01EA
:1070F00020E030E040EA51E40F94726587FF3AC027
:10710000A70196016091220B7091230B8091240BB3
:107110009091250B0F94306D2B013C01AC019B012C
:107120006091320B7091330B8091340B9091350B41
:107130000F94D7656093320B7093330B8093340BAD
:107140009093350B6091D90A7091DA0A8091DB0A2D
:107150009091DC0A0F947665A30192010F94D76594
:107160000F949D6D6093D90A7093DA0A8093DB0ABD
:107170009093DC0AC092220BD092230BE092240B56
:10718000F092250B9DCF81E0CF911F910F91FF9041
:10719000EF90DF90CF90BF90AF907F906F905F9017
:1071A0004F900D945F43CF911F910F91FF90EF90FF
:1071B000DF90CF90BF90AF907F906F905F904F9097
:1071C00008950F931F93CF93811111C0C42F8B018A
:1071D00007DE8DEE9BE03BDBC80139DBCC2339F0C9
:1071E0008AE32EDB8AE0CF911F910F9129CBCF91BB
:1071F0001F910F9108954F925F926F927F928F929D
:107200009F92AF92BF92DF92EF92FF920F931F93E4
:10721000CF93DF93CDB7DEB764970FB6F894DEBF98
:107220000FBECDBF87E00F94F801811111C080918E
:10723000AB049091AC04A091AD04B091AE046EE0AB
:10724000B695A795979587956A95D1F780FDB0C0BB
:107250000E94BFF20F94D04D6093DD087093DE085A
:107260008093DF089093E008109232026091AE069E
:107270008CE40E94ED25D82E80E00E94952C0F947E
:107280004A0381E080933A0A0F9435078091AB045A
:107290009091AC04A091AD04B091AE0459E1B695C3
:1072A000A795979587955A95D1F7282F2170F22E9B
:1072B00010E080FF0DC081E00F94F801082F82E0FC
:1072C0000F94F80111E0811101C010E0011188C094
:1072D0008091AB049091AC04A091AD04B091AE0448
:1072E00047E1B695A795979587954A95D1F780FD83
:1072F00077C011110DC00091AE04017001130AC0D6
:10730000012FF11207C011E001E0FF24F39402C045
:10731000012F10E082E50E94A623E82E812C912CFB
:1073200030ECA32E30E4B32E882321F00E940A25EE
:107330004B015C01898A9A8AAB8ABC8AE11054C0ED
:10734000E12E111104C0E02E011101C0EF2C80913B
:10735000000B61E082FD64C052C060E083E298E00F
:107360000E9478963DDD81E198E071DA0F947E0508
:107370008091390A80933A0AFF2071F080E090E012
:10738000A0E2B1E489839A83AB83BC8341E061E0EE
:10739000CE0101960F944904DD2019F081E00E948E
:1073A000952C0F94310383E0809365020F94E005E0
:1073B00064960FB6F894DEBF0FBECDBFDF91CF91BC
:1073C0001F910F91FF90EF90DF90BF90AF909F9033
:1073D0008F907F906F905F904F900895F82EC6CF5A
:1073E00011118ECF11E087CF20E030E0A901C50157
:1073F000B4010F947265EE24E3948823C1F0A501D3
:1074000094016091560B7091570B8091580B90919D
:10741000590B0F94546C698B7A8B8B8B9C8B60E02F
:10742000EE2039F040E0CE0141960F9449041BD97B
:107430007ED8112309F45CC0002309F456C01092D1
:107440004E0B10924F0B1092500B1092510B10924A
:10745000520B1092530B1092540B1092550B0F9429
:107460007E058EED9BE6ADE8B2E48D879E87AF8703
:10747000B88B87E49BE20E949B2B20E030E040EC3D
:107480005FE30F94D765905869837A838B839C83DD
:1074900083E49BE20E949B2B20E030E040EC5FE322
:1074A0000F94D765905869877A878B879C879E0150
:1074B000235F3F4F46E55BE0BE016F5F7F4FCE012C
:1074C00009960F9469030F949E0A10924E0B109226
:1074D0004F0B1092500B1092510B1092520B1092B6
:1074E000530B1092540B1092550B80E00F944409EB
:1074F000002319F081E00F944409FF2009F436CFEE
:107500008091AB049091AC04A091AD04B091AE0415
:1075100027E0B695A795979587952A95D1F780FD91
:10752000A2C083E00F947E22811158CF0F947E0574
:1075300020913D0A30913E0A40913F0A5091400A05
:1075400060E070E080E792E40F94536C4B015C01C3
:107550002091410A3091420A4091430A5091440AD5
:1075600060E070E080EF91E40F94536C2B013C01DC
:107570008091560B9091570BA091580BB091590BDD
:107580008093840690938506A0938606B093870621
:107590000091781110917911F80120813181428197
:1075A0005381C501B4010F94536C4B015C0180926F
:1075B0007C0690927D06A0927E06B0927F06F8012E
:1075C0002481358146815781C301B2010F94536CE8
:1075D0002B013C0140928006509281066092820607
:1075E0007092830627E137EB41ED58EB0F947B6EE9
:1075F00087FDB3CE23E030E04BE953E4C301B20191
:107600000F94726518160CF4A8CE27E137EB41ED04
:1076100058EBC501B4010F947B6E87FD9ECE23E02D
:1076200030E04BE953E4C501B4010F9472651816BC
:107630000CF493CE19861A861B861C8688E0ECE72C
:10764000F6E0DE01119601900D928A95E1F79E0118
:10765000275F3F4F46E55BE0BE016B5F7F4FCE018A
:1076600001960F94690382E00F9444097FCECF9373
:10767000C82F82E0C11184E040E060E00E942094C5
:10768000AFDB84E396E0CC2311F089E496E0CF9160
:10769000DEC8CF92DF92EF92FF926A017B01D7D8CA
:1076A00042E0C701B601FF90EF90DF90CF900D94BC
:1076B000643ECF93DF93C82F41E06AEE7AE081DD2C
:1076C0008C2F91DBC2EFD0E148A159A16AA17BA127
:1076D00081EE9AE0DEDF21E732EB47E25EE36CA168
:1076E0007DA18EA19FA10F94306DAB01BC018EEDE9
:1076F0009AE0CFDF21E732EB47E25EE368A579A5A8
:107700008AA59BA50F94D765AB01BC018BED9AE0D0
:10771000C0DF8AE0DF91CF9193C8CF93DF9366E01B
:107720007AE00F943343C2E0DBE04CA15DA16EA18F
:107730007FA18DEF99E0ADDF48A559A56AA57BA58E
:107740008CE494E4A6DF4CA55DA56EA57FA589E435
:1077500094E49FDF48A959A96AA97BA986E494E427
:1077600098DF8AE0DF91CF916BC8CF93DF9361EE12
:1077700079E00F943343C2E0DBE0688179818A814C
:107780009B810F947665AB01BC0188ED99E081DFA8
:107790006C817D818E819F810F947665AB01BC01E8
:1077A0008CE494E476DF688579858A859B850F94DF
:1077B0007665AB01BC0189E494E46BDF6C857D8563
:1077C0008E859F850F947665AB01BC0186E494E4B9
:1077D00060DF8AE0DF91CF9133C85BDF8AE030C899
:1077E000CF93DF936FE770E10F943343CDE3DAE09B
:1077F000488159816A817B8186E790E14ADF4C812B
:107800005D816E817F818CE494E443DF48855985F6
:107810006A857B8589E494E4DF91CF91DECFCF93B5
:10782000DF9364E07BE00F943343C6ECD0E148A1E2
:1078300059A16AA17BA18BEF9AE02BDF21E732EB04
:1078400047E25EE36CA17DA18EA19FA10F94306DF4
:10785000AB01BC0188EF9AE01CDF21E732EB47E285
:107860005EE368A579A58AA59BA50F94D765AB01B2
:10787000BC0185EF9AE0DF91CF91AFCF66E87AE067
:107880000F9433436091120B7091130B8091140B82
:107890009091150B0F947665AB01BC018DE79AE0D2
:1078A000F8DE4091420B5091430B6091440B709174
:1078B000450B8AE79AE0EDDE4091460B5091470B6D
:1078C0006091480B7091490B87E79AE0E2DE4091A6
:1078D000C90A5091CA0A6091CB0A7091CC0A84E718
:1078E0009AE07BCFCF93DF936AE27AE00F94334341
:1078F000C2E0DBE04CA95DA96EA97FA981E29AE014
:10790000C8DE48AD59AD6AAD7BAD8EE19AE0C1DE0F
:107910004CAD5DAD6EAD7FAD87E79AE0DF91CF9165
:107920005CCFCF93811110C040E066EC79E049DC78
:107930008091C306811104C089EB99E00E9427342D
:107940008AE00E9420344CDAC091C30680EB99E0B3
:107950000E9427346C2F70E090E080E00F944A3E44
:107960004091BF065091C0066091C1067091C20659
:107970008DEA99E0CF9131CF2F923F924F925F9253
:107980006F927F928F929F92AF92BF92CF92DF922F
:10799000EF92FF920F931F93CF93DF93CDB7DEB794
:1079A000C955D1090FB6F894DEBF0FBECDBF2DB7B4
:1079B0003EB724963FAF2EAF249787E00F947E22E8
:1079C000382E81110BC061E086E50E94FF258DA74E
:1079D000853070F08CE499E00E9427342496EEAD57
:1079E000FFAD24970FB6F894FEBF0FBEEDBF33C4B2
:1079F0003DA5332321F08CE299E00E9427346AE010
:107A000080E50E94FF25D82E8CEF8D0D8F3218F067
:107A100088E099E0E1CF60E085E40E94ED258823CD
:107A200009F44AC081E022968FAF22970091781125
:107A300010917911D8012D913D914D915C916091FA
:107A40004E0B70914F0B8091500B9091510B0F94F6
:107A5000546CAB01BC0188E50E94382569877A87A0
:107A60008B879C87F80124813581468157816091FD
:107A7000520B7091530B8091540B9091550B0F94B6
:107A8000546CAB01BC0189E50E9438256D877E8767
:107A90008F87988BBE01635F7F4FCE0109960F944D
:107AA000AA43C82E81110DC063E684EF98E00E94BE
:107AB00078968CED98E090CF93E022969FAF229736
:107AC000B5CF8CE40E945823182F882309F46CC189
:107AD0000E94CD258EA7803118F085EB98E07CCFF1
:107AE000FEA5F13009F462C160E083E50E94ED2556
:107AF00025968FAF2597882321F0111102C037E01A
:107B00003EA78DA5833020F08BE998E00E942734B2
:107B10009091AE062C969FAF2C9780E00E94952CFA
:107B20000F944A031D8E1E8E1F8E18A219A21AA230
:107B30001BA21CA283EF9FE4A3ECB7E48DA39EA33A
:107B4000AFA3B8A783EF9FE4A3ECB7EC89A79AA7EC
:107B5000ABA7BCA7AD2DB0E0BCAFABAFEDB7FEB7E8
:107B600024E0D29EE019F10911240FB6F894FEBF6B
:107B70000FBEEDBF8DB79EB7019627969FAF8EAF14
:107B800027978091FD0A882309F413C160E070E013
:107B900080EE90E400E010E020E830EC09831A83E6
:107BA0002B833C8320E030E040EA50E40F94546C97
:107BB0006D8B7E8B8F8B988FDE0155967D018E01AC
:107BC0000F5F1F4F2DA522964FAD2297BE01635F19
:107BD0007F4FCE0109960F94A4459B01AC010F94F1
:107BE0000A6F8111E9C20F94D04D611571058105AD
:107BF000910511F00F9407613C2C212C21961CAEAD
:107C00001DAE1EAE1FAE2197EEA5E150FF0B66968E
:107C1000FFAFEEAF66978D2D90E0B0E0A0E06A96E2
:107C20008CAF9DAFAEAFBFAF6A97A22DB0E0BCAB3B
:107C3000ABABEBADFCADAE17BF070CF0BDC2119600
:107C4000B8ABAFA7FF93EF93BF93AF9387E898E0EC
:107C50009F938F9381E998E09F938F931F920E9447
:107C6000C7D32DB73EB7275F3F4F0FB6F8943EBF3F
:107C70000FBE2DBF3EA5332309F492C10F94B86007
:107C80002AE030E040E050E00F94BE6B0F9478653E
:107C900020E030E040EA50E40F947B6E0FEF1FEFDE
:107CA000181614F001E010E00F94B86028E631E0F7
:107CB00040E050E00F94BE6B0F9478652B013C01BF
:107CC0000F94B86021E230E040E050E00F94BE6BCA
:107CD0006B5F7F4F8F4F9F4F0F9478656FAB78AF7F
:107CE00089AF9AAF8DA58430D1F44FA958AD69AD55
:107CF0007AAD89E798E0CDDCB301A20181E798E095
:107D0000C8DC8BE698E00E9427340130110519F495
:107D100083E40E94203487E698E00E942734312CC7
:107D2000C801110FAA0BBB0B64968CAF9DAFAEAF11
:107D3000BFAF64976696AEADBFAD66973A161B06A9
:107D40000CF02EC164966CAD7DAD8EAD9FAD649789
:107D50000F9478656B017C012596BFAD2597BB23F9
:107D600061F1AC019B010F94546C20E030E040E9DC
:107D700052E40F94D7659B01AC01C301B2010F948B
:107D8000546C2B013C0120E030E044EB53E40F94B1
:107D90007B6E18161CF520E030E044EB53E4C30181
:107DA000B2010F94536CEDCF1EA69ECE22E02EA7FB
:107DB0009BCE60E070E0CB01EDCE0F94B86024E183
:107DC00030E040E050E00F94BE6B675E7F4F8F4F16
:107DD0009F4F0F947865A7019601CBCF20E030E04C
:107DE000A901C301B2010F94726587FF0BC020E0A7
:107DF00030E044EB53E4C301B2010F94546C2B0107
:107E00003C01ECCFA0907811B0907911F50124815C
:107E10003581468157816D857E858F8598890F9440
:107E2000536C60966CAF7DAF8EAF9FAF60972BEDBC
:107E30003FE049E450E4C301B2010F94D76520E06C
:107E400030E044E353E40F94306D6B017C010F94F8
:107E50002D6D2B966CAF7DAF8EAF9FAF2B97D5015D
:107E60002D913D914D915C9169857A858B859C859D
:107E70000F94536C4B015C012FA938AD49AD5AAD3D
:107E80002B966CAD7DAD8EAD9FAD2B970F94D765C6
:107E90009B01AC01C501B4010F94546C4B015C0112
:107EA00089829A82AB82BC82C701B6010F94B76EF9
:107EB0002FA938AD49AD5AAD0F94D76560962CAD5A
:107EC0003DAD4EAD5FAD60970F94546C6B017C017E
:107ED000CD82DE82EF82F88620E030E0A901C50184
:107EE000B4010F94726587FF34C019821A821B8215
:107EF0001C8220E030E0A901C701B6010F94726531
:107F000087FF3AC01D821E821F821886BDA5B4302D
:107F100071F449815A816B817C818BE598E0B9DBF2
:107F20004D815E816F8178858CE494E456DC198EF6
:107F30001A8E1B8E1C8E9E01275E3F4F46E55BE02E
:107F4000BE016B5F7F4FCE0101960F94690333949E
:107F5000F1CE20E030E04BE953E4C501B4010F94C9
:107F60007B6E181634F680E090E0ABE9B3E48983C9
:107F70009A83AB83BC83BDCF20E030E04BE953E470
:107F8000C701B6010F947B6E18160CF0BFCF80E0CE
:107F900090E0ABE9B3E48D839E83AF83B887B6CF1F
:107FA0008091FD0A882309F403C160E070E080EE4F
:107FB00090E400E010E020E830EC09831A832B8382
:107FC0003C8320E030E040EA50E40F94546C698B2D
:107FD0007A8B8B8B9C8BFE0171967F018E010F5FDC
:107FE0001F4F20E022964FAD2297BE01635F7F4F67
:107FF000CE0109960F94A4456B017C01312CAC0194
:108000009B010F940A6F811102C033243394A7019E
:108010009601C701B6010F940A6F8111CDC0EBA97B
:10802000FCA9EE0FFF1FEE0FFF1F27962EAD3FADF1
:108030002797E20FF31FC082D182E282F3822DA143
:108040003EA14FA158A5C701B6010F94726587FFE5
:1080500004C0CDA2DEA2EFA2F8A629A53AA54BA5A1
:108060005CA5C701B6010F947B6E181624F4C9A64F
:10807000DAA6EBA6FCA6A701960121966CAD7DAD14
:108080008EAD9FAD21970F94546C21966CAF7DAF50
:108090008EAF9FAF21978FA598A9092E000CAA0B30
:1080A000BB0B8FA798ABA9ABBAABBC01CD010F94AA
:1080B00078652B013C01AC019B0121966CAD7DAD37
:1080C0008EAD9FAD21970F94306D6BAB7CAB8DABBC
:1080D0009EAB6D8F7E8F8F8F98A32796AEADBFAD71
:1080E0002797B8AFAFAB10E0812C912C5401EFA9CA
:1080F000F8AD6191719181919191F8AFEFAB2BA99E
:108100003CA94DA95EA90F94536C9B01AC010F943F
:10811000D7659B01AC01C501B4010F94546C4B01B0
:108120005C011F5F211618F7A30192010F94306DB7
:108130000F94C16E69A37AA38BA39CA3FDA5F23013
:10814000A8F16FA578A989A99AA90F944A3E86E556
:1081500098E00E9427346A966CAD7DAD8EAD9FADE0
:108160006A970F944A3E80E598E00E94273443E0E6
:10817000C701B6010F94643E80E20E94203481E082
:108180002DA523300CF480E0E12C8E01075D1F4FFC
:108190009E012B5D3F4FAE014F5D5F4FBE01635EA1
:1081A0007F4F0E94F6348AE00E94203423943DCD14
:1081B00060E070E0CB01FDCE80E00E94A12B332077
:1081C000C1F185E498E00E94273481E03DA51316B3
:1081D0000CF080E0EE24E3948E01075D1F4F9E01BA
:1081E0002B5D3F4FAE014F5D5F4FBE01635E7F4F22
:1081F0000E94F63469A17AA18BA19CA108521109B1
:1082000026E042E00F944F609F938F9384E398E0C1
:108210009F938F938EE398E09F938F931F920E947A
:10822000C7D38DB79EB707960FB6F8949EBF0FBE03
:108230008DBF0F9431032C968FAD2C970E94952CF7
:108240000F94E0052496AEADBFAD24970FB6F89419
:10825000BEBF0FBEADBF24962EAD3FAD24970FB667
:10826000F8943EBF0FBE2DBFC75ADF4F0FB6F8942C
:10827000DEBF0FBECDBFDF91CF911F910F91FF9059
:10828000EF90DF90CF90BF90AF909F908F907F90B6
:108290006F905F904F903F902F900895CF93DF9312
:1082A000EB010E942734BE0190E080E0DF91CF9186
:1082B0000D94E03DCF93DF93EB010E942734BE0184
:1082C000DD0F880B990BDF91CF910D944A3E5F92A1
:1082D0006F927F928F929F92AF92BF92CF92DF92D6
:1082E000EF92FF920F931F93CF93DF931F92CDB71F
:1082F000DEB77C0139018B015B01A40EB51ED12CC8
:10830000C12CA016B10609F450C0F70180809180FD
:10831000F80151908F015982C4010F94776B581660
:10832000B9F1652DC4010F947F6BFFEFCF1ADF0AFF
:10833000C6018F779927892B21F162E070E080E0F8
:1083400090E00F949D4DC4010F94776B998189172C
:10835000F9F00E94F0368BE193E00E94273481E02F
:108360000F90DF91CF911F910F91FF90EF90DF90D1
:10837000CF90BF90AF909F908F907F906F905F90C5
:10838000089562E070E080E090E00E949C30DBCFD6
:10839000BE016F5F7F4FC3010F94C83CF70180811E
:1083A0009181019691838083ACCF80E0D9CF0E94E8
:1083B00027348AE00C942034CF93DF9369EC73E187
:1083C0000F943343C0917811D0917911488159812C
:1083D0006A817B8180EC93E15CD94C815D816E8107
:1083E0007F818CE494E455D94091741150917511BA
:1083F000609176117091771189E494E44AD98DEBFC
:1084000093E10E94273487E59FE2DF91CF91CFCFA0
:10841000CF93DF93C82F41E06BE17BE00E94E1380E
:108420008C2F0E94F336C7EBD6E04C815D816E81C4
:108430007F8182E19BE02DD9488159816A817B81CE
:108440008FE09BE026D98CE09BE00E94273487E5F3
:108450009FE2DF91CF91ABCFCF93DF93EC0160E050
:1084600085E096E00E946B35CE01DF91CF919FCFE2
:108470002F923F924F925F926F927F928F929F9234
:10848000AF92BF92CF92DF92EF92FF920F931F9322
:10849000CF93DF93CDB7DEB7CC55D1090FB6F894A3
:1084A000DEBF0FBECDBF70E060E085E40E94C02556
:1084B000182F8F3F09F480C0882309F181EB96E1E2
:1084C0000E94273489E996E1C45ADF4F0FB6F89429
:1084D000DEBF0FBECDBFDF91CF911F910F91FF90F7
:1084E000EF90DF90CF90BF90AF909F908F907F9054
:1084F0006F905F904F903F902F900C94273428EC12
:1085000030E069963FAF2EAF699783E40E94A623BF
:10851000882309F458C00E94BD258BA783E50E94DB
:10852000A623882331F00E94BD2569969FAF8EAFA8
:10853000699760E085E50E94ED252B968FAF2B971C
:1085400060E08CE896E10E9478960F94D04D6C879D
:108550007D878E879F871F3F09F0CCC469964EADFB
:108560005FAD69974F3651050CF4CCC18FE796E1AA
:108570000E94273480E696E10E94273489E396E141
:108580006BDFC45ADF4F0FB6F894DEBF0FBECDBF0E
:10859000DF91CF911F910F91FF90EF90DF90CF90DF
:1085A000BF90AF909F908F907F906F905F904F9013
:1085B0003F902F900D94E6524CE350E069965FAFE8
:1085C0004EAF6997A2CF55E05BA7A8CF20E030E07F
:1085D00040E05EE322962CAF3DAF4EAF5FAF2297F7
:1085E000CEC12AE939E949E15FE326962CAF3DAFD8
:1085F0004EAF5FAF2697D1C1B091F610B9832090EE
:10860000F7103090F8100091F91075C22A96EEAD6F
:10861000FFAD2A978083CEC24BEEC42ED12CE12C25
:10862000F12C59C384E190E0A0E0B0E0888B998BF5
:10863000AA8BBB8B34E1C32ED12CE12CF12C5BC374
:10864000C88AD98AEA8AFB8A56C32A96EEADFFAD5C
:108650002A9780831FC4D301C20128A939A94AA936
:108660005BA9821B930BA40BB50BB7FD4EC0812FEA
:1086700017FD80E00E94FCE88AE00E942034D301CC
:10868000C2018053984FAF4FBF4F88AB99ABAAAB95
:10869000BBAB9CA9911170C02DA93EA94FA958ADA3
:1086A0006981722D832D902F0F947B6E18160CF01C
:1086B0004FC020E030E040E050E46981722D832D0E
:1086C000902F0F94546C6DAB7EAB8FAB98AF2CA5F5
:1086D0003DA54EA55FA5240D351D461D571D29AF8F
:1086E0003AAF4BAF5CAF6B966CAD7DAD8EAD9FADD1
:1086F0006B970F9478652981322D432D502F0F945D
:108700007265881F8827881F8CAB8C859D85AE85F8
:10871000BF8588169906AA06BB0610F4D501C401C8
:10872000481A590A6A0A7B0A31E843163FE453069D
:1087300032E163067104B8F188E695E18DDE8BE5E0
:1087400095E10E94273489E495E10E94273462C2B2
:10875000D301C20129AD3AAD4BAD5CAD821B930B89
:10876000A40BB50B45EA58E364EB78E3B7FDCDCF36
:10877000812F0F940223C9CF67966CAD7DAD8EAD6E
:108780009FAD67970F9478659B01AC016981722D4D
:10879000832D902F0F94726587FFB7CF45E759E37C
:1087A00065E879E3E5CF28964EAD5FAD28978E81D9
:1087B0009F81481759070CF0A2C003970CF49FC083
:1087C0008CE395E10E9427348BEE94E10E942734DC
:1087D0008BED94E141DE1F3F09F073C0ABECB4E1D7
:1087E000BF83AE8389EB94E10E9427348E819F8101
:1087F0000E9427344A815B816C817D8187ED94E101
:108800000E94ED3B89EB94E10E9427348E819F8189
:108810000E9427344F8D58A169A17AA183ED94E17C
:108820000E94ED3B89EB94E10E9427348E819F8169
:108830000E9427344B8D5C8D6D8D7E8D8FEC94E185
:108840000E94ED3B2B96FFAD2B97FF23B1F121E763
:1088500032EB47E25EE36F8D78A189A19AA10F9474
:10886000D7656B017C0121E732EB47E25EE36B8D5C
:108870007C8D8D8D9E8D0F94306D2A813B814C8136
:108880005D811F3F19F12093121130931311409312
:10889000141150931511C0921611D0921711E09235
:1088A0001811F092191160931A1170931B11809393
:1088B0001C1190931D110E94972B81E0809352020E
:1088C00060CEEAECF4E1FF83EE838CCF2093E610D8
:1088D0003093E7104093E8105093E910C092EA10EB
:1088E000D092EB10E092EC10F092ED106093EE104D
:1088F0007093EF108093F0109093F110DECF0E94F0
:10890000F3BEDAC08CE296E10E94273484E296E15D
:108910000E9427340E9443EB8FE78093D01024EB12
:1089200030E0A8EEB3E00F94EA6B6CA77DA78EA7AA
:108930009FA72C853D854E855F85260F371F481FD5
:10894000591F29AF3AAF4BAF5CAF1092520260E0B3
:1089500089E196E10E94789681E08093630232E09B
:10896000310F3AA7323008F031CE8BEA9AEAAAEA00
:10897000BEE322968CAF9DAFAEAFBFAF22973AA5B4
:10898000323008F02ECE8DEC9CECACE4BEE32696A3
:108990008CAF9DAFAEAFBFAF26978C859D85AE8562
:1089A000BF8588AB99ABAAABBBAB4C015D011B8EFD
:1089B0001C8E1D8E1E8E1F8E18A219A21AA21A823C
:1089C0001B821C821D822FE730E040E050E0288BA4
:1089D000398B4A8B5B8B188630E43C8B4CE14D8B9A
:1089E00056E45E8B1F8A188E198E1A8EFFE7CF2EE3
:1089F000D12CE12CF12C1CAA1DAA1EAA1FAA18AE6C
:108A00001EA21FA218A619A681E08DA31F821E8296
:108A10001982212C312C00E069962EAD3FAD69976B
:108A2000032E000C440B550B2F962CAF3DAF4EAFD1
:108A30005FAF2F974BA5042E000C550B28965FAF08
:108A40004EAF28975CE21502C0011124DC01A4504E
:108A5000BF4E2A96BFAFAEAF2A9769968EAD9FAD37
:108A600069974E969C01990F440B550B63962CAF5A
:108A70003DAF4EAF5FAF639769968EAD9FAD69977F
:108A80004E979C01990F440B550B67962CAF3DAF49
:108A90004EAF5FAF679769964EAD5FAD6997465031
:108AA0005109CA01092E000CAA0BBB0B6B968CAFA7
:108AB0009DAFAEAFBFAF6B9780916302882309F47F
:108AC000A9C00F94D04D2B013C019091D9089DAFC6
:108AD000992309F484C00F94A9241092D9081F3F48
:108AE00009F08ACDA091CA10A9832090CB103090B4
:108AF000CC100091CD102F89388D498D5A8D698108
:108B0000722D832D902F0F947B6E18162CF4E98113
:108B1000EF8B288E398E0A8F28853C894D895E8996
:108B20006981722D832D902F0F94726587FF05C088
:108B3000F981F8872C8A3D8A0E8B2F966CAD7DAD1E
:108B40008EAD9FAD2F970F9478656C966FAF6C9735
:108B50006D967FAF6D978BA39CA32DA1222309F463
:108B60005EC09B01AC016981722D832D902F0F9403
:108B70007B6E1816A4F5B301A201481959096A09B8
:108B80007B09DB01CA0188589341A109B109B7FDEE
:108B900026C088899989AA89BB898C199D09AE0943
:108BA000BF09B595A795979587951F3F09F02ECDDD
:108BB0008093D0104EA35FA368A779A76C96FFADF2
:108BC0006C97FF8B6D962FAD6D97288F3BA1398FDA
:108BD0004CA14A8F4C865D866E867F861DA2639669
:108BE0006CAD7DAD8EAD9FAD63970F947865298197
:108BF000322D432D502F0F94726587FF2CCD81EAC3
:108C000095E10E94273482E895E10E94273489E3A8
:108C100096E122DC109263020E9443EB4ECE6C96EA
:108C20002FAD6C976D963FAD6D974BA15CA169819F
:108C3000722D832D902F0F94726587FFD0CFD301B3
:108C4000C2012C853D854E855F85821B930BA40B4D
:108C5000B50BAC01BD01485853416109710977FD5D
:108C6000BECF4E815F81452B09F403C18EA09FA02A
:108C7000A8A4B9A4880E991EAA1EBB1E2EA13FA1AE
:108C800048A559A5281B390B4A0B5B0BC701B60138
:108C90000F948D6BA50194010F94BE6BC888D98881
:108CA000EA88FB88C20ED31EE41EF51E54E1C516E9
:108CB000D104E104F1040CF4B5CC8CEEC816D10457
:108CC000E104F1040CF0A8CC90E8C916D104E10449
:108CD000F1040CF4B5CCC88AD98AEA8AFB8A8EEFF3
:108CE00090E0A0E0B0E09C01AD012C193D094E09D7
:108CF0005F0969017A01488959896A897B8981E11B
:108D000096E10E943434B701A6018CE096E10E94FE
:108D1000343448855C896D897E8985E096E10E94BE
:108D2000493B4F89588D698D7A8D8EEF95E10E9470
:108D3000493BAE81BF8113970CF49BC0C701B601BC
:108D40000F94786520E030E040E850E40F94D76558
:108D50006A837B838C839D8328853C894D895E89CA
:108D60006F89788D898D9A8D0F94536C2BED3FE030
:108D700049E450E40F94D76520E030E040E05FE341
:108D80000F94D7659B01AC016A817B818C819D81A9
:108D90000F94306D688779878A879B87C501B401F6
:108DA0000F9478652FE632E143E85AE30F94D765D4
:108DB0004B015C0126962CAD3DAD4EAD5FAD2697C7
:108DC000688579858A859B850F94D7656A837B83BF
:108DD0008C839D839B01AC010F94546CA50194017D
:108DE0000F94306D6F8F78A389A39AA32A813B815A
:108DF0004C815D81C501B4010F94D76522962CADDD
:108E00003DAD4EAD5FAD22970F94D7656B8F7C8FD4
:108E10008D8F9E8F488559856A857B8588EF95E182
:108E20000E94493BB501A40182EF95E10E94ED3B10
:108E3000BAA583EE95E1B23010F084ED95E10E9481
:108E400027344A815B816C817D818EEC95E10E94A3
:108E5000493B4F8D58A169A17AA188EC95E10E9408
:108E6000493B4B8D5C8D6D8D7E8D82EC95E10E9432
:108E7000ED3B88899989AA89BB898C0D9D1DAE1D02
:108E8000BF1DB595A795979587951F3F09F0DDCB39
:108E90008093D0102896FFAD2897FF932BA52F9392
:108EA0003F813F934E814F938EEA95E19F938F933D
:108EB00089EB95E19F938F931F920E94C7D38E8178
:108EC0009F8101969F838E830FB6F894DEBF0FBEFD
:108ED000CDBF6C96BFAD6C97B8876D96EFAD6D97B3
:108EE000EC8BFBA1FD8B2CA12E8B530142013DADE0
:108EF0003DA375CE69968EAD9FAD6997813F9F4327
:108F00000CF034CB8CE296E10E94273484E296E1A7
:108F10000E9427340E9443EB3CE21302F00111242B
:108F2000EE50FF4E8FE7828728E230E0FACCEC016A
:108F30008B01F42E0E9443EB209709F480C00E941D
:108F4000F036CE0134DA0115110511F40AEC14E102
:108F50000E94F7971F930F93DF93CF938CE995E0CF
:108F60009F938F9381E08F930E94C7D30E940594B3
:108F7000C091AA18C695C69585EA98E10E94C1BE1F
:108F8000DC2FDD0F1D2F1C0F8DB79EB707960FB678
:108F9000F8949EBF0FBE8DBF83E00E94059810928B
:108FA000E018C093E1188CE390E10E9454994DE8D9
:108FB00055E06D2F80E00E945C9940E855E0612FFC
:108FC00080E00E945C9989EA98E10F943651811102
:108FD000E3CF0E94F53585EB95E00E94273461E0F0
:108FE00083EA95E00E946B3589EE93E0019739F0B2
:108FF00000C00000EEE5F9E03197F0F7F7CFF89404
:1090000089EE93E0019739F000C00000E6EEF3E04E
:109010003197F0F7F7CF0E9443EBFF2041F00E9419
:10902000D9EC0E94F523909905C0A895FCCF0E9429
:109030009EECF7CF909B02C0A895FCCFFFCF011507
:10904000110511F40AEC14E1CCEAD5E081CF80914E
:109050006A0B90916B0B2FEF3FEF981751F0E92FB0
:10906000F0E0E659F44F228130E09F5F9F779093C4
:109070006B0BC90108952F923F924F925F926F92AE
:109080007F928F929F92AF92BF92CF92DF92EF9298
:10909000FF920F931F93CF93DF9300D01F92CDB712
:1090A000DEB7B82E8091570C843008F0D4C171E639
:1090B000D72E8091570C843008F00CC180916A0B38
:1090C00090916B0B891B8F7709F404C1C0DF97FF68
:1090D0000BC00E94F53581E694E00E942734809110
:1090E0006A0B80936B0BE5CF8A3019F08D3009F055
:1090F000E8C01092520C8091F00B9091F10BFC01A2
:10910000E451F44F1682892B19F40F949925D1CF8D
:109110001092F10B1092F00B02EF1BE0F80181911D
:10912000803209F449C08E3409F0B6C06CE574E0B1
:10913000C8010F94F1647C01892B41F06EE470E06A
:10914000C80104960F94616F009709F4C8014AE0C2
:1091500050E070E060E001960F9466622B013C01E4
:109160008091EC0B9091ED0BA091EE0BB091EF0B79
:10917000AC01BD014F5F5F4F6F4F7F4F44165506E7
:1091800066067706D9F0EF28C9F4AC01BD0141505D
:10919000510961097109441655066606770634F0CF
:1091A00084159505A605B7050CF083CF60E089E22C
:1091B00094E00F94AB427DCF8F01B0CF6AE270E0B4
:1091C000C8010F94906F9C01009709F1982F901B94
:1091D000F12C992339F09150F801E90FF11D8081AC
:1091E000F826F7CF4AE050E070E060E0C901019650
:1091F0000F9466622F2D30E050E040E06217730755
:109200008407950741F060E08AE094E0D2CF60E007
:1092100080EE93E0CECF4092EC0B5092ED0B60923B
:10922000EE0B7092EF0B80918C0A8130E1F467E4D1
:1092300070E0C8010F94616F0097A9F04AE050E018
:1092400070E060E001960F946662643071058105FC
:10925000910548F48FE393E00E94273460E085E3B2
:1092600093E00E9478968091F20B8B3309F421CF22
:109270008091570C843008F01CCF8091590C8D9D43
:10928000C001112462EF7BE0865A934F0F946C6FFC
:1092900080E00F9467420DCF8091F01880FFC3CF1C
:1092A00068E171E4C8010F94F164009731F0FC01AA
:1092B000838180538A3008F0B6CF60E086EB93E07C
:1092C00078CF20EF3BE042EF5BE062E57CE00E947C
:1092D000DA22EFCE8091F01883FDBDC082FFBBC0C3
:1092E00087FDB9C01A82198241E6F42E54E0E52EBA
:1092F00069E6D62E8091570C843008F0ACC00E94ED
:1093000012238111A8C041E050E0BE016D5F7F4F84
:1093100085E59AE10E94E0E40B8110E0019711F0ED
:109320000FEF1FEF80915D1A90915E1AA0915F1A66
:10933000B091601A8093EC189093ED18A093EE18FA
:10934000B093EF180E9412230F3F100749F48111C8
:1093500007C00E94F53589E794E00E942734CACF00
:109360004091590C242F30E00A3061F00D3051F05B
:10937000882309F462C089819A81009719F00196C7
:109380009A83898310921A0489819A81F29EF0014E
:10939000F39EF00D1124E95AF34FE80FF91F1382E1
:1093A000892B59F50F9499250E941223882309F4DB
:1093B000A1CF85E59AE10E949DE78091E718882377
:1093C00091F181508093E7188D9DC001112462E0D6
:1093D0008A51974F0F94601BE091E71824E0E29FB9
:1093E000F0011124EE51F74F6081718182819381E8
:1093F0000E9498240E9432E07DCF1A82198281E077
:109400000F9467428091EC189091ED18A091EE189E
:10941000B091EF188093530C9093540CA093550C7B
:10942000B093560CC1CF0E94A5E78091F0188860D8
:109430008093F018E0928C0A5DCF4F9DA00111241B
:10944000465A534F9E012F5F3F4F6AE174E0802FD1
:109450000E94DA224FCF0F94D04D6B017C01B110E6
:1094600005C08091E10820E0882349F0C092DD0822
:10947000D092DE08E092DF08F092E00821E08091CF
:109480008B0490918C04A0918D04B0918E04009770
:10949000A105B10551F14091DD085091DE086091C0
:1094A000DF087091E008840F951FA61FB71FB70152
:1094B000A601481B590B6A0B7B0BDB01CA01B7FDE8
:1094C00014C00E94F53587ED94E00E942734609126
:1094D0004C0B70914D0B8CEA94E00F94775440E064
:1094E00070E060E090E080E022DD90917D1180915D
:1094F0007E11981741F0C092DD08D092DE08E0920C
:10950000DF08F092E008409102025091030260915E
:10951000040270910502452B462B472B21F098172A
:1095200001F11092250480912304909124049099D4
:1095300047C00196909324048093230480912304D0
:10954000909124048E3E92400CF440C00E94F53568
:1095500089E994E00E94273488E894E00E94273447
:10956000BECF2111DECF0F94D04D0091DD081091B8
:10957000DE082091DF083091E00880900202909090
:109580000302A0900402B0900502080D191D2A1DC7
:109590003B1D601B710B820B930B97FDC2CF80911B
:1095A00025048111C0CF81E08093250480E00E94D2
:1095B000ADEC81E00E94ADEC82E00E94ADECB3CF57
:1095C000181619060CF0BACF0197B4CF80911F047A
:1095D00090912004A0912104B091220446015701EA
:1095E000881A990AAA0ABB0AD501C401B7FD3BC172
:1095F00030917D1190917E11209100028091510255
:10960000391709F491C0E0917E113FE6E39FF00124
:109610001124EB50FE4E9081899FC0011124880FC8
:10962000892F881F990B9195281741F0809300028C
:109630000F94D04D809100028093DC0880915E02EF
:10964000882309F403C18090560290905702C40108
:1096500002972091FA103091FB10281739070CF46B
:10966000F5C010917E11612C712C00E01C8280915C
:109670007D11811709F45BC0812F90E04FE6489F70
:10968000F001499FF00D1124E156FE4E458956899F
:109690006789708D452B462B472B81F4418D528D68
:1096A000638D748D452B462B472B41F4458D568D8C
:1096B000678D70A1452B462B472B99F15FE6589F8C
:1096C0009001599F300D1124B90161567E4E5B0106
:1096D000FB0161A172A183A194A10F9476651B0186
:1096E0002C01F50165A176A187A190A50F9476655F
:1096F0009B01AC01C201B1010F94306DF5012181D4
:109700003281438154810F94D7652B015C01930111
:10971000402F5C810F947B6E18161CF432010A2DC9
:10972000BC821F5F1F70A3CF9091E50A75CFB40173
:10973000990C880B990B0F947865562EA72EB82E8E
:10974000192F20915A0230915B0240915C02509196
:109750005D02B301802F9C810F94D765252D3A2D92
:109760004B2D512F0F94546C462E672E782E092FB7
:109770008090580290905902262F372F482F592F4A
:10978000652D7A2D8B2D912F0F947B6E1816CCF0B2
:10979000B401990C880B990B0F947865562EA72E5F
:1097A000B82E192F262F372F482F592F642D762D9D
:1097B000872D902F0F947B6E18161CF0542C53019C
:1097C000102F60901B0470901C0480901D049090DA
:1097D0001E04252D3A2D4B2D512FC401B3010F949A
:1097E0007B6E1816F4F420E037ED43EA5CE3652D58
:1097F0007A2D8B2D912F0F94D7651B012C0128E416
:1098000031EE4AE75FE3C401B3010F94D7659B01D2
:10981000AC01C201B1010F94546C562EA72EB82E84
:10982000192F852D9A2DAB2DB12F80931B0490936A
:109830001C04A0931D04B0931E04652D7A2D8B2D5E
:10984000912F0F94986DCB010F94C012F4E6CF0EB8
:10985000D11CE11CF11CC0921F04D0922004E092A4
:109860002104F09222040F94992580918C0A882378
:1098700009F40EC280914F02882309F47DC08091C3
:10988000F80A811179C00E94C030811105C0809111
:10989000E108882309F470C0F894649B10C080919B
:1098A0004B0290914C02A0914D02B0914E028093D8
:1098B0000E0890930F08A0931008B09311086091C0
:1098C0000E0870910F0880911008909111087894FB
:1098D00020E030E0A9010F94726587FF4DC001E0E0
:1098E0000093F80A8091E108811144C00E948035FC
:1098F00000934A0B60E08DEF92E40E946B3585E0A7
:1099000093E40E94273480E20E94203489E195E0AC
:109910000E94273480E30E9420348AE00E94203491
:109920000E949B351091900460E010278FEB96E029
:1099300069F487E095E00E946B3580E30E94203453
:109940008AE00E94203460E08AEE94E00E946B3549
:1099500085EF94E00E94273480E30E9420348AE05F
:109960000E942034112331F080EF94E090934A0A52
:109970008093490A0E94BFF290910901892F809536
:10998000817010910102811709F46CC02091F018C8
:1099900020642093F0188093010290FD10C064EFC2
:1099A00071E080E090E00E949C300E94D6E78091B8
:1099B000F01884FD98C1112309F454C002C00E941C
:1099C000B4E71230E8F100E00E948F9783E08093C3
:1099D00065020F94D04D6C597F4F8F4F9F4F60930E
:1099E000B6047093B7048093B8049093B90400232D
:1099F000C9F11230B9F58091F01884FF1BC00F94A3
:109A00000953882379F081E00F94E45440EB50E04F
:109A100062E178E086EF98E10E94E0E486EF98E169
:109A20000E949DE70E94C72B811116C00E94AB2B9C
:109A30000F946E5581E08093E6180F94A15312C0E5
:109A400060E08AE295E00E9478968091B50A8111E3
:109A5000BACF0E940594B7CF88E395E090934A0A65
:109A60008093490A0F94D04D6B017C01109106023E
:109A70001123F1F08091FB0A8823D1F04091260454
:109A800050912704609128047091290446015701E0
:109A9000841A950AA60AB70AB501A40177FD1AC06F
:109AA000833009F41BC10CF00AC181300CF00FC1E6
:109AB000212F30E0A8EEB3E00F94EA6BC60ED71E5C
:109AC000E81EF91EC0922604D0922704E0922804D2
:109AD000F092290480913810813009F073C00F94FE
:109AE000D04D6B017C0180912E0490912F04A091A8
:109AF0003004B0913104A7019601281B390B4A0BA1
:109B00005B0BDA01C901B7FD3AC0D701C601805F1E
:109B1000984DAF4FBF4F80932E0490932F04A09386
:109B20003004B093310480909C0690909D06A090E4
:109B30009E06B0909F060F94AC0AAB01BC01409307
:109B40009C0650939D0660939E0670939F0680919D
:109B50002D0A90912E0AA0912F0AB091300A8819EF
:109B60009909AA09BB09840F951FA61FB71F8093E7
:109B70002D0A90932E0AA0932F0AB093300A809159
:109B80002A0490912B04A0912C04B0912D04B701CC
:109B9000A601481B590B6A0B7B0BDB01CA01B7FD01
:109BA00011C050E8C50E5EEED51E56E3E51EF11C51
:109BB000C0922A04D0922B04E0922C04F0922D043F
:109BC0000E946CF10F9460110E94F3BE80918A0490
:109BD000882379F10F94D04D6B017C01809186042C
:109BE00090918704A0918804B0918904460157019F
:109BF000881A990AAA0ABB0AD501C401B7FD19C07F
:109C000020918A0430E0A8EEB3E00F94EA6BC60E10
:109C1000D71EE81EF91EC0928604D0928704E092F7
:109C20008804F092890480E00E94FCE88AE00E94A7
:109C3000203480918504882359F10F94D04D6B0115
:109C40007C018091810490918204A0918304B09161
:109C50008404A7019601281B390B4A0B5B0BDA0120
:109C6000C901B7FD15C02091850430E0A8EEB3E02E
:109C70000F94EA6BC60ED71EE81EF91EC09281042F
:109C8000D0928204E0928304F09284040F943453BF
:109C90000F900F900F900F90DF91CF911F910F9128
:109CA000FF90EF90DF90CF90BF90AF909F908F90FC
:109CB0007F906F905F904F903F902F9008958430E9
:109CC00009F0F6CE0E94F0368FE395E004C00E94C2
:109CD000F0368EE695E00E942734EACE0E94F036F8
:109CE00087E595E0F8CF123060F41092C0040F942D
:109CF000DC4D20E040E070E060E084E192ED0E9405
:109D00003D9201E061CE2F923F924F925F926F920F
:109D10007F928F929F92AF92BF92CF92DF92EF92FB
:109D2000FF920F931F93CF93DF93CDB7DEB7639767
:109D30000FB6F894DEBF0FBECDBF9091F70A93FD2A
:109D4000ADC1898389E40E94A623882309F4BFC199
:109D50000E94CD2590E08330910514F082E090E0E0
:109D600026E0289FF001299FF00D1124E357F54FBD
:109D7000828193811A828E36910514F08EE690E0EE
:109D80009093CF108093CE100E9462246091CE10E9
:109D90007091CF10072E000C880B990B0F947865EB
:109DA0002091CA103091CB104091CC105091CD1021
:109DB0000F947B6E60E018160CF02AC18AEA94E1D9
:109DC0000E94789611E06981612789810E942AEBBF
:109DD0003981332309F45CC1109363021C821D8214
:109DE0001E821F8219861A861B861C861E864CE3DD
:109DF0004F875CE1588B86E4898B1B8A312C90E875
:109E00009983AFEBAA8B1B82B1E0BD87812C912C8B
:109E100054016091CE107091CF10072E000C880B6A
:109E2000990B0F9478657B018C012B89332D498127
:109E30005A890F9472658823B9F02091CA10309125
:109E4000CB104091CC105091CD108A81B701811177
:109E5000E2C0C8010F947265881F8827881F8B8312
:109E6000EB8A3F2C09831A8B0F94D04D6B017C0138
:109E7000DC01CB0129853A854B855C85821B930BE0
:109E8000A40BB50BB7FD2EC0D701C60188519C4F5E
:109E9000AF4FBF4F89879A87AB87BC8780E00E940E
:109EA000FCE887E994E10E94273481149104A1041D
:109EB000B10409F4DBC0C501B40168577C4E8F4F73
:109EC0009F4F6C197D098E099F0928EE33E040E011
:109ED00050E00F949C6BCA01B9010F944A3E8AE08E
:109EE0000E94203480E0C7D80F94D04D6093DD08E5
:109EF0007093DE088093DF089093E0082090CA10EA
:109F00009091CB1098870091CC101091CD10222DFC
:109F1000392FA8016B89732D89819A890F94536C0D
:109F20002B013C0120E030E0A9010F947B6E87FFFC
:109F300004C077FA709477F8709481149104A104A6
:109F4000B10409F097C020E030E040E85FE3C301CE
:109F5000B2010F94726587FF10C0AD85812C912CE2
:109F60005401AA2331F082E8882E86E0982EA12C95
:109F7000B12C8C0C9D1CAE1CBF1CBB81BB2389F17A
:109F80002C813D814E815F812115310541055105AF
:109F900041F0D701C601821B930BA40BB50BB7FD93
:109FA00020C0222D3885A8016E857F8588899989F2
:109FB0000F94536C20E030E040E85FE30F9472654B
:109FC00087FD2EC0D701C601805A9541AF4FBF4FC4
:109FD0008C839D83AE83BF832E8698859F87088B55
:109FE000198B809163028823D9F081149104A10414
:109FF000B10461F0A8E8CA1AA3E1DA0AE108F1089D
:10A00000C818D908EA08FB08F7FE0AC01D8601CF68
:10A010008BE994E1D5CEC8010F94726587FF20C00B
:10A02000809163028823D1F11092630263960FB688
:10A03000F894DEBF0FBECDBFDF91CF911F910F917E
:10A04000FF90EF90DF90CF90BF90AF909F908F9058
:10A050007F906F905F904F903F902F900D94E652BD
:10A06000EB8A3F2C09831A8B1B82FECE8FE30E9462
:10A07000203435CF20E030E040E450E4C301B201A9
:10A080000F947B6E18160CF078CF4601570175CFF0
:10A0900081EB92E290933B1080933A1063960FB657
:10A0A000F894DEBF0FBECDBFDF91CF911F910F910E
:10A0B000FF90EF90DF90CF90BF90AF909F908F90E8
:10A0C0007F906F905F904F903F902F90089583E521
:10A0D0000E94A6238A83811108C029812223F1F2DC
:10A0E00082E50E94A6238823C9F20E94BD2543CEA3
:10A0F0002F923F924F925F926F927F928F929F9298
:10A10000AF92BF92CF92DF92EF92FF920F931F9385
:10A11000CF93DF93CDB7DEB7CF56D1090FB6F89402
:10A12000DEBF0FBECDBF2A969FAF8EAF2A972C966B
:10A130007FAF6EAF2C9749AB222EDB014D905D9027
:10A140006D907C901397A301920150582EAB3FABBA
:10A1500048AF59AF1496CD90DD90ED90FC901797D5
:10A16000D701C601B0588AAB9BABACABBDABA3016A
:10A170009201C301B2010F94D7654B015C01A701A5
:10A180009601C701B6010F94D7659B01AC01C501CB
:10A19000B4010F94546C0F94C16E64966CAF7DAF94
:10A1A0008EAF9FAF649780904E0B90904F0BA09016
:10A1B000500BB090510BA3019201C501B4010F9453
:10A1C000546C68966CAF7DAF8EAF9FAF689720914F
:10A1D000520B3091530B4091540B5091550B29A3C6
:10A1E0003AA34BA35CA3A701960169A17AA18BA115
:10A1F0009CA10F94546C6C966CAF7DAF8EAF9FAFEB
:10A200006C972A96AEADBFAD2A974D905D906D903C
:10A210007C9068962CAD3DAD4EAD5FAD6897C301A7
:10A22000B2010F94536C6DA37EA38FA398A72A96B7
:10A23000EEADFFAD2A97C480D580E680F7806C969E
:10A240002CAD3DAD4EAD5FAD6C97C701B6010F941F
:10A25000536C69A77AA78BA79CA7A3019201C5019C
:10A26000B4010F94536C4B015C012DEB37E346E8CE
:10A2700055EB0F947B6E87FD9AC12DEB37E346E8D3
:10A2800055E3C501B4010F94726518160CF48FC123
:10A29000A701960169A17AA18BA19CA10F94536C8F
:10A2A0006B017C012DEB37E346E855EB0F947B6E99
:10A2B00087FD7DC12DEB37E346E855E3C701B601C5
:10A2C0000F94726518160CF472C1C9A8C11004C2AB
:10A2D00020E330E03BAF2AAF4BED842E4FE0942ECD
:10A2E00049ECA42E40E4B42E750164012091560B74
:10A2F0003091570B4091580B5091590B2A96AEADA7
:10A30000BFAD2A9718966D917D918D919C911B9769
:10A310000F94536C762E672E582E492E6DA77EAF64
:10A320008FAF21969FAF219720915A0B30915B0BF5
:10A3300040915C0B50915D0B2A96EEADFFAD2A97D4
:10A3400064857585868597850F94536C162F072F26
:10A350008DA399A722966FAF229726967FAF269757
:10A3600027968FAF279728969FAF2897222009F42A
:10A37000A1C0312CB101032C000C880B990B0F9458
:10A3800078652BED3FE049EC50E40F94D765A501CB
:10A3900094010F94546C9B01AC016BED7FE089EC50
:10A3A00090E40F94306D69A37AA38BA39CA39B01C7
:10A3B000AC01672D762D852D942D0F94D7652B013B
:10A3C0003C0129A13AA14BA15CA1612F702F8DA165
:10A3D00099A50F94D76569A37AA38BA39CA320E1C9
:10A3E000EEE4FBE0CE010196DC0101900D922A958E
:10A3F000E1F78C01F1E02F1A3108A3019201698580
:10A400007A858B859C850F94546C69877A878B87B6
:10A410009C8729A13AA14BA15CA16D857E858F8582
:10A4200098890F94546C6D877E878F87988B20E076
:10A4300049A92C966EAD7FAD2C97C80159DE211429
:10A440003104C1F62091560B3091570B4091580BB7
:10A450005091590B2A96AEADBFAD2A9718966D91C3
:10A460007D918D919C911B970F94536C6DA77EAF3E
:10A470008FAF21969FAF219720915A0B30915B0BA4
:10A4800040915C0B50915D0B2A96EEADFFAD2A9783
:10A4900064857585868597850F94536C22966FAF7A
:10A4A000229726967FAF269727968FAF27972896D5
:10A4B0009FAF289764962CAD3DAD4EAD5FAD6497D0
:10A4C000C501B4010F94D76569AB79A38DA399A792
:10A4D00027E137EB41ED58E30F94726587FF11C117
:10A4E0002DEB37E346E855EB6DA57EAD8FAD21969C
:10A4F0009FAD21970F947B6E87FD03C12DEB37E352
:10A5000046E855E36DA57EAD8FAD21969FAD2197B1
:10A510000F94726518160CF4F4C02DEB37E346E87F
:10A5200055EB22966FAD229726967FAD26972796FC
:10A530008FAD279728969FAD28970F947B6E87FD48
:10A5400014C02DEB37E346E855E322966FAD229712
:10A5500026967FAD269727968FAD279728969FAD95
:10A5600028970F947265181644F480918C0A8330F2
:10A5700020F00E94CD260F947027C159DF4F0FB6EF
:10A58000F894DEBF0FBECDBFDF91CF911F910F9129
:10A59000FF90EF90DF90CF90BF90AF909F908F9003
:10A5A0007F906F905F904F903F902F9008952EA9CD
:10A5B0003FA948AD59AD6DA17EA18FA198A50F947B
:10A5C000D7656B017C012AA93BA94CA95DA969A5A6
:10A5D0007AA58BA59CA50F94D7659B01AC01C701FB
:10A5E000B6010F94546C6B017C012EA93FA948ADB4
:10A5F00059AD69A57AA58BA59CA50F94D7654B018C
:10A600005C012AA93BA94CA95DA96DA17EA18FA1DE
:10A6100098A50F94D7659B01AC01C501B4010F94B7
:10A62000536CA70196010F94C76C6B017C0120E06D
:10A6300030E0A9010F947265882309F49ECF20E0D1
:10A6400030E0A901C701B6010F94726587FD2DC0E6
:10A6500090E080E039A9832B8130910549F1029780
:10A6600091F120E030E0A901C701B6010F947B6EA3
:10A670004601570187FF04C0B7FAB094B7F8B09409
:10A680002BED3FE049EC50E4C501B4010F94306D6F
:10A6900020E030E040E452E40F94D7650F941A6D47
:10A6A0000F949D6D7BAF6AAF21CE82E090E0D2CF58
:10A6B0002BED3FE049EC50E4C701B6010F94536C19
:10A6C0006B017C01CECF2BED3FE049EC50E4C7019C
:10A6D000B6010F94546CF4CF40E350E05BAF4AAF47
:10A6E0002BED822E2FE0922E29ECA22E20E4B22E0A
:10A6F0003BEDC32E3FE0D32E39ECE32E30ECF32EAE
:10A70000F5CD2AE037ED43E25CE3609127027091DA
:10A7100028028091290290912A020F94D7654B015B
:10A720005C016091250270912602072E000C880BB7
:10A73000990B0F9478659B01AC01C501B4010F948E
:10A74000D7656D8F7E8F8F8F98A369A979A18DA111
:10A7500099A50F94C96D5B018C012AAD3BADB90180
:10A7600090E080E00F9476653B014C019B01AC01C9
:10A77000B501C8010F947B6E181614F053018401C3
:10A780009501A80169A979A18DA199A50F94306DB2
:10A790002B013C0120E030E040E85FE30F947B6E4A
:10A7A00018160CF098C269A979A18DA199A50F94EA
:10A7B0001A6D0F949D6D1B01198A1A8A1B8A1C8AB7
:10A7C0001D8A1E8A1F8A188E198E1A8E1B8E1C8E49
:10A7D0006230710508F454C290E080E00F94766511
:10A7E00060966CAF7DAF8EAF9FAF60979B01AC0161
:10A7F000C701B6010F94306D6AAF7BAF8CAF9DAFD0
:10A800009B01AC010F94D7656B017C01AC019B01EE
:10A810006AAD7BAD8CAD9DAD0F94D76520E030E087
:10A8200040EC50E40F94306D9B01AC016AAD7BAD00
:10A830008CAD9DAD0F94536CA0966CAF7DAF8EAF79
:10A840009FAFA09720E030E040E05FE3C701B60192
:10A850000F94D7659B01AC0160E070E080E89FE356
:10A860000F94536CA4966CAF7DAF8EAF9FAFA4973F
:10A8700060962CAD3DAD4EAD5FAD60976DA57EADE4
:10A880008FAD21969FAD21970F94306DAC966CAF34
:10A890007DAF8EAF9FAFAC9760962CAD3DAD4EAD0A
:10A8A0005FAD609722966FAD229726967FAD269773
:10A8B00027968FAD279728969FAD28970F94306DD8
:10A8C000E0966CAF7DAF8EAF9FAFE0978091560B57
:10A8D0009091570BA091580BB091590B89879A878B
:10A8E000AB87BC8780915A0B90915B0BA0915C0B5E
:10A8F000B0915D0B8D879E87AF87B88B0F94D04D3D
:10A900009B01AC0128533F4F4F4F5F4FA8962CAF90
:10A910003DAF4EAF5FAFA8974090060B5090070B2E
:10A920006090080B7090090B6091020B7091030B03
:10A930008091040B9091050B461657066806790620
:10A9400010F4C301B2010F94766525966CAF7DAF0C
:10A950008EAF9FAF2597A090260BB090270BC0908D
:10A96000280BD090290BC301B2010F9476657B01AF
:10A970008C019B01AC01B501C6010F94726587FD86
:10A9800002C0570168016D8D7E8D8F8D98A19B014E
:10A99000AC010F94D765562E772E4C0125962CAD21
:10A9A0003DAD4EAD5FAD259764966CAD7DAD8EAD82
:10A9B0009FAD64970F94D7657B018C019501A6012B
:10A9C000B501C6010F94D765662E7EAF8FAF219675
:10A9D0009FAF21979701A801652D772DC4010F9492
:10A9E0007B6E18161CF0E52CF72C84019701A8014A
:10A9F000662D7EAD8FAD21969FAD21970F94726528
:10AA000087FD06C06E2CFEAE0FAF21961FAF2197BB
:10AA100079A8C9A02696CFAE2697DDA02796DFAEEF
:10AA20002797E9A42896EFAE289744244394512C05
:10AA300029E12DA70F9499250F94D04D8B019C01EE
:10AA4000A896CCACDDACEEACFFACA8970C191D09F8
:10AA50002E093F0937FD0FC09B01AC0128533F4F22
:10AA60004F4F5F4FA8962CAF3DAF4EAF5FAFA8974B
:10AA700080E00E943B483DA531503DA7332309F4B7
:10AA800056C12EA93FA948AD59ADA0966CAD7DAD7C
:10AA90008EAD9FADA0970F94D7656B017C012AA95D
:10AAA0003BA94CA95DA9A4966CAD7DAD8EAD9FADC3
:10AAB000A4970F94D7659B01AC01C701B6010F9411
:10AAC000546C7B018C012EA93FA948AD59ADA496C9
:10AAD0006CAD7DAD8EAD9FADA4970F94D7654B0146
:10AAE0005C012AA93BA94CA95DA9A0966CAD7DADDE
:10AAF0008EAD9FADA0970F94D7659B01AC01C501AA
:10AB0000B4010F94536C6EAB7FAB88AF99AFC701A4
:10AB1000D8018AAB9BABACABBDAB68962CAD3DAD61
:10AB20004EAD5FAD68976EA97FA988AD99AD0F94C2
:10AB3000546C69837A838B839C832AA93BA94CA993
:10AB40005DA96C966CAD7DAD8EAD9FAD6C970F948D
:10AB5000546C6D837E838F839887AC962CAD3DAD0E
:10AB60004EAD5FADAC9769857A858B859C850F94DA
:10AB7000546C69877A878B879C87E0962CAD3DADB6
:10AB80004EAD5FADE0976D857E858F8598890F947A
:10AB9000546C6D877E878F87988BCE0101960F94BA
:10ABA000890260962CAD3DAD4EAD5FAD609769A951
:10ABB00079A18DA199A50F94306D9B01AC01672DF2
:10ABC00026967FAD269727968FAD279728969FAD1F
:10ABD00028970F94536C762E26967FAF269727964C
:10ABE0008FAF279728969FAF289725962CAD3DAD20
:10ABF0004EAD5FAD2597CA01B9010F94546C272D56
:10AC000026963FAD269727964FAD279728965FAD9E
:10AC100028970F94D7657B018C01262D3EAD4FAD53
:10AC200021965FAD21970F947B6E181634F4E62CB5
:10AC3000FEAC0FAD21961FAD2197C701D801898FBA
:10AC40009A8FAB8FBC8FAE014F5E5F4FBE01635ECC
:10AC50007F4FCE0101960F94E248882389F06496D5
:10AC6000CCACDDACEEACFFAC6497CD8ADE8AEF8A6B
:10AC7000F88E2FEF421A520A2414350409F0DACE66
:10AC800080E12A96EEADFFAD2A97DE011196019084
:10AC90000D928A95E1F7CE0101960F9489021D8AE3
:10ACA0001E8A1F8A188E198E1A8E1B8E1C8EAE015C
:10ACB0004F5E5F4FBE01635E7F4FCE0101960F94E2
:10ACC000E24880E1FE013196AEE4BBE001900D92D6
:10ACD0008A95E1F752CC2DEC3CEC4CEC5DE3C301E2
:10ACE000B2010F94726587FF1FC02DEC3CEC4CEC59
:10ACF0005DE369A979A18DA199A50F94306D0F9499
:10AD0000C96D4B015C0120E030E040E85FE30F9447
:10AD1000726587FF06C0812C912C90E8A92E9FE3D5
:10AD2000B92EC501B40145CDB501C80142CDB2016E
:10AD300090E080E00F9476652AAD3BAD4CAD5DAD03
:10AD40000F94D7656B017C010F942D6D6DA77EA7C5
:10AD50008FA798ABC701B6010F94B76E4B015C018A
:10AD60002C96AEADBFAD2C97CD90DD90ED90FC90C4
:10AD70001397F7FAF094F7F8F09414962D913D910B
:10AD80004D915C9117972AAB3BAB4CAB5DAB2DA5BE
:10AD90003EA54FA558A9C701B6010F94D7656EAB64
:10ADA0007FAB88AF99AFA50194016AA97BA98CA953
:10ADB0009DA90F94D7659B01AC016EA97FA988ADB1
:10ADC00099AD0F94546C6EAB7FAB88AF99AFA50172
:10ADD0009401C701B6010F94D7656B017C012DA5C5
:10ADE0003EA54FA558A96AA97BA98CA99DA90F9436
:10ADF000D7659B01AC01C701B6010F94536C6AABD8
:10AE00007BAB8CAB9DABB9E1BDA787CECF93DF9376
:10AE1000C82FD62F8091F70A83FD0AC00E94CB91DC
:10AE2000882331F08091090290910A020F94C01298
:10AE300040E06D2F8BE00E942094CC2331F061E044
:10AE400080E0DF91CF910C946DE980918F0491E0C7
:10AE500089278093630280916302882379F00E949E
:10AE600046972091FA103091FB10821B930B97FFAD
:10AE700003C0919581959109029744F41092630261
:10AE80008091F70A83FF06C081E00FC080E00E9436
:10AE90003B48E1CF0E94CB918823B1F30E94F0366A
:10AEA00083E296E00E94273480E0DF91CF910895FD
:10AEB000AF92BF92CF92DF92EF92FF920F931F93C8
:10AEC000CF93DF93CDB7DEB764970FB6F894DEBFAC
:10AED0000FBECDBF0E94F736D82E87FDA3C08AE5EE
:10AEE0000E94A623882309F4AEC040E050E0BA01D6
:10AEF0008AE50E9438257B018C014D2D63E085E0B9
:10AF00000E9420942091560B3091570B4091580B82
:10AF10005091590B60E070E081EE93E40F94536C14
:10AF20005B016C019701A8010F947B6E181614F059
:10AF300075018601C701D8018D839E83AF83B887D1
:10AF400020E030E0A901B701C8010F9472658823A1
:10AF500021F0CE0105960E94C12480E090E0A8EC8B
:10AF6000B1E489879A87AB87BC8780E090E0A0E74F
:10AF7000B1E48D879E87AF87B88B8CE40E94A623AF
:10AF8000882309F465C00E940A256B017C0120E03A
:10AF900030E0A901C701B6010F947B6E87FF04C0A2
:10AFA000F7FAF094F7F8F094C98ADA8AEB8AFC8A07
:10AFB0000091FA101091FB100430110564F00E940A
:10AFC0004697801B910B97FF03C09195819591093E
:10AFD00001E004970CF400E063E080E017DF8111EA
:10AFE00040C083E0809320021092BF040E94059429
:10AFF0006D817E818F8198858B019C0130580983FA
:10B000001A832B833C8320E030E0A9010F94726502
:10B01000882321F0CE0101960E94C1241092BF0422
:10B020000E94059464960FB6F894DEBF0FBECDBFA4
:10B03000DF91CF911F910F91FF90EF90DF90CF9014
:10B04000BF90AF900895E12CF12C08EC12E455CF9D
:10B05000C090BB06D090BC06E090BD06F090BE0646
:10B0600096CF83E0E82E22E0AE01475F5F4FBE013E
:10B070006F5E7F4FCE010D960F949447B9CF6F92BC
:10B080007F928F929F92AF92BF92CF92DF92EF9278
:10B09000FF920F931F93CF93DF9300D000D01F92A6
:10B0A0001F92CDB7DEB75C014B013A01F22E680169
:10B0B0000091D3081092CF081092D0081092D108B6
:10B0C0001092D2081092D3080F9489128091FA102E
:10B0D0009091FB108C159D051CF4C6010F94C012B5
:10B0E00060E080E093DE81113DC11092BF040E94B8
:10B0F00005941C141D043CF4C6010F94C01260E0BA
:10B1000080E00E946DE940E060E088E00E942094C9
:10B1100060E081E07BDE80E090E0A8ECB1E4898330
:10B120009A83AB83BC8380E090E0A0E0B0EC8D8399
:10B130009E83AF83B887BE016F5F7F4FCE010596B8
:10B140000F94C60487E00F94F801811168C08091C4
:10B150005A0B90915B0BA0915C0BB0915D0B4091F1
:10B16000560B5091570B6091580B7091590BC09032
:10B170007304D0907404E0907504F090760400910C
:10B180006F04109170042091710430917204009347
:10B190007C0610937D0620937E0630937F06C09236
:10B1A0008006D0928106E0928206F0928306409358
:10B1B0008406509385066093860670938706809375
:10B1C000880690938906A0938A06B0938B0680E048
:10B1D00090E0A8E4B3E489839A83AB83BC83CE0177
:10B1E00001960F94F3298091770490917804A091AF
:10B1F0007904B0917A048093840690938506A09395
:10B200008606B093870680E090E0A0E6B1E48983EB
:10B210009A83AB83BC83CE0101960F94F329C12C92
:10B22000D12C88ECE82E81E4F82EC982DA82EB82F8
:10B23000FC8280E090E0A0E0B0E48D839E83AF8349
:10B24000B887BE016F5F7F4FCE0105960F94C6048D
:10B2500020E030E0A90160917B0470917C04809132
:10B260007D0490917E040F94726587FF0BC0C982A4
:10B27000DA82EB82FC82BE016F5F7F4F8BE794E046
:10B280000F94C60480917B0490917C04A0917D046E
:10B29000B0917E0480935A0B90935B0BA0935C0B50
:10B2A000B0935D0B8093880690938906A0938A06DD
:10B2B000B0938B0688E896E00F9454001092BF0478
:10B2C0000E94059461E082EE96E00E946B358091C9
:10B2D000E10881508093E1084BEC58E16AEE76E09A
:10B2E00085E00F943C4380913810823011F40F9424
:10B2F0006B0B8091E108882381F081508093E108F5
:10B300000E9432E08091C406882339F040E060E07A
:10B3100070E080E090E40E9409268091A1068823D5
:10B3200031F01092A1068091A0068093E50A0E9458
:10B33000E2230F94E6520E94059428960FB6F894E3
:10B34000DEBF0FBECDBFDF91CF911F910F91FF9058
:10B35000EF90DF90CF90BF90AF909F908F907F90B5
:10B360006F900895E12C2F2DA301B401C5010F9416
:10B370009447BFCECF92DF92EF92FF920F931F932D
:10B38000CF93DF93CDB7DEB72C970FB6F894DEBF1F
:10B390000FBECDBF83E50E94A623882321F00E9423
:10B3A000A1250E94982484E50E94A6238823A9F061
:10B3B0000E94A1256B017C010F94500BC09298064E
:10B3C000D0929906E0929A06F0929B06CD28CE285C
:10B3D000CF2819F081E0809338108091E10888230C
:10B3E00059F180E090E0A8ECB1E489879A87AB87B7
:10B3F000BC871D821E821F82188619821A821B82B8
:10B400001C8210E000E020E0AE01475F5F4FBE010C
:10B410006B5F7F4FCE01019632DE2C960FB6F8940B
:10B42000DEBF0FBECDBFDF91CF911F910F91FF9077
:10B43000EF90DF90CF9008950E94E330882381F051
:10B440000E9432E00E9407318EE498E00E94ADE84D
:10B450001092530C1092540C1092550C1092560CE2
:10B4600061E083E099E10E946B354BEC58E168EDB7
:10B4700073E185E00F943C430F94E652CECF4F9298
:10B480005F926F927F92AF92BF92CF92DF92EF92D4
:10B49000FF921F93CF93DF9300D000D01F921F9293
:10B4A000CDB7DEB75C01E62EF42E642F80E0AEDC73
:10B4B000182F81111BC0EE2021F01092BF040E94B2
:10B4C0000594812F28960FB6F894DEBF0FBECDBF2E
:10B4D000DF91CF911F91FF90EF90DF90CF90BF90C1
:10B4E000AF907F906F905F904F900895EE2029F07D
:10B4F00040E06F2D83E00E942094C12CD12C88EC79
:10B50000E82E81E4F82ECD82DE82EF82F88680E09C
:10B5100090E0A0E8BFEB89839A83AB83BC83BE0134
:10B520006B5F7F4FCE0101960F94C60460E971E016
:10B5300080E090E00E949C3080E090E0A0E8B0E4E1
:10B540008D839E83AF83B88780E090E0A0E0B1E474
:10B5500089839A83AB83BC83BE016B5F7F4FCE012F
:10B5600001960F94C60440903A0B50903B0B6090AC
:10B570003C0B70903D0BC0923A0BD0923B0BE0928B
:10B580003C0BF0923D0B80E090E0A0E1B1E48D83B4
:10B590009E83AF83B887F50180819181A281B381B9
:10B5A00089839A83AB83BC83BE016B5F7F4FCE01DF
:10B5B00001960F94C60440923A0B50923B0B609256
:10B5C0003C0B70923D0B0E949EEC64E670E080E0C4
:10B5D00090E00E949C3075CF8F929F92AF92BF9265
:10B5E000CF92DF92EF92FF921F93CF93DF9300D021
:10B5F00000D01F921F92CDB7DEB70E94F736182FEA
:10B6000087FDACC08AE50E94A623812C912C98EC82
:10B61000A92E92E4B92E882341F040E050E0BA010F
:10B620008AE50E9438254B015C01412F64E083E0EC
:10B630000E94209420E030E0A901C501B4010F94DC
:10B640007B6E18167CF580E090E0A0E6B1E48D8377
:10B650009E83AF83B8872091560B3091570B409152
:10B66000580B5091590BC501B4010F94546C6B01E8
:10B670007C0120E030E041EE53E40F94726587FDD9
:10B6800006C0C12CD12C81EEE82E83E4F82EC982AD
:10B69000DA82EB82FC82BE016B5F7F4FCE010196A6
:10B6A0000F94270485E50E945823882309F468C075
:10B6B0000E940A256B017C0120E030E0A901C7014E
:10B6C000B6010F947B6E87FF04C0F7FAF094F7F889
:10B6D000F094F7FAF094F7F8F094C982DA82EB82EA
:10B6E000FC8244E061E0CE010196C9DE20E030E05A
:10B6F000A901C501B4010F947B6E18165CF580E0BA
:10B7000090E0A0E6B1E48D839E83AF83B887A50166
:10B7100094016091560B7091570B8091580B90914A
:10B72000590B0F94536C6B017C0120E030E0A901B0
:10B730000F947B6E18161CF0C12CD12C7601C98297
:10B74000DA82EB82FC82BE016B5F7F4FCE010196F5
:10B750000F9427041092BF040E94059428960FB6F8
:10B76000F894DEBF0FBECDBFDF91CF911F91FF9048
:10B77000EF90DF90CF90BF90AF909F908F90089503
:10B7800088E01802F0011124E954F94FC080D180FB
:10B79000E280F38091CF2F923F924F925F926F920F
:10B7A0007F928F929F92AF92BF92CF92DF92EF9251
:10B7B000FF920F931F93CF93DF9300D000D000D060
:10B7C000CDB7DEB74C018B014987590161E08FEBA2
:10B7D00096E00E946B354BEC58E16CED76E085E02D
:10B7E0000F943C439091E10881E0890F8093E10838
:10B7F0008091F01882FB222720F9288782FF08C059
:10B8000087FDCCC08B7F8093F0189E5F9093E108FA
:10B810000F94A10B80E1EEE4FBE0AFE6B4E0019011
:10B820000D928A95E1F787E00F94F801782E60E099
:10B8300070E080E090E4711040C02090560B309092
:10B84000570B4090580B5090590B20E030E040E0EF
:10B8500050E4C201B1010F94546C6B017C0120E0F3
:10B8600030E041EE53E40F947B6E181634F4C12C93
:10B87000D12C81EEE82E93E4F92EF8016084F18555
:10B88000FD83F801F285FE83F801F385FF839601BD
:10B89000A701662D7D818E819F2F0F947B6E1816D8
:10B8A00024F06C2CDD82EE82FF82A2019101662DD4
:10B8B0007D818E819F810F94536C2885222349F0CE
:10B8C0002091C406222329F041E0711040E00E943B
:10B8D00009260E94BFF28091A106811109C081E072
:10B8E0008093A1068091E50A8093A0061092E50A54
:10B8F00020E030E0A901F4016081718182819381AF
:10B900000F947265882391F00E944AF281110EC053
:10B9100080E090E0A8ECB1E489839A83AB83BC8398
:10B92000BE016F5F7F4FC4010F94C604711038C011
:10B93000B80180E00F94A91020E030E0A901F501E2
:10B9400060817181828193810F947265882321F0D7
:10B9500042E06985C50193DD0E949EEC64E670E0DB
:10B9600080E090E00E949C3081E029960FB6F89428
:10B97000DEBF0FBECDBFDF91CF911F910F91FF9022
:10B98000EF90DF90CF90BF90AF909F908F907F907F
:10B990006F905F904F903F902F900895188638CF0A
:10B9A00060E086EC96E00E947896C6CFCF92DF9258
:10B9B000EF92FF92CF93DF936B017C01D42FC09164
:10B9C000FB0A83E08093FB0A81E08093FA0AC114AA
:10B9D000D104E104F10431F00F94D04DC60ED71E0E
:10B9E000E81EF91E8091FA0A882389F0C114D10457
:10B9F000E104F10421F48D2F0E943B48F3CF0F9412
:10BA0000D04D6C197D098E099F0997FDF4CF1092D6
:10BA1000FA0A8091C70A82FF07C062E370E080E003
:10BA200090E00E949C30F5CFC093FB0ADF91CF914C
:10BA3000FF90EF90DF90CF9008951F93CF93DF9307
:10BA4000D82FC62F0E94373B61E08C2F0E94DF2B3E
:10BA50000F94D04D685370458F4F9F4F6093CF0820
:10BA60007093D0088093D1089093D2081092D30895
:10BA70001091FB0A83E08093FB0A81EB96E00E9421
:10BA8000D03581E08093FA0A8091FA0A882309F47C
:10BA900066C060E08C2F0E94DF2B8091D308882342
:10BAA00009F459C040E060E08AE00E9420940E94BE
:10BAB000F03687E996E00E94273430E020E041E844
:10BAC00056E068E876E082E00E94A43541E060E05C
:10BAD00070E0CB016BDF30E020E050E040E064E755
:10BAE00076E085E00E94A43560E084E796E00E945D
:10BAF00078961092CF081092D0081092D108109228
:10BB0000D2081092D3080F94891260E080E07ED9A9
:10BB10008D2F0E94373B0F94D04D685370458F4F47
:10BB20009F4F6093CF087093D0088093D108909373
:10BB3000D2081092D30888E696E00E94D03560E0E3
:10BB400088E696E00E94789681E08093FA0A61E0A8
:10BB50008C2F0E94DF2B81E00E943B4895CF1093F1
:10BB6000FB0ADF91CF911F910895CF92DF92EF9260
:10BB7000FF920F931F93CF93DF93CDB7DEB76C97F0
:10BB80000FB6F894DEBF0FBECDBF8CE40E94A62393
:10BB9000882309F4B1C00E940A256B017C0120E0D2
:10BBA00030E0A9010F947B6E87FF04C0F7FAF09490
:10BBB000F7F8F094F7FAF094F7F8F094C98EDA8E6B
:10BBC000EB8EFC8E8CE0E2E7F2E0DE011196019054
:10BBD0000D928A95E1F788E50E94A6238823A1F0BB
:10BBE00040E050E0BA0188E50E94382520915E0BC4
:10BBF00030915F0B4091600B5091610B0F94536C2F
:10BC000069837A838B839C8389E50E94A62388239A
:10BC1000A1F040E050E0BA0189E50E94382520916A
:10BC2000620B3091630B4091640B5091650B0F9444
:10BC3000536C6D837E838F8398878AE50E94A62349
:10BC4000882351F040E050E0BA018AE50E9438258F
:10BC500069877A878B879C8740E061E080E00E945B
:10BC6000209460E080E50E94ED251D861E861F86DB
:10BC7000188A9091E108911130C09E01235F3F4FD7
:10BC8000482FBE016F5F7F4FCE01499684DD882328
:10BC900021F160E080E0D1DE898D9A8DAB8DBC8D85
:10BCA000B0588D8B9E8BAF8BB88F198A1A8A1B8ADE
:10BCB0001C8A1D861E861F86188A8091E1088823AB
:10BCC00061F010E000E020E0AE014B5E5F4FBE018E
:10BCD0006F5E7F4FCE010D96D2D96C960FB6F89459
:10BCE000DEBF0FBECDBFDF91CF911F910F91FF90AF
:10BCF000EF90DF90CF900895C12CD12CE12C80E4FF
:10BD0000F82E58CF1F920F920FB60F9211240F905A
:10BD10000FBE0F901F9018951F920F920FB60F92A3
:10BD200011240BB60F920F931F932F933F934F93B2
:10BD30005F936F937F938F939F93AF93BF93CF93B3
:10BD4000DF93EF93FF93C091C60000916B0BD091EE
:10BD50006A0B11E01D0F1F7790911704943108F0C2
:10BD6000B1C0E92FF0E08827E754F14A8F4F0D94D6
:10BD7000396CCD5EFC5E0B5F1D5F245F625F285FE8
:10BD8000625F2C5F305F625F345F385F625F3D5F90
:10BD9000425F475F4F5F625F5A5FC03229F028F50C
:10BDA000CA3011F0CD3031F5011731F0ED2FF0E050
:10BDB000E659F44FC283D12FD0936A0BFF91EF91D4
:10BDC000DF91CF91BF91AF919F918F917F916F91B3
:10BDD0005F914F913F912F911F910F910F900BBE4B
:10BDE0000F900FBE0F901F901895CD3481F081E019
:10BDF000CE3471F083E10CC0CA3338F4C033A0F6FE
:10BE0000C03291F2CD32B1F7CFCFCD3499F782E085
:10BE100080931704C9CFC43371F030F4C03221F2DB
:10BE200083E0C133A9F3E6CF8BE0C53389F38EE01D
:10BE3000C83371F3DFCF88E0EBCF84E0C03341F348
:10BE400086E0C13329F3D6CF85E0C83399F6E0CF39
:10BE500087E0C23379F6DCCF89E0C13359F6D8CF19
:10BE60008AE0C03339F6D4CF8CE0C23319F6D0CF94
:10BE70008DE0C43309F0BECFCBCF8FE0C73309F0DC
:10BE8000B9CFC6CF80E1C63309F0B4CFC1CFC0323D
:10BE900009F48ACFC33509F0ADCF81E1B9CF80ED88
:10BEA0008C0F8A3008F080CF92E190931704809332
:10BEB00016047ACFCA3019F0CD3009F075CF109240
:10BEC000170472CFCA3019F0CD3009F06DCF8091D0
:10BED000E4188823A1F39A3071F140F4953031F1E0
:10BEE000973069F781E08093CE08E9CF9D3039F132
:10BEF000923129F79091160480914A0B10924A0BC7
:10BF00008230B1F0843011F18130C9F69923D9F033
:10BF10009130A9F682E08093F90A8091F80A88238B
:10BF200071F210924F020E94E223C9CF1092630275
:10BF30001092FA0AC4CF81E08093CD08C0CF81E08F
:10BF40008093CC08BCCF8093F90AB9CF8AE099E1FD
:10BF500090934A0A8093490AB2CF8EBD0DB407FE72
:10BF6000FDCF08958FEF8EBD0DB407FEFDCF8EB5CA
:10BF70000895909164009B7F90936400982F906A3D
:10BF800096959CBD80FD03C091E0863009F490E059
:10BF90009DBD0895CF92DF92EF92FF92CF93DF93F2
:10BFA00080E50E94A623C12CD12C7601882321F0A4
:10BFB0000E94FA246B017C0183E50E94A62388235A
:10BFC00061F00E940A2520E030E04AE754E40F9433
:10BFD000D7650F949D6D6B017C010E94BFF280912B
:10BFE000AF049091B004009799F10F94B052C091B2
:10BFF000AF04D091B004209789F10E94803582E08F
:10C0000080934A0B60E08DEF92E40E946B3584E9E7
:10C0100093E10E94273480E20E942034CE010F94E5
:10C02000A4528AE00E9420348AE293E4009711F03F
:10C030000E9489350E949B3540E0C701B601B6DCFD
:10C04000DF91CF91FF90EF90DF90CF900D94E6526B
:10C0500060E08AEA93E10E947896C9CF8091B204A9
:10C060009091B304892B29F48AE993E10E94D03599
:10C07000E3CF82EA93E1FACFCF93DF93EB010E9403
:10C080002734CE01DF91CF910D94A452CF93DF934B
:10C09000CDB7DEB76A970FB6F894DEBF0FBECDBF3F
:10C0A00070E060E083E50E94C0258E34910569F45C
:10C0B0000E948EF10F94E6526A960FB6F894DEBF96
:10C0C0000FBECDBFDF91CF9108958EE794E10E941E
:10C0D00027346091290A70912A0A85E794E10E9429
:10C0E0004E4160912B0A70912C0A88E694E10E94DF
:10C0F0004E416091290A70912A0A80912B0A9091F1
:10C100002C0A681B790B80913810815021E030E0B7
:10C11000823010F030E020E0621B730B8DE594E17B
:10C120000E944E418AE00E94203485E594E10E94FD
:10C13000273480912D0A90912E0AA0912F0AB09158
:10C14000300A8F8B988FA98FBA8FBE016F5F7F4F98
:10C15000CE0147960E944E29BE016F5F7F4F88E453
:10C1600094E18ADF8091310A9091320AA091330ADA
:10C17000B091340A8F8B988FA98FBA8FBE016F5FF1
:10C180007F4FCE0147960E944E29BE016F5F7F4FC1
:10C1900088E394E171DF20E030E04AE754E4609105
:10C1A000350A7091360A8091370A9091380A0F94B7
:10C1B000306DAB01BC0180E294E10E94493B8DE609
:10C1C0000E9420348AE00E94203476CFAF92BF9242
:10C1D000CF92DF92EF92FF920F931F93CF93DF9353
:10C1E000EC0182EE95E00E942734209711F4C5EC13
:10C1F000D6E010E007E0015021F080E20E942034F8
:10C20000FACF812F0E94F6E81F5F193099F78AE074
:10C210000E94203410E080E20E942034812F0E948E
:10C22000F6E85E0109E080E20E942034F501C0805A
:10C23000D180E280F380A7019601C701B6010F9477
:10C240000A6F882361F180E20E9420348DE30E940E
:10C2500020348DE30E9420348DE30E9420348DE34E
:10C260000E9420348DE30E9420340150F4E2AF0E8E
:10C27000B11C0111D8CF8AE00E9420341F5F2496A0
:10C28000193049F68AE0DF91CF911F910F91FF900D
:10C29000EF90DF90CF90BF90AF900C94203420E0CF
:10C2A00030E0A901C701B6010F947B6E87FD03C082
:10C2B0008BE20E94203443E0C701B6010F94643E34
:10C2C000D4CF2F923F924F925F926F927F928F9234
:10C2D0009F92AF92BF92CF92DF92EF92FF920F9315
:10C2E0001F93CF93DF93CDB7DEB76C970FB6F8945B
:10C2F000DEBF0FBECDBF83E50E945823182F3090BC
:10C30000AE06882319F00E94DE25382E80914E0B50
:10C3100090914F0BA091500BB091510B898F9A8F38
:10C32000AB8FBC8F8091520B9091530BA091540B0B
:10C33000B091550B8D8B9E8BAF8BB88F8091560B28
:10C340009091570BA091580BB091590B898B9A8BF8
:10C35000AB8BBC8B112329F0311003C080E00E940D
:10C36000952C8091AB049091AC04A091AD04B09158
:10C37000AE0425E1B695A795979587952A95D1F7AF
:10C380002C013D01E1E04E2255246624772420E073
:10C3900030E0A9016091AF067091B0068091B106BE
:10C3A0009091B2060F947265882309F4D2C083E499
:10C3B0000E945823882309F4A2C00E940A254B0139
:10C3C0005C0185EC96E0998788879E838D83B9E030
:10C3D000BF831D861E86E8ECEF87F2ECF88B1A8689
:10C3E000212C28EC2B8782E48C87D12CC12CF601E0
:10C3F000EE0FFF1FEE0FFF1FAD81BE81EA0FFB1F87
:10C40000E080F180028113812A85322D4B855C8585
:10C41000B701C8010F94726587FF04C0EA862F2C0C
:10C420000B871C872D853E854F855889B701C8012C
:10C430000F947B6E181624F4ED86FE860F87188BFA
:10C44000BFEFCB1ADB0AE9E0CE16D10481F6FF81FB
:10C45000F150FF838D819E8184969E838D83F1119F
:10C46000C4CF2D853E854F8558896A85722D8B8571
:10C470009C850F94546C20E030E040E05FE30F9423
:10C48000D765A50194010F94546C6B017C012DEBD1
:10C4900037E346E855EB0F947B6E87FD0AC02DEB22
:10C4A00037E346E855E3C701B6010F9472651816E5
:10C4B00034F580E00E94952C19E0A884B98409E045
:10C4C000D5016D917D918D919D915D014D01B4E0FE
:10C4D0008B1A9108A70196010F94536CF4016083A5
:10C4E000718382839383015059F711508885998510
:10C4F0008496998788871111E0CF0E94FC2F4528E8
:10C500004628472891F020E030E0A9016091AF066D
:10C510007091B0068091B1069091B2060F94726549
:10C52000882319F090E080E051DE8AE50E945823CC
:10C53000882359F00E940A2569837A838B839C8320
:10C5400060E0CE0101960E940D2D832D0E94952C56
:10C550000CC0311004C045284628472831F30E94FA
:10C56000F03682E397E00E942734332051F0809127
:10C57000AE06811106C00E94F53583E197E00E9466
:10C5800027340E94F03685E097E00E94273480919E
:10C59000AE060E94D7350E94F03688EF96E00E94E2
:10C5A0002734C090AA06D090AB06E090AC06F0907D
:10C5B000AD0620E030E0A901C701B6010F947B6E03
:10C5C00018160CF051C042E0C701B6010F94643E4A
:10C5D0000F949E52298D3A8D4B8D5C8D60914E0B40
:10C5E00070914F0B8091500B9091510B0F9472658D
:10C5F00081111FC02D893E894F89588D6091520B42
:10C600007091530B8091540B9091550B0F94726560
:10C6100081110FC02091560B3091570B4091580B50
:10C620005091590B69897A898B899C890F9472651D
:10C6300081110F94E0056C960FB6F894DEBF0FBE23
:10C64000CDBFDF91CF911F910F91FF90EF90DF90C1
:10C65000CF90BF90AF909F908F907F906F905F90A2
:10C660004F903F902F90089583EF96E00E942734DB
:10C67000B1CF2F923F924F925F926F927F928F92A3
:10C680009F92AF92BF92CF92DF92EF92FF920F9361
:10C690001F93CF93DF93CDB7DEB7CF54D1090FB639
:10C6A000F894DEBF0FBECDBF2E968FAF2E97209190
:10C6B000FB0A2D962FAF2D9721E02093FB0A809146
:10C6C000B4048D3409F47DC6843511F40C941F79BB
:10C6D000873409F0B3C18091B2049091B3048C31D6
:10C6E000910509F405C208F09BC18430910508F05A
:10C6F00052C120918C0A8230910508F4B0C12330D8
:10C7000008F4B3C111E0029709F010E00E94CD26B1
:10C7100019821A821B821C821D821E821F82188629
:10C7200082E50E94A623882309F4B5C10E940A2548
:10C730006B017C0120E030E0A9010F947265882331
:10C7400009F408C140904E0B50904F0B6090500B75
:10C750007090510B8091520B9091530BA091540B00
:10C76000B091550B27968CAF9DAFAEAFBFAF27975B
:10C7700080907C0690907D06A0907E06B0907F060B
:10C780008091800690918106A0918206B0918306E7
:10C790002B968CAF9DAFAEAFBFAF2B97A501940189
:10C7A000C301B2010F947265811111C02B962CAD9B
:10C7B0003DAD4EAD5FAD2B9727966CAD7DAD8EAD8B
:10C7C0009FAD27970F947265882309F4C3C0A30116
:10C7D0009201C501B4010F94536C20E030E040E0B9
:10C7E0005FE30F94D76523966CAF7DAF8EAF9FAF9D
:10C7F000239727962CAD3DAD4EAD5FAD27972B9679
:10C800006CAD7DAD8EAD9FAD2B970F94536C20E03A
:10C8100030E040E05FE30F94D7652B013C0120E05E
:10C8200030E0A901C701B6010F947265881F8827FF
:10C83000881F181709F426C180E090E0A0E8BFEB3C
:10C8400027968CAF9DAFAEAFBFAF279723962CAD89
:10C850003DAD4EAD5FAD2397CA01B9010F94D765C9
:10C860004B015C01A3019201C301B2010F94D76592
:10C870009B01AC01C501B4010F94546C0F94C16EBF
:10C880004B015C01AC019B01C701B6010F94536CD5
:10C890002B966CAF7DAF8EAF9FAF2B97A501940108
:10C8A000C701B6010F94546C9B01AC012B966CAD83
:10C8B0007DAD8EAD9FAD2B970F94D7656B017C013D
:10C8C00020E030E0A9010F947B6E87FDE0C0C70136
:10C8D000B6010F94C16E6B017C01C301B201905887
:10C8E000A50194010F94306D27962CAD3DAD4EAD52
:10C8F0005FAD27970F94D765A70196010F94D76571
:10C9000023962CAD3DAD4EAD5FAD23970F94546C87
:10C9100069837A838B839C83A501940123966CADF4
:10C920007DAD8EAD9FAD23970F94306D27962CADC6
:10C930003DAD4EAD5FAD27970F94D765A70196012A
:10C940000F94D765A30192010F94546C6D837E837D
:10C950008F83988760E080E50E94FF25082F853649
:10C9600030F00E94F53583E09CE00E942734202FB0
:10C97000412FBE016F5F7F4F8CE796E00E94785099
:10C980000F94D04D6093DD087093DE088093DF082C
:10C990009093E0086AC08531910509F466C08B3137
:10C9A000910509F48CC0049709F048C080E50E9405
:10C9B000A623C12CD12C7601882321F00E94FA24D1
:10C9C0006B017C0183E50E94A623882361F00E940D
:10C9D0000A2520E030E04AE754E40F94D7650F942D
:10C9E0009D6D6B017C010E94BFF280913C10811112
:10C9F00005C060E089E19CE00E9478960F94D04DDC
:10CA0000C60ED71EE81EF91E0F94D04D6C197D0975
:10CA10008E099F0997FF29C080E00E943B48F4CF10
:10CA20008A32910509F448C360F48E31910509F406
:10CA3000BFC008F460C0839709F4A6C10F9469547D
:10CA400014C08B35910509F413C48C35910509F494
:10CA500013C48A35910591F71092E31806C023306C
:10CA600020F00E94CD260F9470272E962FAD2E9782
:10CA7000211102C00F9477552D963FAD2D9730931D
:10CA8000FB0AA9C580E090E0A0E8BFE3D9CEC12CA5
:10CA9000D12C760122CF89E40E94A623882331F08D
:10CAA0000E940A2569837A838B839C838AE40E948F
:10CAB000A623882309F44ECF0E940A2547CF87E09A
:10CAC0000F947E228111D1CF8CE0EEE7F2E0DE01FF
:10CAD000119601900D928A95E1F770E060E080E593
:10CAE0000E94B125BE016F5F7F4F0F94A910BDCF8B
:10CAF0000E94FB38BACF14E00F94D04D6093DD084C
:10CB00007093DE088093DF089093E0088091AE0672
:10CB100081112CC08091AB049091AC04A091AD0424
:10CB2000B091AE0495FF04C082E29CE00E9482793D
:10CB300087E00F947E2281111FC00E94237E8823EC
:10CB4000D9F0115001F130E020E04BEC58E164E6FF
:10CB50007CE085E00E94A43561E088E29CE00E94D0
:10CB60006B3585E39CE00E948279C6CF60E08FE45C
:10CB70000E94ED25882371F20E94803582E09DE0BD
:10CB80000E94827972CF61E081E79CE00E946B3560
:10CB90008DE89CE00E94827961E086EB98E10E943A
:10CBA0006B3540E070E060E08EE79CE00E949747C4
:10CBB00088E0EEE4FBE0DE015C9601900D928A9540
:10CBC000E1F788E0EEE4FBE0DE01119601900D92C2
:10CBD0008A95E1F788E50E94A623082F882381F033
:10CBE0000E940A2520915E0B30915F0B4091600BF3
:10CBF0005091610B0F94536C69837A838B839C8370
:10CC000089E50E94A623182F882381F00E940A2517
:10CC10002091620B3091630B4091640B5091650B36
:10CC20000F94536C6D837E838F839887BE016B5FF7
:10CC30007F4FCE0101960F94AA43882309F49AC02E
:10CC4000002341F089819A81AB81BC818C8F9D8FBB
:10CC5000AE8FBF8F112341F08D819E81AF81B8854A
:10CC600088A399A3AAA3BBA380E00E94952C0F944C
:10CC70004A0361E085E40E94ED25B82E8091FD0A0B
:10CC8000882309F473C060E070E080EE90E400E077
:10CC900010E020E830EC0FAB18AF29AF3AAF20E03E
:10CCA00030E040EA50E40F94546C6BAF7CAF8DAF32
:10CCB0009EAFDE01DB967D018E01095C1F4F20E0F7
:10CCC0004B2DBE016B5F7F4FCE0101960F94A445A3
:10CCD0006B017C01AC019B010F940A6F81112EC086
:10CCE00020915E0B30915F0B4091600B5091610B76
:10CCF00069817A818B819C810F94546CAB01BC015A
:10CD000085E39DE00E94493B2091620B3091630BCB
:10CD10004091640B5091650B6D817E818F81988568
:10CD20000F94546CAB01BC0180E39DE00E94493B31
:10CD3000B701A6018BE29DE00E94ED3B0F94310309
:10CD40001FAA18AE19AE1AAE9E01295C3F4F46E5E8
:10CD50005BE0BE01605E7F4FCE014C960F9469038D
:10CD6000B1100E94A6240F94E0057FCE60E070E031
:10CD7000CB018DCF8AE19DE00E94D74160E08AE13E
:10CD80009DE00E94789671CE8E010F5F1F4F80E16B
:10CD9000F80111928A95E9F76EE183E50E94FF257B
:10CDA0008FAF8E51863130F48FAD6AE00F94F96BFE
:10CDB000923028F08BE89DE00E94273456CE0E94E6
:10CDC000BFF2F091AE062896FFAF289780E00E9450
:10CDD000952C8091010B8770873021F086E89DE0CB
:10CDE0000E94827925961FAF0EAF259766E9662EC1
:10CDF00062E0762ED12CC12C212C312C70E8472EEC
:10CE000070EC572E8091FD0A882309F46AC060E017
:10CE100070E080EE90E42C8E3D8E4E8E5F8E20E092
:10CE200030E040EA50E40F94546C6FAB78AF89AFB8
:10CE30009AAF9E01295C3F4F79018E01045E1F4F1E
:10CE400020E043E0B3016C5F7F4FC3010F94A44522
:10CE50004B015C01AC019B010F940A6FB6016F5F3F
:10CE60007F4F882309F441C081E79DE00E945A4129
:10CE70008EE69DE00E942734F601EE0FFF1FEB5E69
:10CE8000F54D859194910E94273489E20E942034C7
:10CE9000860153E0000F111F5A95E1F70A561D4F06
:10CEA000D8014D915D916D917C9188EB9EE00E943F
:10CEB000493BF80144815581668177818CE494E493
:10CEC0000E94ED3B80E69DE00E94273428968FADBE
:10CED00028970E94952C80E00E94A12B0F94DC449F
:10CEE000C4CD60E070E0CB0196CF2596AEADBFAD6E
:10CEF00025978D929D92AD92BD922596BFAFAEAF14
:10CF000025976B01B8E06B0E711C6430710509F058
:10CF100079CF8CE0EAE8F2E0DE015C9601900D92B8
:10CF20008A95E1F72FAD2E51330BC9016AE070E00D
:10CF30000F94266C1E0135E0230E311C10E000E03A
:10CF4000660F771F660F771F6C0F7D1FCB014C9606
:10CF500060969FAF8EAF6097BFACB0949B2D9170E1
:10CF60002C969FAF2C97D1012D913D914D915D91C4
:10CF70001D0169817A818B819C810F94536C6B01B7
:10CF80007C0120E030E0A9010F947B6E87FF8DC00B
:10CF9000C701B60190582FE632E143E85AE30F94F7
:10CFA000726587FD85C06096EEADFFAD609720810C
:10CFB000318142815381C701B6010F94306D6B01FD
:10CFC0007C01C701B6010F94036F0F94986D2B017C
:10CFD000072E000C880B990B0F9478659B01AC0110
:10CFE000C701B6010F94536C20E030E040E752E4F3
:10CFF0000F94D7650F94036F0F94986D4B0125968E
:10D000007FAF6EAF25978AE59DE00E942734F80137
:10D01000E95EF54D859194910E942734F1E0FFAFD0
:10D0200020E030E0A901C701B6010F947B6E18160D
:10D030000CF01FAE2C962FAD2C973FAD6AEE73E02F
:10D04000231302C06BEE73E088E59DE015D8B201B2
:10D0500057FE04C0662777276419750983E59DE0AC
:10D060000E945A418CE49DE00E94273425968EADA3
:10D070009FAD2597892B79F0B40197FE04C06627F0
:10D0800077276819790986E49DE00E945A418DE36B
:10D090009DE00E9427348AE00E9420340E5F1F4FDB
:10D0A0000630110509F05FCF11CFC701B60173CF6C
:10D0B000C12CD12C760185CF80918C0A833008F465
:10D0C000D4CC89E40E94A623082FF12C882319F0E0
:10D0D0000E94BD25F82E8AE40E94A623E82E88230C
:10D0E00089F00E94BD25182F002329F098E09F1594
:10D0F00020F0EE2051F0193040F08FEB9DE00E94BF
:10D100002734B3CC10E00111F1CF80E1EEE4FBE075
:10D11000ACE7B6E001900D928A95E1F7002311F19A
:10D120006F2D70E090E080E00F9478652091AF065D
:10D130003091B0064091B1065091B2060F94D76578
:10D140002091A2063091A3064091A4065091A50615
:10D150000F94546C60937C0670937D0680937E06DA
:10D1600090937F06EE2011F1612F70E090E080E057
:10D170000F9478652091B3063091B4064091B506BE
:10D180005091B6060F94D7652091A6063091A70658
:10D190004091A8065091A9060F94546C60938006A4
:10D1A00070938106809382069093830660E080E509
:10D1B0000E94ED258823C1F10023D1F0E091781180
:10D1C000F0917911208131814281538160917C06F7
:10D1D00070917D0680917E0690917F060F94536C2E
:10D1E00060937C0670937D0680937E0690937F0605
:10D1F000EE20D1F0E0917811F09179112481358100
:10D2000046815781609180067091810680918206E7
:10D21000909183060F94536C6093800670938106FF
:10D22000809382069093830640E050E0BA0186E442
:10D230000E9438256B017C0120E030E0A9010F94A9
:10D240007B6E18168CF420E030E040E752E4C70112
:10D25000B6010F94306D69837A838B839C83CE01F2
:10D2600001960F94F32901CC60E070E0CB01F3CF7D
:10D270008FE08093E318F9CB8091B104882381F18A
:10D28000893009F0F2CB9AECA92E92E0B92E2EE467
:10D29000C22E2BE0D22EE12C00E010E0D5018D91C2
:10D2A0005D010E94A623F82E882361F0133011F04F
:10D2B000E82EF02E0E940A25F60160837183828396
:10D2C00093830F2D1F5FF4E0CF0ED11C143031F784
:10D2D000EE2009F464C00F947E050F94E005C5CBE1
:10D2E0008AECC82E82E0D82EF12CE12C00E010E070
:10D2F000D6018D916D010E94A623382E882309F452
:10D3000047C00E940A254B015C01133059F0F70118
:10D31000E25AF44F20813181428153810F94536C42
:10D320004B015C01F701E25BF44F208131814281C6
:10D330005381C501B4010F94536C2B013C012DEBBB
:10D3400037E346E855EB0F947B6E87FD0AC02DEB63
:10D3500037E346E855E3C301B2010F94726518162E
:10D36000BCF4133021F1F701E059F94F5F01A3013B
:10D37000920160817181828193810F94546CD501F7
:10D380006D937D938D939C931397812F0F94D80168
:10D390001F5FB4E0EB0EF11C143009F0A9CF00239D
:10D3A00009F49BCF8AE59BE00F94540096CF8092BE
:10D3B0005A0B90925B0BA0925C0BB0925D0B032D0D
:10D3C000E7CF8091B2049091B3048D37910509F4B1
:10D3D0003FC008F0C2C18E34910509F47CC608F044
:10D3E0008EC08A31910509F408C5A8F584319105EC
:10D3F00009F4AFC488F48131910509F461C430F4B3
:10D40000029708F01BCB0E94CA5F2FCB429709F00E
:10D4100015CB0E944D2529CB8731910509F4D6C43F
:10D4200080F48531910509F4CDC4469709F006CB07
:10D430008091F01882FF02C087FF17CB0E94B4E7EB
:10D4400014CB8831910509F4D4C4499709F0F6CA80
:10D450000E94B55D0ACB8032910509F45EC5A8F53E
:10D460008D31910509F442C570F48B31910509F4B1
:10D47000D7C44C9709F0E2CA8091AF049091B004F0
:10D480000F949654F2CA8E31910509F436C54F9720
:10D4900009F0D4CA0F94AC0A6C8F7D8F8E8F9F8F4A
:10D4A000BE016F5F7F4FCE014C960E944E29CE0188
:10D4B00001960F94B0520E94F036BE016F5F7F4F0D
:10D4C00088E39EE00F947754D0CA8B34910509F419
:10D4D000FAC550F48132910509F44AC5C09709F0A4
:10D4E000ADCA0E94BC3CC1CA8C34910509F4EFC599
:10D4F0008D34910509F0A2CA0E941931B6CA8D3641
:10D50000910509F4F1C508F089C08C35910509F43D
:10D51000ADC608F03FC08335910509F49FC678F485
:10D520008135910509F483C68235910509F086CAD3
:10D530008091E3188F7D80618093E31896CA8435CB
:10D54000910509F466CF8535910509F077CA83E521
:10D550000E945823882309F488CA0F94D04D609301
:10D56000DD087093DE088093DF089093E0080E9446
:10D570000A2520E030E04AE754E40F94D7650F9481
:10D580009D6D60938B0470938C0480938D049093B5
:10D590008E046BCA8A36910509F4ABC5B0F588369E
:10D5A000910509F49CC58936910509F047CA0E9486
:10D5B000F736182F87FD0AC085E49EE00E942734C5
:10D5C000812F0E94FCE88AE00E9420342D96EFAD66
:10D5D0002D97E093FB0AC15BDF4F0FB6F894DEBFD7
:10D5E0000FBECDBFDF91CF911F910F91FF90EF90B4
:10D5F000DF90CF90BF90AF909F908F907F906F9073
:10D600005F904F903F902F9008958B36910509F4CD
:10D61000A4C58C36910509F428CA10CA8337910530
:10D6200009F428C608F057C08037910509F41DCACF
:10D6300008F042C08E36910509F49AC58F369105DF
:10D6400009F0FCC983E50E94A623882321F00E94EB
:10D65000CD258093F70A0E94F03686E59EE00E9471
:10D6600027348091F70A882309F495C510E000E07B
:10D6700020E08091F70A90E0002E02C095958795F2
:10D680000A94E2F780FF12C0FF24F394F20E2223E3
:10D6900019F08CE20E942034F801EE0FFF1FE45BCA
:10D6A000F14F859194910E9427342F2D0F5F1F4FCA
:10D6B00005301105F1F6E7C38137910509F46EC510
:10D6C0008237910509F0BAC90F94CE428FE891E1F3
:10D6D0000E94F3EBCAC98737910509F4FBC570F5C1
:10D6E0008537910509F4CAC58637910509F0A6C9A1
:10D6F0000091AF041091B00494E0F12C40E09150FF
:10D7000009F4D5C5F8018081282F2B7F213409F039
:10D71000C7C52181213309F0CAC5813409F4D7C5B1
:10D72000853409F441E098012E5F3F4F89012F5F56
:10D730003F4FF80180818032C9F3E1CF88379105EE
:10D7400009F4CCC58937910509F078C910923A0AD5
:10D750001092390A0F94350788C98239E1E09E0793
:10D7600011F40C94657608F024C1833D910509F409
:10D77000AEC708F05FC0883C910509F430C6C8F414
:10D780008139910509F4B3C540F48C38910509F04D
:10D7900055C980E00E94834E68C98B39910509F410
:10D7A0001FC58E3B910509F049C981E00E94834E57
:10D7B0005CC98C3C910509F4AEC6D0F4893C910556
:10D7C00009F44BC68B3C910509F038C98091AB0434
:10D7D00084FD7EC68091AD04887809F079C6809179
:10D7E000AE04837009F074C681E00E948D3B3DC990
:10D7F0008D3C910509F4E4C68E3C910509F01EC9E3
:10D800008091AB049091AC04A091AD04B091AE04B2
:10D810006AECC62E62E0D62E7DE3E72E7AE0F72E84
:10D8200010E0892B8A2B8B2B09F037C781E00E94EF
:10D83000F03B1BC98D3221E0920711F40C947575F1
:10D8400008F06CC08831A1E09A0711F40C94A2741E
:10D8500008F045C08C3D910511F40C9442748D3D47
:10D86000910509F0EBC80E94F736082F87FDFDC827
:10D8700083E50E94A623002E000C110B7801EE0C0C
:10D88000FF1C882311F40C9488740E94BD25F701B5
:10D89000E55DFD4F91838083000F111F000F111F65
:10D8A000F801EA59FD4F7F01BC01990F880B990BD4
:10D8B0000F9478652AE037ED43E25CE30F94D76577
:10D8C0000457194FD8012D913D914D915C910F94C2
:10D8D000D765F7016083718382839383C6C88232E0
:10D8E000E1E09E0711F40C94E7748C32914009F04A
:10D8F000A5C864E071E083E50E94B1258C0168EE63
:10D9000073E080E50E94B1258938F3E19F0710F0AC
:10D9100088E893E1B8010F94612AA7C8803321E019
:10D92000920711F40C94BF7568F48E32A1E09A0747
:10D9300011F40C9409768F32914009F07FC80E944F
:10D94000384293C88039E1E09E0711F40C944F7679
:10D950008139914009F072C8C090AB04D090AC04FA
:10D96000E090AD04F090AE0417E0F694E794D794FD
:10D97000C7941A95D1F721E0C222DD24EE24FF24BA
:10D9800083E50E945823CD28CE28CF2811F00C948F
:10D99000537681110C94557660E082E50E94ED2566
:10D9A0009091FC0A911199CC682F81E00F94FA08AC
:10D9B00094CC883F31E0930711F40C94567708F02B
:10D9C000FEC08C3AB1E09B0711F40C94DA7608F0B3
:10D9D000CBC08D39F1E09F0711F40C94037908F066
:10D9E00048C08A3931E0930709F43FC88C39914027
:10D9F00009F024C88091AB04887811F00C948576E6
:10DA00008091AD04867011F00C9485760E94F036FA
:10DA10008FE99FE00E94273480914F02882311F400
:10DA20000C947D768AE79FE00E94273440914B0258
:10DA300050914C0260914D0270914E0282E99FE03C
:10DA40000E94493B8FE89FE00E9427348DE79FE0CA
:10DA50000E94273480919004882311F40C948176DD
:10DA60008AE79FE00E9427348AE00E9420340C94C9
:10DA70003565843AB1E09B0711F40C94C776853A7A
:10DA8000914011F00C941E656FEF7FEF89E40E94C6
:10DA9000C025082F6FEF7FEF8AE40E94C025182F62
:10DAA0008AE50E94A623D12C811108C081E50E943D
:10DAB000A623D82E882311F40C944C79C02E81E033
:10DAC000800F8A3010F00C94D276912E81E0810F75
:10DAD0008A3010F00C94D2760E940A252B013C016A
:10DAE000F02E07FDF12C07FF02C0A8E0CA2E812E00
:10DAF00017FD812C17FF02C0F8E09F2EE9E03E2EB3
:10DB0000CF1410F40C94CE76E82C3F9C50011124D5
:10DB10009E1410F40C94CB760E2D10E020E030E033
:10DB2000A901DD2069F0F501E00FF11FEE0FFF1FE5
:10DB3000EE0FFF1FEB53F94F20813181428153815A
:10DB40000A0D1B1D000F111F000F111F0B53194F42
:10DB5000C301B2010F94546CD8016D937D938D93E2
:10DB60009C931397E394D4CF853FF1E09F0711F482
:10DB70000C944E7778F4863E31E0930711F40C94C0
:10DB8000DE76843F914011F00C941E650E9416EEE3
:10DB90000C943565863FB1E09B0711F40C945277E5
:10DBA000873F914011F00C941E6561E083E50E946F
:10DBB000ED2591E089270E94FBEC0C9435658335B7
:10DBC000F3E09F0711F40C940D7828F58B3532E0C3
:10DBD000930711F40C947D7778F48C30B2E09B07B6
:10DBE00011F40C9467778835924011F00C941E65FF
:10DBF0000E940F7D0C9435658D3BF2E09F0711F478
:10DC00000C9409788E3B924011F00C941E650E9492
:10DC1000EC5A0C943565873E33E0930711F40C946D
:10DC2000F378C8F48C36B3E09B0711F40C94356597
:10DC3000803A934011F00C941E652091AF0430910E
:10DC4000B0049091F01892609093F018C9010F946D
:10DC500096540C943565883EF3E09F0711F40C94BC
:10DC60001579893E934011F00C941E650E94BFF215
:10DC70008091F018877F8B7F8093F0188091E61851
:10DC800081110C9418790E94AB2B0F946E550F9450
:10DC9000AC0A6D3371058105910520F080E690E1B5
:10DCA0000E9482798CE590E10E94827988E490E17B
:10DCB0000E94273484E490E10E9482790C943565B7
:10DCC0000E944723882399F185E40E9458238823E2
:10DCD00061F080917F0490918004892B21F00E9453
:10DCE000BD25811102C00E94A6EC0AECE02E02E0E4
:10DCF000F02E10E0D7012D917D0121548091AB04CD
:10DD00009091AC04A091AD04B091AE0404C0B6955E
:10DD1000A795979587952A95D2F780FF03C0812F05
:10DD20000E94E0EC1F5F133029F70C94356560E02A
:10DD300088ED9DE00E94789680E00E94E0EC81E012
:10DD40000E94E0EC82E00E94E0EC0E94A6EC0C94C1
:10DD500035658091F01884FF2DC080EF9DE00E9412
:10DD6000273460E08CE40E94ED25182F8091F01894
:10DD700084FF1AC081E199E10E94F2E88BE1E1E1C0
:10DD8000F9E1DE01119601900D928A95E1F730E0FC
:10DD900020E0412F70E060E0CE0101960F945F1CFF
:10DDA000CE0101960E94D92B81EE9DE00E9427347E
:10DDB0000C9435650E94F03681E09EE00E94273485
:10DDC0000C9435650E94D6E70C9435658091AF04BC
:10DDD0009091B004FC012191222331F02032D9F737
:10DDE000DF0111971C92F7CF60E00F94601B0C9439
:10DDF00035650E94BA590C9435658091F01884FD00
:10DE000002C00C94356583E50E94A623882311F493
:10DE10000C9435650E94A1250E9498240C943565C8
:10DE20008091AB049091AC04A091AD04B091AE048C
:10DE300012E0B695A795979587951A95D1F780FF2B
:10DE40002CC085E19EE00E9427348091581A8823D7
:10DE5000F9F0BE016F5F7F4F85E59AE10E9442E8CD
:10DE6000CE0101960F94A452CE0101960F943B541B
:10DE70008091F60F882339F080E20E94203486EFEB
:10DE80009FE00F94A4528AE00E9420340C943565E0
:10DE90008BE09EE00E942734F6CF83E50E94A62304
:10DEA000882301F10E94CD25182F8C3308F08CE3D4
:10DEB000809385040F94D04D6B017C01212F30E0BD
:10DEC000A8EEB3E00F94EA6BC60ED71EE81EF91E4B
:10DED000C0928104D0928204E0928304F092840480
:10DEE0000C9435650F9434530C9435658091F0187B
:10DEF0008E7F8093F0180C9435658091F01884FD26
:10DF000002C00C9435650F9445438091AF04909105
:10DF1000B0040F940A550C9435658091F01882FF77
:10DF200003C087FF0E94BFF28091F01884FD02C0F9
:10DF30000C94356560E080E50E94ED25182F682F70
:10DF40008091AF049091B0040F94601B83E50E9410
:10DF5000A623882321F00E94A1250E9498240E94D4
:10DF600032E011110C9435650E9407310C9435652F
:10DF70000091AF041091B004D12CC12C01151105F2
:10DF8000C1F0F80101900020E9F731979F01201BB3
:10DF9000310B6901D801CD01801B910B82179307CA
:10DFA00044F48D918F32B9F7CD010197FC011082B5
:10DFB000F2CF8BE1E1E1F9E1DE015C9601900D9297
:10DFC0008A95E1F7F12CE12CEC14FD040CF05DC016
:10DFD000F801EE0DFF1D8081811103C0FFEFEF1AE4
:10DFE000FF0A5801AE0CBF1CD5018C91882309F49F
:10DFF0004CC0BFEFEB1AFB0AF801EE0DFF1D7F01CD
:10E00000E01AF10A81918111FACFCE014C960E945B
:10E01000F2E88BE1FE017C96DE01119601900D92F3
:10E020008A95E1F7B501CE0101960E94CCE0CE01C0
:10E0300001960E94D92B8FE20E9420348091F60F26
:10E04000882361F186EF9FE00F94A4528091F0182D
:10E0500085FF1BC019821C8221E0A501BE01645E00
:10E060007F4FCE0101960F94BF1881111AC08AE02C
:10E070000E9420340E94F036B50184E29EE00E94A6
:10E080003C60CE0101960E94D92B8AE00E94203488
:10E09000CE014C960E94D92B0C94356589EE9FE0F9
:10E0A000D3CFCE014C960E949DE78BE1FE013196C5
:10E0B000DE015C9601900D928A95E1F7CE01019602
:10E0C0000E94D92B81CF0E9407310C9435650F94A3
:10E0D000A10B0C9435650E9446600C94356580E078
:10E0E0000E941E370C94356581E00E941E370C9407
:10E0F000356560E080E50E94FF2581110C9435654F
:10E100008091AB046091E50A062F10E080FD02C00B
:10E110000FEF10E089E40E94A623882311F40C94E9
:10E1200040790E94CD2590E08330910514F082E083
:10E1300090E026E0289FF001299FF00D1124E3577D
:10E14000F54F048115810F3F110519F010F00FEF05
:10E1500010E00093E50A0C94356560E080E50E94CC
:10E16000FF2581110C9435651092E50A0C943565F4
:10E170008EE40E94A623882311F40C9435650E9436
:10E18000A1256093EC0B7093ED0B8093EE0B9093B5
:10E19000EF0B0C94356588E49EE07CCE83E50E940D
:10E1A000A623882369F00E94CD258D3320F4809327
:10E1B00006020C9435658CE3809306020C94356559
:10E1C0000E94F036109106028DE59EE00E942734F1
:10E1D000812F0E94F6E88AE00E9420340C94356575
:10E1E00083E50E94A623882311F40C9435650E94D0
:10E1F000CD25182F8C3308F08CE380938A040F947C
:10E20000D04D6B017C01212F30E0A8EEB3E00F94DC
:10E21000EA6BC60ED71EE81EF91EC0928604D09285
:10E220008704E0928804F09289040C9435650E947A
:10E23000D0F21092E50A0E9443EB0E94193168EE79
:10E2400073E080E090E00E949C3060E084E69EE015
:10E250000E9478960E94F5230C9435658091E3180E
:10E260008F7E80628093E3180C9435650E942C3871
:10E270000C9435650E9457340C9435658091AF0439
:10E280009091B004009741F0DC012C91222321F001
:10E290000F94B0520C9435650F94E6520C9435658A
:10E2A000803529F4818180538A3008F43CCA4111B9
:10E2B0000E94F036FF2021F084E79EE00E94273480
:10E2C000C8010F94A4520F949E520C943565FF24FC
:10E2D000F39429CA0F94EA060C94356581E0809383
:10E2E0003A0A8093390A0F9435070C94356570E02B
:10E2F00060E083E50E94C025833040F00E94F53540
:10E3000087E79EE00E9427340C9435658C01112725
:10E3100088E40E94A6238823E9F00E94BD2520916D
:10E32000090230910A028217930754F00E94BD251A
:10E3300024E031E0853091401CF40E94BD259C0111
:10E3400086E0809FF001819FF00D1124E357F54F87
:10E350003183208382E40E94A6238823A9F00E94AF
:10E36000BD25059784F10E94BD258F36910574F572
:10E370000E94BD2526E0209FF001219FF00D112471
:10E38000E357F54F9383828386E40E94A623882374
:10E3900011F40C9435650E94BD2597FD1AC00E94AA
:10E3A000BD258F3F910509F0BCF40E94BD2526E0F4
:10E3B000209FF001219FF00D1124E357F54F958325
:10E3C00084830C94356585E090E0D4CF8EE690E0B0
:10E3D000D1CF90E080E0EBCF8FEF90E0E8CF80915D
:10E3E000AB0483FD09C08091AD048C7029F481E0F9
:10E3F0000E94913C0C9435650E94F736182F87FFD8
:10E4000002C00C9435650091C30684E40E94A623E3
:10E41000F82E8823B1F00E940A254B015C0120E010
:10E4200030E0A9010F9472658823A9F024E012025C
:10E43000F0011124E154F94F80829182A282B382CB
:10E440000F2D602F83E50E94ED258093C3060E9467
:10E45000C2D70C94356580E0F8CF8091AB0484FD81
:10E460000DC08091AD04887849F48091AE0483702A
:10E4700029F481E00E94B53B0C9435650E94F73683
:10E4800087FF02C00C9435650AEC12E0F2E0EF2E33
:10E49000FBE0FF2EAEECCA2EA2E0DA2ED8018D9161
:10E4A0008D010E94A623882359F00E940A250F940B
:10E4B0009D6DF70160837183828393830E944EF286
:10E4C000F4E0EF0EF11CC016D10641F70C9435654F
:10E4D0000E94F73687FF02C00C943565EAECEE2EF9
:10E4E000E2E0FE2E10E000E0D7018D917D010E9458
:10E4F000A623882349F00E940A25F801EE5FF44F15
:10E5000064A375A386A397A30C5F1F4F0031110569
:10E5100059F70C9435658091AC0487FD09C0809152
:10E52000AD048E7029F481E00E94723C0C94356534
:10E5300083E50E94A623882391F00E940A25609318
:10E54000360B7093370B8093380B9093390B609395
:10E550003E0B70933F0B8093400B9093410B80E5F3
:10E560000E94A623882351F00E940A256093360B4F
:10E570007093370B8093380B9093390B82E50E9490
:10E58000A623882351F00E940A2560933A0B7093CA
:10E590003B0B80933C0B90933D0B84E50E94A6239C
:10E5A000882311F40C9435650E940A2560933E0B74
:10E5B00070933F0B8093400B9093410B0C94356507
:10E5C0008091AB049091AC04A091AD04B091AE04E5
:10E5D000892B8A2B8B2B29F481E00E943E3C0C94E2
:10E5E000356582E40E94A623882351F00E94FA2414
:10E5F0006093120B7093130B8093140B9093150B75
:10E6000083E50E94A623882351F00E940A25609387
:10E61000420B7093430B8093440B9093450B84E51E
:10E620000E94A623882351F00E940A256093460B7E
:10E630007093470B8093480B9093490B8AE40E9498
:10E64000A623882311F40C9435650E940A256B01DA
:10E650007C012AE037ED43E25CE30F947B6E87FD9B
:10E6600014C02AE939E949E95EE3C701B6010F940C
:10E670007265181654F0C092C90AD092CA0AE09284
:10E68000CB0AF092CC0A0C9435650E94F53589E9E5
:10E690009EE00E9427340C943565F60181916F014C
:10E6A0000E94A623882359F00E940A25D7016D9362
:10E6B0007D938D939C931397812F0F94D8011F5FA7
:10E6C000B4E0EB0EF11C133041F70C946D6983E557
:10E6D0000E945823882331F00E94DE258093310266
:10E6E0000C9435656AED7EE081E00F943343109120
:10E6F0003102105D81ED9EE00E942734812F0E943F
:10E7000020348DEC9EE00E942734809131020E94DB
:10E71000D73540905E0B50905F0B6090600B70900F
:10E72000610B2091330230913402409135025091B7
:10E730003602C301B2010F94546C23966CAF7DAFC7
:10E740008EAF9FAF23978090620B9090630BA09049
:10E75000640BB090650B20913702309138024091E4
:10E76000390250913A02C501B4010F94546C2796B6
:10E770006CAF7DAF8EAF9FAF2797C090660BD090E8
:10E78000670BE090680BF090690B20913B02309191
:10E790003C0240913D0250913E02C701B6010F94E8
:10E7A000546C2B966CAF7DAF8EAF9FAF2B972091A3
:10E7B0003F02309140024091410250914202C30118
:10E7C000B2010F94546C2B013C0120914302309113
:10E7D00044024091450250914602C501B4010F9494
:10E7E000546C4B015C0120914702309148024091EA
:10E7F000490250914A02C701B6010F94546C6B0153
:10E800007C0185EC9EE00E94273423964CAD5DADE3
:10E810006EAD7FAD239788EB9EE00E94493B279623
:10E820004CAD5DAD6EAD7FAD27978CE494E40E9456
:10E83000493B2B964CAD5DAD6EAD7FAD2B9789E41A
:10E8400094E40E94493B83EC9EE00E9427348BEBCA
:10E850009EE00E942734B301A20188EB9EE00E9453
:10E86000493BB501A4018CE494E40E94493BB70103
:10E87000A60189E494E40E94493B8AE00E94203486
:10E880000C9435658091AB049091AC04A091AD04DB
:10E89000B091AE0460912502709126020097A10507
:10E8A000B10551F48BEE9EE00E945A4188EE9EE045
:10E8B0000E9427340C9435658C019D0151E13695F9
:10E8C0002795179507955A95D1F700FF08C0209115
:10E8D0000702309108023093260220932502B69554
:10E8E000A7959795879580FF04C070930802609361
:10E8F000070283E50E94A623882311F40C94356552
:10E900000E94BD2590932602809325020C943565C4
:10E910000E94F03685E40E94203480E3800F0E943C
:10E920002034F701E55DFD4F608171818FEE9EE03F
:10E930000E945A4185E20E9420348AE00E942034DD
:10E940000C94356580E50E94A623882311F40C946D
:10E9500035650E94BD258C01892B61F583E50E94F8
:10E96000A623882389F00E94BD2597FD07C0BC011E
:10E9700089E691E10E948D310C94356589E691E13B
:10E980000E941E310C9435650E94F03670E060E004
:10E990008AEF9EE00E945A4189E691E10E94F823A5
:10E9A000BC0187EF9EE00E945A418AE00E94203419
:10E9B0000C9435650E94F535B80181E19FE00E9415
:10E9C0005A4182E09FE00E9427340C9435658AE525
:10E9D0000E94A623882309F45EC00E940A2520E035
:10E9E00030E040E050EC0F94726587FD71C00E94EA
:10E9F0000A2520E030E040E050E40F947B6EC12C0B
:10EA0000D12CE12C00E4F02E181624F00E940A25E7
:10EA10006B017C0180901E0B90901F0BA090200B2F
:10EA2000B090210B84E00F94F80181110BC0A50177
:10EA30009401C701B6010F94D7650F94986DCB016F
:10EA40000E947D3061E080E50E94ED25882341F140
:10EA5000A7019601609174117091751180917611E2
:10EA6000909177110F94546C609374117093751199
:10EA700080937611909377110E94F0364091741133
:10EA800050917511609176117091771187E29FE036
:10EA90000E94ED3B05C083E50E94A62381119DCF16
:10EAA0008091AD0487FD1AC08091AE048370B1F4EB
:10EAB0000E94F03640917411509175116091761159
:10EAC0007091771188E19FE00E94ED3B0C943565D1
:10EAD000C12CD12CE12C80ECF82E9CCF82E50E9439
:10EAE00058238111E5CF0C9435658091AB0483FDEB
:10EAF00009C08091AC04817829F481E00E94593BDF
:10EB00000C94356580E50E94A623882351F00E946D
:10EB10000A2560931211709313118093141190932E
:10EB2000151189E40E94A623882381F00E940A25FA
:10EB300021E732EB47E25EE30F94D765609316114D
:10EB400070931711809318119093191184E40E9407
:10EB5000A623882381F00E940A2521E732EB47E2B1
:10EB60005EE30F94306D60931A1170931B118093C4
:10EB70001C1190931D110E94972B0C943565809168
:10EB8000AB0483FD09C08091AC04817829F481E055
:10EB90000E940F3C0C94356580E50E94A6238823D3
:10EBA00051F00E940A256093E6107093E71080935D
:10EBB000E8109093E91089E40E94A623882381F04D
:10EBC0000E940A2521E732EB47E25EE30F94D76506
:10EBD0006093EA107093EB108093EC109093ED101B
:10EBE00084E40E94A623882311F40C9435650E94C6
:10EBF0000A2521E732EB47E25EE30F94306D609324
:10EC0000EE107093EF108093F0109093F1100C942D
:10EC1000356583E50E945823182F882369F00E94E8
:10EC2000BD259C0190930A028093090291E0232B59
:10EC300009F090E090938F0480E50E945823882388
:10EC400061F02091090230910A02232B11F00E94F9
:10EC5000DE2580938F040C94356511110C94356575
:10EC60000E94F03682E59FE00E94273480918F0455
:10EC7000882391F08AE39FE00E9427346091090283
:10EC800070910A0281E49FE00E945A418DE39FE067
:10EC90000E9427340C94356586E39FE0EDCF0E94F7
:10ECA000BFF20C943565882321F00E94DE25809305
:10ECB000FD0A0E94F03685E69FE00E94273480918D
:10ECC000FD0A0E94D7350C94356560E082E50E940C
:10ECD000ED250E94A12B80E090E0A0EAB0E48983BA
:10ECE0009A83AB83BC8340E061E0CE0101960F9430
:10ECF00049040F94E0050C94356586E79FE00C9479
:10ED0000146D86E79FE00C94326D88E40E945823CE
:10ED1000882321F00E94DE2580939004C090AB04EC
:10ED2000D090AC04E090AD04F090AE04B1E1F69464
:10ED3000E794D794C794BA95D1F731E0C322DD2484
:10ED4000EE24FF2483E50E945823182FCD28CE28D7
:10ED5000CF2811F4882341F00E94E223112321F0EF
:10ED60000E94DE2580934F0284E40E94A62388231C
:10ED700011F40C9435650E940A2560934B02709340
:10ED80004C0280934D0290934E020C9435650E9484
:10ED900061610C943565F3940C94806D0E94FC2F96
:10EDA0000C9435650E94F53580ED9FE00E94273474
:10EDB0000C9435650E94F8350C94356584E50E9405
:10EDC00058238823A1F01092BA041092BB04109229
:10EDD000BC041092BD041092BE048FEF0E94B223B7
:10EDE00061E070E084E50E94C0258093BE0483E565
:10EDF0000E94A623882321F00E94BD250E94B223F1
:10EE000083E40E945823882331F080911F028032CE
:10EE100010F40E94692C80E50E94A623882331F01B
:10EE20000E94BD25803210F40E94692C85E50E9465
:10EE3000A623882311F40C9435650E94BD258032E9
:10EE400010F00C94356541E050E0082E02C0440FEC
:10EE5000551F0A94E2F740955095052E000C660B5D
:10EE6000770B0091BA041091BB042091BC0430913F
:10EE7000BD0440235123622373234093BA0450936B
:10EE8000BB046093BC047093BD0490911F0289136E
:10EE90000C9435651092F60A0C9435650F94652232
:10EEA0000C9435650F9444070C943565209309083C
:10EEB0000F945A221092090881110C9435650E9412
:10EEC000F03689EE9FE00E9427340C94356510914E
:10EED000F01812FF0AC017FD08C00E94E33080FB43
:10EEE00017F91093F0180C94356514FD02C00C94BA
:10EEF00035650F9445430C9435658091AC0483FDD2
:10EF000009C08091AD04887129F481E00E94084213
:10EF10000C9435650E94F736082F87FF02C00C94C9
:10EF2000356585E50E94A623882351F10E940A25B4
:10EF30004B015C01E02E002E000CFF0820E030E0C9
:10EF4000A9010F947B6E87FF04C0B7FAB094B7F89D
:10EF5000B09420E030E849ED53E4C501B4010F94CA
:10EF60007B6E970143E0220F331F4A95E1F7295446
:10EF7000394F1816CCF1F90180829182A282B382B6
:10EF80008CE40E94A623882311F40C9435650E941A
:10EF90000A256B017C01002E000C110B20E030E0F3
:10EFA000A9010F947B6E87FF04C0F7FAF094F7F87D
:10EFB000F09420E030E849ED53E4C701B6010F9426
:10EFC0007B6E980193E0220F331F9A95E1F7295445
:10EFD000394F18169CF0D9011496CD92DD92ED921E
:10EFE000FC9217970C94356580E090E8A9EDB3E4A6
:10EFF000F90180839183A283B383C2CF80E090E83C
:10F00000A9EDB3E4F90184839583A683B7830C94B7
:10F0100035650E9458570C9435658091AD0487FD85
:10F0200009C08091AE04837029F481E00E94DC4124
:10F030000C94356520906C1130906D1140906E11DC
:10F0400050906F11609070117090711180907211DA
:10F05000F0917311FFAFC0907411D0907511E090D2
:10F060007611F090771188E50E94A623182F882347
:10F0700009F48AC00E940A25962EA72EB82E092FC1
:10F0800020E030E04BE953EC0F947B6E87FD0DC020
:10F0900020E030E04BE953E4692D7A2D8B2D902F41
:10F0A0000F94726518160CF071C066E371E081E38D
:10F0B00090E10E945A4166E371E08CE290E10E9487
:10F0C0005A4189E290E10E94273410E089E50E94CC
:10F0D000A623882361F10E940A25962EA72EB82E1A
:10F0E000092F20E030E04BE953EC0F947B6E87FD55
:10F0F0000DC020E030E04BE953E4692D7A2D8B2DD3
:10F10000902F0F94726518160CF045C066E371E0FD
:10F1100086E190E10E945A4166E371E081E190E16D
:10F120000E945A418EE090E10E94273410E08AE567
:10F130000E94A6238823A1F10E940A256B017C016D
:10F1400020E030E040E251EC0F947B6E87FD0AC076
:10F1500020E030E040E251E4C701B6010F9472654F
:10F160001816F4F466EF7FEF8CEF9FE00E945A418F
:10F170006AE070E087EF9FE00E945A4184EF9FE0D1
:10F180000E9427340C94356511E0A0CF292C3A2C2D
:10F190004B2C502E9BCF692C7A2C8B2C0FAFC7CFCA
:10F1A000112311F40C943565C101D20180936C11C7
:10F1B00090936D11A0936E11B0936F11C301A82DA0
:10F1C000BFAD8093701190937111A0937211B093A1
:10F1D0007311C0927411D0927511E0927611F09271
:10F1E00077110C94356583E080938C0A109291100E
:10F1F00060E083E50E94ED2581110C9435650F9444
:10F2000090420C94356583E50E945823882341F091
:10F210000E94DE258093C4060E94B32B0C943565B2
:10F2200081E00E94E1350C943565DED00C943565A3
:10F230000F94A15381110C9435650C94436E109179
:10F24000B2040F94D04D6093DD087093DE08809374
:10F25000DF089093E008112311F40C9435650E94A7
:10F26000F03684E50E942034812F0E94F6E880E287
:10F270000E94203484E690E10E9427340C94356586
:10F2800083E50E94A623882311F40C94A3700E94A6
:10F29000A1258B010C94A3700E94F53580EB9FE0B3
:10F2A0000E9427340C943565DF92EF92FF920F9302
:10F2B0001F93CF93DF93EC01E0904C0BF0904D0B3C
:10F2C0008AE0D82E6AE070E0CE010F94616F8C0165
:10F2D000009711F0FC011082CE010E942D2A81E0DE
:10F2E0000E9439630115110519F0E801D992EACF9E
:10F2F000C701DF91CF911F910F91FF90EF90DF90A9
:10F300000C942D2A4F925F926F927F928F929F92D0
:10F31000AF92BF92CF92DF92EF92FF920F931F9323
:10F32000CF93DF93CDB7DEB77C014DB65EB660906C
:10F330004C0B70904D0B8DB69EB66AE070E0C70125
:10F340000F94AF646C018C010E191F09892B21F4F5
:10F35000C7010F94C1648C01C80101962DB73EB757
:10F36000281B390B0FB6F8943EBF0FBE2DBF8DB7CB
:10F370009EB701965C01A801B7010F94E264F50104
:10F38000E00FF11F1082C5010E942D2A81E00E942A
:10F390003963C114D10451F076019FEFE91AF90ADB
:10F3A0000FB6F8949EBE0FBE8DBEC5CF0FB6F894B3
:10F3B0009EBE0FBE8DBEC3010E942D2A0FB6F894CB
:10F3C0005EBE0FBE4DBEDF91CF911F910F91FF909A
:10F3D000EF90DF90CF90BF90AF909F908F907F90F5
:10F3E0006F905F904F9008952F923F924F925F924F
:10F3F0006F927F928F929F92AF92BF92CF92DF9245
:10F40000EF92FF920F931F93CF93DF93CDB7DEB7A9
:10F41000C659D1090FB6F894DEBF0FBECDBF0E940A
:10F42000C72B8823D9F08091AB049091AC04A091B4
:10F43000AD04B091AE04AC01BD0132E176956795A3
:10F44000579547953A95D1F740FF22C020E040E01C
:10F4500070E060E08AE091EA0E943D92CA56DF4F78
:10F460000FB6F894DEBF0FBECDBFDF91CF911F91D5
:10F470000F91FF90EF90DF90CF90BF90AF909F9053
:10F480008F907F906F905F904F903F902F90089556
:10F4900022E0B695A795979587952A95D1F780FF95
:10F4A00003C00E941B94DACF4090B7085090B80870
:10F4B0006090B9087090BA088091C00881FF05C0BB
:10F4C0009091F70A98609093F70A82FB882780F959
:10F4D00080938F048091F01887FDC0CF85EC9BE06E
:10F4E00011DF80914708909148089E012F5F3F4FA0
:10F4F00079010097B1F09F938F938DEB9BE09F93E1
:10F500008F933F932F930F940B658091F0180F907A
:10F510000F900F900F900F900F9087FD9FCFC70116
:10F52000C3DE8091450890914608843B910514F410
:10F5300084EB90E09F938F9385EB9BE09F938F9359
:10F54000FF92EF920F940B658091F0180F900F903F
:10F550000F900F900F900F9087FD80CFC701A4DE12
:10F560008091F01887FD7ACF30911B08CF56DF4F7E
:10F570003883C159D04080911C08CE56DF4F888314
:10F58000C259D04020911D08CD56DF4F2883C35962
:10F59000D04030911E08CC56DF4F3883C459D0403C
:10F5A000209125083091260840912708509128087D
:10F5B000CF56DF4F6881C159D040782FCD56DF4FED
:10F5C0008881C359D040CC56DF4F9881C459D04070
:10F5D0000F94546C1B014C018DEA9BE093DE8091EB
:10F5E000C0085101640180FD14C0CF56DF4FA880D0
:10F5F000C159D040CE56DF4FB880C259D040CD5609
:10F60000DF4FC880C359D040CC56DF4FD880C45993
:10F61000D0408E010F571F4F23E041E0B501C601D6
:10F620000F944F609F938F9384EA9BE09F938F93F7
:10F63000FF92EF920F940B658091F0180F900F904E
:10F640000F900F900F900F9087FD08CFC7012CDE11
:10F650009501A601B101C4010F947B6E1816F4F454
:10F6600023E041E0B101C4010F944F609F938F9359
:10F670008AE99BE09F938F93FF92EF920F940B6523
:10F680008091F0180F900F900F900F900F900F90A7
:10F6900087FDE4CEC70108DE510164018091F018B6
:10F6A00087FDDCCE82E99BE02DDE87E08093010BB5
:10F6B0008093000B60914A0870914B0880914C0830
:10F6C00090914D088E010F571F4F21E041E00F949C
:10F6D0004F609F938F938091C00883FB882780F9A8
:10F6E000CB56DF4F8883C559D040CA56DF4F1882AA
:10F6F000C659D040CB56DF4F88819981C559D0403B
:10F70000C0969F938F9387E89BE09F938F93FF9280
:10F71000EF920F940B658091F0180FB6F894DEBF4E
:10F720000FBECDBF87FD9ACEC701BEDD21E041E00F
:10F73000B501C6010F944F609F938F938EE79BE0B6
:10F740009F938F93FF92EF920F940B658091F01827
:10F750000F900F900F900F900F900F9087FD7ECE1F
:10F76000C701A2DD8091C00884FF22C060914108DA
:10F7700070914208809143089091440823E041E051
:10F780000F944F609F938F9386E79BE09F938F9397
:10F79000FF92EF920F940B658091F0180F900F90ED
:10F7A0000F900F900F900F9087FD58CEC7017CDD12
:10F7B00080914508909146080097B1F09F938F93F0
:10F7C0008EE69BE09F938F93FF92EF920F940B65D1
:10F7D0008091F0180F900F900F900F900F900F9056
:10F7E00087FD3CCEC70160DD809149088823B9F0D0
:10F7F0001F928F931F921F9283E69BE09F938F939C
:10F80000FF92EF920F940B658091F0180FB6F89469
:10F81000DEBF0FBECDBF87FD21CEC70145DD6091A4
:10F820001708709118088091190890911A088E0194
:10F830000F581F4F23E041E00F944F60D82EC92E80
:10F840006091130870911408809115089091160822
:10F85000005F1F4F23E041E00F944F60CF92DF9293
:10F860009F938F9385E59BE09F938F93FF92EF92F9
:10F870000F940B658091F0180FB6F894DEBF0FBEA1
:10F88000CDBF87FDEBCDC7010FDD23E041E0CF56B3
:10F89000DF4F6881C159D040CE56DF4F7881C259C1
:10F8A000D040CD56DF4F8881C359D040CC56DF4F72
:10F8B0009881C459D0400F944F609F938F938BE4ED
:10F8C0009BE09F938F93FF92EF920F940B65809133
:10F8D000F0180F900F900F900F900F900F9087FDE2
:10F8E000BDCDC701E1DC809124088F93809123086E
:10F8F0008F9385E49BE09F938F93FF92EF920F94F9
:10F900000B658091F0180F900F900F900F900F9053
:10F910000F9087FDA3CDC701C7DC60911F087091D0
:10F920002008809121089091220823E041E00F9463
:10F930004F609F938F938CE39BE09F938F93FF92F5
:10F94000EF920F940B658091F0180F900F900F902D
:10F950000F900F900F9087FD81CDC701A5DC8CE043
:10F96000E9E2F8E0ADE3BAE001900D928A95E1F7A3
:10F970008CE0E5E3F8E0A0E7B6E001900D928A950F
:10F98000E1F780E00F94D80181E00F94D80182E084
:10F990000F94D8018091BF088093E31881E0809391
:10F9A000C4060E94B32B8EE498E09F938F938DE260
:10F9B0009AE39F938F93FF92EF920F940B65809140
:10F9C000F0180F900F900F900F900F900F9087FDF1
:10F9D00045CDC70169DC8091BE088F938091BD0839
:10F9E0008F938091BC088F938091BB088F937F92F7
:10F9F0006F925F924F9280E39BE09F938F93FF9271
:10FA0000EF920F940B658091F0180FB6F894DEBF5B
:10FA10000FBECDBF87FD22CDC70146DC1FCDBF92F3
:10FA2000CF92DF92EF92FF920F931F93CF93DF93CA
:10FA3000CDB7DEB7A0970FB6F894DEBF0FBECDBF2F
:10FA40000E94F73687FDE9C0482F61E081E00E94FF
:10FA500020948091010B8770873019F081E999E239
:10FA600051DC85E40E94A623882309F4E6C00E94A5
:10FA70000A256B017C0120E030E0A9010F947B6E28
:10FA800087FF04C0F7FAF094F7F8F094F7FAF094CF
:10FA9000F7F8F094C98EDA8EEB8EFC8E8CE0E2E7FC
:10FAA000F2E0DE01119601900D928A95E1F788E56A
:10FAB0000E94A623882351F040E050E0BA0188E577
:10FAC0000E94382569837A838B839C8389E50E9411
:10FAD000A623882351F040E050E0BA0189E50E9456
:10FAE00038256D837E838F8398878AE50E94A623BD
:10FAF000882351F040E050E0BA018AE50E943825A1
:10FB000069877A878B879C87C090B706D090B806A4
:10FB1000E090B906F090BA0685E50E94A6238823F6
:10FB200021F00E940A256B017C0120E030E0A90150
:10FB3000C701B6010F947B6E87FF04C0F7FAF094FB
:10FB4000F7F8F094F7FAF094F7F8F094CD8EDE8E93
:10FB5000EF8EF8A262E070E082E40E94C025B82E29
:10FB60008091E108811159C09E01235E3F4F41E021
:10FB7000BE016F5F7F4FCE0149960E94CB5B882309
:10FB800009F44BC06B2D81E00E941D5D70E060E0C8
:10FB900082E50E94C0258C0180E090E0A8ECB1E4F1
:10FBA0008D8B9E8BAF8BB88FC090BB06D090BC0660
:10FBB000E090BD06F090BE068CE40E94A623882348
:10FBC00021F00E940A256B017C0120E030E0A901B0
:10FBD000C701B6010F947B6E87FF04C0F7FAF0945B
:10FBE000F7F8F094C98ADA8AEB8AFC8A80E090E020
:10FBF000A0E7B1E48D879E87AF87B88B8091E1083D
:10FC0000882359F02B2DAE014B5E5F4FBE016F5E16
:10FC10007F4FCE010D960E943F58A0960FB6F894E4
:10FC2000DEBF0FBECDBFDF91CF911F910F91FF902F
:10FC3000EF90DF90CF90BF900895C12CD12CE12C94
:10FC400080E4F82E23CF2F923F924F925F926F92D3
:10FC50007F928F929F92AF92BF92CF92DF92EF925C
:10FC6000FF920F931F93CF93DF93CDB7DEB7C658A4
:10FC7000D1400FB6F894DEBF0FBECDBF8091AE0667
:10FC8000888B8091AB049091AC04A091AD04B091AD
:10FC9000AE04AC01BD0116E1769567955795479581
:10FCA0001A95D1F740FF07C120E030E0A90160912B
:10FCB000AF067091B0068091B1069091B2060F9494
:10FCC0007265811107C00E94F5358FEF97E00E94A1
:10FCD0002734C5C08AE50E94A623882339F10E94F3
:10FCE0000A252091660B3091670B4091680B50916B
:10FCF000690B0F94536C6B017C0120E030E040E213
:10FD000051ECC701B6010F947B6E87FD0AC020E05D
:10FD100030E040E251E4C701B6010F947265181655
:10FD200074F40E94F53582EF97E0D1CFC090560B66
:10FD3000D090570BE090580BF090590BDECF40E07D
:10FD400050E060EC7FE788E50E94382520915E0B4B
:10FD500030915F0B4091600B5091610B0F94536C8D
:10FD60002B013C0140E050E060EC7FE789E50E9418
:10FD700038252091620B3091630B4091640B5091B8
:10FD8000650B0F94536C4B015C016FEF89E40E948B
:10FD9000FF25182F6FEF8AE40E94FF25082FA3018B
:10FDA0009201C301B2010F940A6F811156C0A501DF
:10FDB0009401C501B4010F940A6F81114EC02091C6
:10FDC000A2063091A3064091A4065091A506C30156
:10FDD000B2010F94536C2091AF063091B006409160
:10FDE000B1065091B2060F94306D20E030E040E053
:10FDF0005FE30F94546C0F94986D162F2091A60614
:10FE00003091A7064091A8065091A906C501B401FA
:10FE10000F94536C2091B3063091B4064091B5060F
:10FE20005091B6060F94306D20E030E040E05FE383
:10FE30000F94546C0F94986D062F812F012E000C97
:10FE4000990B97FD0EC0099774F4802F002E000CBB
:10FE5000990B97FD0AC0099754F4193050F010E03F
:10FE600033C410E0F2CF18E0F0CF00E0F6CF08E0A6
:10FE7000F4CF0930A0F780E00E94952C29E012020F
:10FE8000F0011124E00FF11D07FDFA95EE0FFF1FA1
:10FE9000EE0FFF1FEB53F94FC082D182E282F38253
:10FEA0000E94FC2F88898823D1F281E00E94952C42
:10FEB0000F94E005D4CF79E0B695A79597958795EF
:10FEC0007A95D1F780FD0CC070E060E086E50E9475
:10FED000C0259A838983059730F08DEC97E0F7CEA3
:10FEE0000E94C32CBCCF60E084E40E94ED258F8784
:10FEF00040E050E0BA018AE50E9438256BA77CA754
:10FF00008DA79EA740E050E86BE376E483E50E946E
:10FF1000382520E030E040E752E40F94306D6093E4
:10FF20006A0270936B0280936C0290936D02009151
:10FF3000781110917911F801C080D180E280F380AE
:10FF400020E030E0A901C701B6010F94546CC558F8
:10FF5000DE4F6883CB57D140C058DE4F7883C058FE
:10FF6000D140CF57DE4F8883C158D140CE57DE4FA6
:10FF70009883C258D14020E030E040E251E40F9431
:10FF8000726587FF16C0C558DE4F1882CB57D14027
:10FF9000C058DE4F1882C058D140F0E2CF57DE4F34
:10FFA000F883C158D14021E4CE57DE4F2883C25890
:10FFB000D14020E030E04BE953E4C701B6010F9493
:10FFC000546C362E272EF82EE92E20E030E046E93C
:10FFD00053E40F947B6E181634F4312C212C56E91F
:10FFE000F52E63E4E62EF80184809580A680B78024
:10FFF00020E030E0A901C501B4010F94546C6B01FD
:020000021000EC
:100000008C0120E030E040E251E40F94726587FFFC
:1000100004C0C12CD12C00E211E420E030E04BE917
:1000200053E4C501B4010F94546C962EA72EB82E3C
:10003000C158DE4F9883CF57D14020E030E046E9E9
:1000400053E40F947B6E181654F4912CA12C46E9BE
:10005000B42EF3E4C158DE4FF883CF57D14088E483
:100060000E945823882309F488C20E940A250F940D
:10007000986DCD57DE4F688379838A839B83C358FD
:10008000D140CD57DE4F68817981C358D14077FF89
:1000900002C06F5F7F4F7595679571956195710986
:1000A00065567F4F072E000C880B990B0F947865CF
:1000B000562E672E782E892E9601A8010F947B6EFE
:1000C000181624F4C52CD62C072D182DC558DE4F34
:1000D0002881CB57D140C058DE4F3881C058D1401D
:1000E000CF57DE4F4881C158D140CE57DE4F58819F
:1000F000C258D140652D762D872D982D0F947B6E9B
:100100001816A4F0C558DE4F5880CB57D140C058C0
:10011000DE4F6880C058D140CF57DE4F7880C1583D
:10012000D140CE57DE4F8880C258D140852D962DC4
:10013000A72DB82D8B8B9C8BAD8BBE8BC601D801A8
:100140008F8B988FA98FBA8FCD57DE4F2881398139
:10015000C358D140B901330F880B990B0F947865C0
:10016000C558DE4F688379838A839B83CB57D14000
:100170009B01AC01B601C8010F94546C6B018C015A
:10018000292D3A2D4B2DC158DE4F5881CF57D140E4
:100190000F94726587FF08C09C2CAD2CB02EC158FF
:1001A000DE4F1883CF57D140C558DE4F28813981A3
:1001B0004A815B81CB57D140652D762D872D982DB7
:1001C0000F94546C6B018C01232D322D4F2D5E2D1D
:1001D0000F94726587FF04C03C2C2D2CF02EE12E6D
:1001E000832D922DAF2DBE2D8B8F9C8FAD8FBE8F0B
:1001F000892D9A2DAB2DC158DE4FB881CF57D140F4
:100200008F8F98A3A9A3BAA3BE01695E7F4FCE01C9
:1002100043960F94AA43882309F4F2C1BE01615E9C
:100220007F4FCE014B960F94AA43C82E882309F422
:10023000E7C12F89388D498D5A8D6F8D78A189A19D
:100240009AA10F94536C20E030E040E05EE30F94FD
:10025000D7654B015C012B893C894D895E896B8D8B
:100260007C8D8D8D9E8D0F94536C20E030E040E0AE
:100270005EE30F94D7656BA37CA38DA39EA38FA28F
:1002800098A6A9A6BAA689819A811816190674F4A7
:100290008BE997E00E9427348F85882321F081E93C
:1002A00097E00E9427348AE00E9420340E94BFF227
:1002B0000F944A0380E00E94952C80E090E0A0E239
:1002C000B1E4CD58DE4F88839983AA83BB83C3579B
:1002D000D14040E061E0CE018D589E4F0F9449041B
:1002E0008F85811143C02091AF063091B0064091B7
:1002F000B1065091B2066BA17CA18DA19EA10F9475
:100300007265811130C02091B3063091B4064091DE
:10031000B5065091B6066FA178A589A59AA50F9448
:100320007265811120C02091A2063091A3064091F0
:10033000A4065091A5066B897C898D899E890F94AE
:100340007265811110C02091A6063091A7064091D8
:10035000A8065091A9066F89788D898D9A8D0F9482
:100360007265882319F00E94C32C188A60E085E426
:100370000E94ED25882309F446C131E0C158DE4FC3
:100380003883CF57D1401B861C861D861E861A8A4D
:10039000412C512C20E8622E20EC722E1A89193043
:1003A0000CF04DC16B857C858D859E859B01AC01D4
:1003B0000F940A6F811143C1CC2009F42BC191E045
:1003C000C558DE4F9883CB57D14099E0392E91E044
:1003D000C92699E0199FD02C1124D394898B1989AF
:1003E0006A89131509F427C1062E000C770B880BB8
:1003F000990B0F9478652FA138A549A55AA50F949C
:10040000D7652F89388D498D5A8D0F94546C4B01C7
:100410005C01612F110F770B880B990B0F94786596
:100420002BA13CA14DA15EA10F94D7652B893C89DE
:100430004D895E890F94546C6B837C838D839E837E
:100440008F829886A986BA8689819A81892B91F0B4
:100450008DE797E00E9427348D2D0E94F6E88BE708
:1004600097E00E94273481E50E94F6E888E797E04C
:100470000E9427341F9281E58F931F92DF9221E61D
:1004800037E03F932F93EFE6F7E0FF93EF931F9250
:100490000E94C7D30FB6F894DEBF0FBECDBF8091C8
:1004A000FD0A882309F4C0C060E070E080EE90E4AB
:1004B000CD58DE4F488259826A827B82C357D14031
:1004C000298020E030E040EA50E40F94546CC95891
:1004D000DE4F688379838A839B83C757D140FE01AF
:1004E000E958FE4F7F018E010D581E4F222DC15835
:1004F000DE4F4881CF57D140BE01695F7F4FCE01AB
:1005000003960F94A4454B015C018B869C86AD86B7
:10051000BE86AC019B010F940A6F811189C00989C5
:100520008A8929E0020380011124080F111D87FD2B
:100530001A95000F111F000F111F81E090E08C0F22
:100540009D1F080F191FA50194016BA57CA58DA502
:100550009EA50F94546CF80166A777A780AB91AB6A
:10056000188A81E00E943B48D3948989C558DE4FA0
:10057000F881CB57D1408F0F31CFA601B80186E467
:100580000E9438252B013C01C558DE4F4881CB57CE
:10059000D140C058DE4F5881C058D140CF57DE4FB0
:1005A0006881C158D140CE57DE4F7881C258D140C2
:1005B0008CE40E9438256B8B7C8B8D8B9E8B4F8AB5
:1005C000588E698E7A8E492D5A2D6B2DC158DE4F6B
:1005D0007881CF57D14082E40E9438254B015C01DD
:1005E000432D522D6F2D7E2D82E50E9438256B8F75
:1005F0007C8F8D8F9E8F8F8E98A2A9A2BAA204CED7
:1006000081EB97E064CB83E0C158DE4F8883CF57FE
:10061000D140B9CEEFEFC558DE4FE883CB57D1407C
:1006200033243A9488E0D3CE60E070E0CB0140CF31
:1006300088890E94952C8A898F5F8A8BAFCE0F9410
:10064000E65280E00E94A12B882359F088890E94FD
:10065000952C80E090E0A0ECBFE78B879C87AD876E
:10066000BE876B857C858D859E859B01AC010F9433
:100670000A6F811111C08F85882309F440C0CE0113
:100680008F960E94E6608F85882319F088898823D9
:1006900019F081E00E94952C0F9431030E94A6244A
:1006A0000E94BFF281E497E00E9482790F94E005F6
:1006B0006B857C858D859E8511E09B01AC010F9437
:1006C0000A6F882309F4CBCB812FCA57DE4F0FB6B0
:1006D000F894DEBF0FBECDBFDF91CF911F910F9178
:1006E000FF90EF90DF90CF90BF90AF909F908F9052
:1006F0007F906F905F904F903F902F900895BE0134
:100700006D5E7F4FCE0183960E94103084E491E0AD
:10071000FE01BF96A5ECB6E001900D920197E1F7BE
:100720000E94FC2F90E080E0ACCFCF93DF93C0918C
:10073000580CC093C80A81E6C89FE0011124C65A2C
:10074000D34F8091F70A80FF07C00E94F036CE0198
:100750000F94A4520F949E52CE010E942D2A80E045
:10076000DF91CF910C9439638091E5188823F1F0E3
:100770002FEF3FEF3093600220935F028150809310
:10078000E518E1E1F9E1882351F08150990B2BE163
:10079000289FF001299FF00D1124E95BF64E8BE1B3
:1007A000ACE2B9E101900D928A95E1F72091E5184C
:1007B000211105C08091F01880648093F01881E0C9
:1007C00090E0A0E0B0E0211103C080E090E0DC0107
:1007D0008093B00A9093B10AA093B20AB093B30A7F
:1007E0001092A80A81E08093A60A83E080936502B4
:1007F000089581E08093F90A089582E08093F90AD0
:100800000895CF93DF93EC01642F70E090E080E0D7
:100810000F94786529EC38EC48EC5EE30F94306D6A
:1008200020E030E040E05FE30F94546C0F949D6D46
:100830006883DF91CF910895E091BE0A86E0E802D7
:10084000F0011124E357F54F8091AB0A90E09583B6
:10085000848308958F929F92AF92BF92CF92DF923E
:10086000EF92FF92CF936B017C0120E030E0A90171
:100870000F94726587FD9FC06DEB77E386E095E38B
:10088000A70196010F94546C6B017C0120E030E0CD
:1008900040E251E40F94D76520E030E048EC52E4A8
:1008A0000F94D7654B015C0120E030E0A901C7013E
:1008B000B6010F94726520E030E040EA50E487FF13
:1008C00004C020E030E040EA50ECC501B4010F94D0
:1008D000546C20E030E040E251E40F94306D0F940E
:1008E000986D6B017C018BE2F7FE09C0F094E094F7
:1008F000D094C094C11CD11CE11CF11C8DE28093EA
:100900006806C701B60120E137E240E050E00F94ED
:10091000BE6B8AE0882E912CA12CB12CCA01B901A2
:10092000A50194010F94BE6B605D60936906C701D9
:10093000B60128EE33E040E050E00F94BE6BCA01F0
:10094000B901A50194010F94BE6B605D60936A06C6
:10095000C701B60124E630E040E050E00F94BE6BE2
:10096000CA01B901A50194010F94BE6B605D60934B
:100970006B068EE280936C06C701B601A501940157
:100980000F94BE6BC62FCA01B901A50194010F9443
:10099000BE6B605D60936D06C05DC0936E0688E6B9
:1009A00096E0CF91FF90EF90DF90CF90BF90AF9007
:1009B0009F908F9008956DEB77E386E095EB60CF85
:1009C0008F929F92AF92BF92CF92DF92EF92FF925F
:1009D0006B017C0120E030E0A9010F94726587FD76
:1009E0006BC06DEB77E386E095E3A70196010F946A
:1009F000546C6B017C0120E030E040E251E40F9444
:100A0000D76520E030E040E251E40F94D7654B0118
:100A10005C0120E030E0A901C701B6010F947265C6
:100A200020E030E040EA50E487FF04C020E030E0FE
:100A300040EA50ECC501B4010F94546C20E030E062
:100A400040E251E40F94306D0F94986D9B018BE25E
:100A500037FF05C022273327261B370B8DE28093F3
:100A60006A06C90164E670E00F94266CCB01EAE0E7
:100A7000F0E0BF010F94266C805D80936B06C90186
:100A8000BF010F94266C282FCB01BF010F94266C59
:100A9000805D80936C068EE280936D06205D2093CE
:100AA0006E068AE696E0FF90EF90DF90CF90BF90C1
:100AB000AF909F908F9008956DEB77E386E095EB74
:100AC00094CF8F929F92AF92BF92CF92DF92EF928C
:100AD000FF92CF936B017C0120E030E0A9010F94DD
:100AE000726587FDD6C06DEB77E386E095E3A701DD
:100AF00096010F94546C6B017C0120E030E0A90159
:100B00000F94726587FFCAC0C701B601905820E0F4
:100B100030E040E251E40F94D76520E030E048EC4B
:100B200052E40F94D76520E030E040EA50E40F949F
:100B3000546C20E030E040E251E40F94306D0F94AB
:100B4000986D6B017C0160E280E4C81682E4D806EF
:100B50008FE0E806F1048CF0C701B60120E432E42E
:100B60004FE050E00F94BE6BCA01B9012AE030E0BB
:100B700040E050E00F94BE6B605D6093670660E2FA
:100B800080EAC81686E8D80681E0E806F1048CF011
:100B9000C701B60120EA36E841E050E00F94BE6B91
:100BA000CA01B9012AE030E040E050E00F94BE6B8A
:100BB000605D6093680660E280E1C81687E2D8064F
:100BC000E104F1048CF0C701B60120E137E240E016
:100BD00050E00F94BE6BCA01B9012AE030E040E05A
:100BE00050E00F94BE6B605D6093690660E288EE32
:100BF000C81683E0D806E104F1048CF0C701B60101
:100C000028EE33E040E050E00F94BE6BCA01B9011A
:100C10002AE030E040E050E00F94BE6B605D6093EE
:100C20006A06C701B60124E630E040E050E00F94C8
:100C3000BE6B8AE0882E912CA12CB12CCA01B9017F
:100C4000A50194010F94BE6B605D60936B068EE20C
:100C500080936C06C701B601A50194010F94BE6B89
:100C6000C62FCA01B901A50194010F94BE6B605D46
:100C700060936D06C05DC0936E0687E696E0CF91E7
:100C8000FF90EF90DF90CF90BF90AF909F908F90AC
:100C900008956DEB77E386E095EB29CF20E030E017
:100CA00040E251E4C701B60136CF8F929F92AF92D6
:100CB000BF92CF92DF92EF92FF92CF936B017C01B4
:100CC00020E030E0A9010F94726587FD93C06DEBC1
:100CD00077E386E095E3A70196010F94546C6B01CE
:100CE0007C0120E030E040E251E40F94D76520E041
:100CF00030E04AE754E40F94D7654B015C0120E0F3
:100D000030E0A901C701B6010F94726520E030E020
:100D100040EA50E487FF04C020E030E040EA50ECB5
:100D2000C501B4010F94546C20E030E040E251E47E
:100D30000F94306D0F94986D6B017C01C114D10438
:100D4000E104F10409F45BC0F7FE59C0F094E094AB
:100D5000D094C094C11CD11CE11CF11C8DE2809385
:100D60006906C701B60128EE33E040E050E00F9479
:100D7000BE6B8AE0882E912CA12CB12CCA01B9013E
:100D8000A50194010F94BE6B605D60936A068EE2CC
:100D900080936B06C701B60124E630E040E050E0E6
:100DA0000F94BE6BCA01B901A50194010F94BE6BEB
:100DB000605D60936C06C701B601A50194010F94B4
:100DC000BE6BC62FCA01B901A50194010F94BE6B79
:100DD000605D60936D06C05DC0936E0689E696E027
:100DE000CF91FF90EF90DF90CF90BF90AF909F900A
:100DF0008F9008956DEB77E386E095EB6CCF80E202
:100E0000AECFCF93DF93EC01CB01BA010F9478659D
:100E100020E030E048EC52E40F94306D2FE632E1F0
:100E200043E85AE30F94546C688379838A839B83E5
:100E3000DF91CF910895CF93DF93EC01CB01BA01FD
:100E40000F94786520E030E048EC52E40F94306D68
:100E50002FE632E143E85AE30F94546C68837983B8
:100E60008A839B83DF91CF9108950F94786520E06A
:100E700030E048EC52E40F94306D2FE632E143E865
:100E80005AE30F94546C1DCECF93DF93EC01CB014A
:100E9000BA010F94786520E030E040E251E40F940D
:100EA000306D2AE037ED43E25CE30F94546C6883C5
:100EB00079838A839B83DF91CF910895CF93DF93CA
:100EC000EC01CB01BA010F94786520E030E040E2FC
:100ED00051E40F94306D2AE037ED43E25CE30F9468
:100EE000546C688379838A839B83DF91CF910895C3
:100EF0000F94786520E030E040E251E40F94306DCB
:100F00002AE037ED43E25CE30F94546C59CDCF9364
:100F1000DF93EC01CB01BA010F9476652AE037ED3F
:100F200043E25DE30F94306D0F949D6D6883798388
:100F30008A839B83DF91CF910895CF93DF93EC0158
:100F4000CB01BA010F9478652AE037ED43E25DE307
:100F50000F94306D688379838A839B83DF91CF916F
:100F60000895CF93DF93EC01CB01BA010F9478651C
:100F7000688379838A839B83DF91CF910895CF9390
:100F8000DF93EC01CB01BA010F9478656883798314
:100F90008A839B83DF91CF910895CF93DF93EC01F8
:100FA000CB01BA010F94786520E030E048EC52E4C0
:100FB0000F94306D2FE632E143E85AE30F94546CFE
:100FC000688379838A839B83DF91CF9108950F94FF
:100FD000786520E030E048EC52E40F94306D2FE665
:100FE00032E143E85AE30F94546C34CCFC01518352
:100FF00040830895CF93DF93EC01CB01BA010F94A6
:101000007865688379838A839B83DF91CF91089584
:10101000CF93DF93EC01CB01BA010F94786520E008
:1010200030E04AE754E40F94306D27E137EB41EDAF
:1010300058E30F94546C688379838A839B83DF9190
:10104000CF9108950F94786520E030E04AE754E4AA
:101050000F94306D27E137EB41ED58E30F94546C5A
:1010600024CE8091AB0A9091AC0AA091AD0AB091C8
:10107000AE0A80934B0290934C02A0934D02B09322
:101080004E020895FC01A081B1811C92A281B3811E
:101090008C918F5F8C930280F381E02D90818CE0A6
:1010A000989F800D1124E5EAF8E113AE84AF08950E
:1010B000119800C09091020187FD909591709093D6
:1010C0000001119A00C000C0119800C09091020167
:1010D00086FD9095917090930001119A00C000C018
:1010E000119800C09091020185FD909591709093A8
:1010F0000001119A00C000C0119800C09091020137
:1011000084FD9095917090930001119A00C000C0E9
:10111000119800C09091020183FD90959170909379
:101120000001119A00C000C0119800C09091020106
:1011300082FD9095917090930001119A00C000C0BB
:10114000119800C09091020181FD9095917090934B
:101150000001119A00C000C0119800C080910201E6
:10116000817080930001119A00C000C0089590E042
:1011700080E008959091AE0681E089270C94952C2B
:10118000CF92DF92EF92FF926B017C0120E030E082
:10119000A9010F94726587FD26C06DEB77E386E0A9
:1011A00095E3A70196010F94546C6B017C0120E03C
:1011B00030E0A9010F94726520E030E040E05FE389
:1011C00087FF04C020E030E040E05FEBC701B601DC
:1011D0000F94546C0F94986DCB01FF90EF90DF90BB
:1011E000CF900D9449106DEB77E386E095EBD9CF66
:1011F0000F947865C5CFCB010D94491061E08BEA5F
:101200009AE00C940D2D69E379EA82E00D94C355C0
:101210006BE379EA81E00D94C3556DE379EA80E0F0
:101220000D94C3556FEE76EA83E00D94C355EF92AB
:10123000FF920F931F938EE9E82E81E2F82E10E0C3
:1012400000E020EA31E24AEB52E960EB71E285EB23
:1012500091E20F946E501F910F91FF90EF900895BF
:10126000EF92FF920F931F938091F60F09EE1FE00C
:10127000882311F006EF1FE089E5E82E81E2F82EC1
:101280002BE531E24CE054E967E671E28EE691E24B
:101290000F946E501F910F91FF90EF900895EF9271
:1012A000FF920F931F9380EAE82E80E2F82E10E061
:1012B00000E026E331E244ED56E962EA70E287EAB3
:1012C00090E20F946E501F910F91FF90EF90089550
:1012D000EF92FF920F931F93F12CE12C10E000E0AE
:1012E0002CEE3BE144E95AE863E27CE187E39CE1D0
:1012F0000F946E501F910F91FF90EF900895EF9211
:10130000FF920F931F93F12CE12C10E000E02CEEE4
:101310003BE141EA5AE863E27CE189E49CE10F9415
:101320006E501F910F91FF90EF900895EF92FF92F2
:101330000F931F93F12CE12C10E000E02CEE3BE129
:1013400045EE52E363E27CE186E69CE10F946E5049
:101350001F910F91FF90EF900895EF92FF920F93DE
:101360001F93F12CE12C10E000E02CEE3BE14FEF5D
:1013700052E363E27CE18EE69CE10F946E501F9194
:101380000F91FF90EF900895EF92FF920F931F93AC
:10139000CF93DF9300D01F92CDB7DEB72091BE0A66
:1013A0001C821B8280E2898380E22A302CF0822F0B
:1013B0006AE00F94056C805D8A83822F6AE00F9447
:1013C000056C905D9B838CEAE82E8BE1F82E8E01F4
:1013D0000F5F1F4F2EEA3BE14FE356E96CEB7BE1D9
:1013E0008FEB9BE10F946E500F900F900F900F902A
:1013F000DF91CF911F910F91FF90EF900895EF92A1
:10140000FF920F931F9381E1E82E8BE1F82E10E0FD
:1014100000E024E23BE146EA54E963E17BE18AE152
:101420009BE10F946E501F910F91FF90EF900895E4
:10143000CF92DF92EF92FF92CF93DF9300D01F9273
:10144000CDB7DEB76B017C0120E030E0A9010F943D
:10145000726587FD1BC06DEB77E386E095E3A7011E
:1014600096010F94546C69837A838B839C83CE019D
:1014700001960F94390C0F900F900F900F90DF9101
:10148000CF91FF90EF90DF90CF9008956DEB77E3D1
:1014900086E095EBE4CF0F94786520E030E040E201
:1014A00051E40F94306D2AE037ED43E25CE30F9492
:1014B000546CBECF84E00D94C44B83E00D94C44BB8
:1014C00082E00D94C44B70E090E080E00F9478656A
:1014D00029EC38EC48EC5EE30F94306D20E030E00E
:1014E00040E05FE30F94546C0F949D6D862F0D9434
:1014F0007E10CF93DF9300D01F92CDB7DEB784EF7D
:1015000091E0A0E0B0E089839A83AB83BC83BE0105
:101510006F5F7F4F88E70E946F320F900F900F90A0
:101520000F90DF91CF9108950E94B1320E94E53271
:101530000E94CB320E94E5320E94973210923B0A01
:1015400008950E94B1320E94FF320E94CB320E9465
:10155000FF320E94973281E080933B0A089563E94D
:1015600072E084E690E00F94612A70E060E08AE027
:1015700090E00F94612A6AEB72E084E690E00D94AB
:10158000612A0F944407EBCF8111E9CF68E270E044
:1015900080E991E00D94612A0E9416EEF5CF0F9438
:1015A0006522F2CF21E732EB47E25EE360915E060F
:1015B00070915F0680916006909161060F94306D86
:1015C00060931A1170931B1180931C1190931D113D
:1015D0000C94972BE7CF21E732EB47E25EE3609173
:1015E0005E0670915F0680916006909161060F948F
:1015F000306D6093EE107093EF108093F010909325
:10160000F110089521E732EB47E25EE360915A065C
:1016100070915B0680915C0690915D060F94D76592
:1016200060931611709317118093181190931911EC
:101630000C94972BE7CF21E732EB47E25EE3609112
:101640005A0670915B0680915C0690915D060F943E
:10165000D7656093EA107093EB108093EC10909331
:10166000ED1008958091560690915706A091580666
:10167000B09159068093121190931311A0931411F5
:10168000B09315110C94972BEDCF80915606909145
:101690005706A0915806B09159068093E610909392
:1016A000E710A093E810B093E9100895CF93DF936B
:1016B00000D01F92CDB7DEB70F94766569837A8329
:1016C0008B839C83CE0101960F94B60B0F900F90E5
:1016D0000F900F90DF91CF9108950F9476652AE0D7
:1016E00037ED43E25DE30F94306D0F949D6DDECFD7
:1016F000CF92DF92EF92FF92CF93DF9300D01F92B1
:10170000CDB7DEB76B017C0120E030E0A9010F947A
:10171000726587FD1BC06DEB77E386E095E3A7015B
:1017200096010F94546C69837A838B839C83CE01DA
:1017300001960F94B60B0F900F900F900F90DF91C2
:10174000CF91FF90EF90DF90CF9008956DEB77E30E
:1017500086E095EBE4CF0F9478652AE037ED43E21D
:101760005DE30F94306DC4CF0F947865C1CFCF92F5
:10177000DF92EF92FF92CF93DF9300D01F92CDB70D
:10178000DEB76B017C0120E030E0A9010F947265A7
:1017900087FD1BC06DEB77E386E095E3A70196011B
:1017A0000F94546C69837A838B839C83CE0101965A
:1017B0000F94B50C0F900F900F900F90DF91CF9179
:1017C000FF90EF90DF90CF9008956DEB77E386E088
:1017D00095EBE4CF0F947865CACFCF92DF92EF926A
:1017E000FF92CF93DF9300D01F92CDB7DEB76B018E
:1017F0007C0120E030E0A9010F94726587FD1BC0D9
:101800006DEB77E386E095E3A70196010F94546CA6
:1018100069837A838B839C83CE0101960F94AD0DEF
:101820000F900F900F900F90DF91CF91FF90EF905E
:10183000DF90CF9008956DEB77E386E095EBE4CFF2
:101840000F94786520E030E048EC52E40F94306D5E
:101850002FE632E143E85AE30F94546CBECF0C9468
:101860009CF20C949CF20C944EF20C944EF20C945C
:101870004EF20C944EF2CF92DF92EF92FF92CF9302
:10188000C82F0F94D04D6B017C0124EA30E74DE75F
:101890005FE3609121027091220280912302909176
:1018A00024020F94726587FD18C08AEF90E0A0E0D3
:1018B000B0E08C0D9D1DAE1DBF1D8093F005909373
:1018C000F105A093F205B093F305C0931A02CF91EE
:1018D000FF90EF90DF90CF90089580E090E0DC01E2
:1018E000E8CFCF92DF92EF92FF920F931F930F9466
:1018F000D04D0091C6051091C7052091C8053091C3
:10190000C9056B017C01C01AD10AE20AF30A9701EA
:10191000860137FD11C02091C50520952093C5058E
:101920006A547C4F8F4F9F4F6093C6057093C705D5
:101930008093C8059093C90581E09091C5059111E8
:1019400001C080E01F910F91FF90EF90DF90CF904A
:1019500008950F94E6521092FA0A109263020E94C0
:10196000F130882331F08AE099E190934A0A80931C
:10197000490A61E083E099E10E946B350D946B0B9D
:10198000BF92CF92DF92EF92FF920F931F93CF936C
:10199000DF936B01E9014A3009F4DFC0453109F0FA
:1019A0008AC0DB011296ED91FC911281C681D7812C
:1019B00080910201809582708093000100C0000038
:1019C00086E290E00197F0F7012F0295007F20E179
:1019D000B22EB10E88EF6CDB00C0000086E290E012
:1019E0000197F0F7103208F0A5C0812F807780684A
:1019F0005FDB802F5DDB00C0000086E290E0019796
:101A0000F0F780E855DB80E053DB00C0000086E2A1
:101A100090E00197F0F78AEF4BDB00C0000086E210
:101A200090E00197F0F77E01B0E1EB0EF11C8881A8
:101A3000807F3EDB89918295807F3ADBCE15DF0582
:101A4000B1F700C0000086E290E00197F0F71F5F59
:101A5000005F1B11BFCF8091020182708093000153
:101A6000D6011296ED91FC9180819281980F92831C
:101A70002181921708F0EDC194819F5F9483938137
:101A8000890F821710F08FEF820F8383458150E01A
:101A9000440F551F70E060E0868197810F94476F77
:101AA00081E0DF91CF911F910F91FF90EF90DF9038
:101AB000CF90BF900895FB0102811381423309F456
:101AC000CAC108F4D2C1463409F4BFC1473409F48D
:101AD000C7C14B3329F789812B81D80112966C91AC
:101AE000129713964C91213009F404C2233009F067
:101AF000E5C138EF380F582F91E0431708F490E014
:101B000041E0531708F040E031E0561708F430E0A8
:101B1000592F542B352319F4942309F4C1CFFA809B
:101B200030E0F901EE52FD4FD08022533D4FF901D4
:101B3000E080DDC180EE810F8068807FB9DA812F7F
:101B40008295807FB5DA00C0000086E290E00197C0
:101B5000F0F780E8ADDA80E857CF8091010182602C
:101B60008093010180910201827080930001809135
:101B70000101816080930101809102018170809355
:101B80000001099A119A80910201809582708093D8
:101B9000000100C0000086E290E00197F0F788E7BE
:101BA00090E0CEE9DFE0FE013197F1F70197D9F738
:101BB00088EF7EDA00C0000086E290E00197F0F73F
:101BC00080E276DA80E074DA00C0000086E290E01D
:101BD0000197F0F780E06CDA80E86ADA00C0000074
:101BE00086E290E00197F0F780E062DA80E160DA67
:101BF00000C0000086E290E00197F0F7CE01019767
:101C0000F1F7CE010197F1F7CE010197F1F7CE017F
